:10000000F01F001031C000002DC000002DC0000006
:100010002DC000002DC000002DC000000000000019
:100020000000000000000000000000002DC00000E3
:100030002DC00000000000002DC000005DB60000D3
:1000400085B6000085B6000085B6000085B60000C4
:1000500085B6000085B6000085B6000085B60000B4
:1000600085B6000085B6000085B6000085B60000A4
:1000700085B600002BC000002BC0000015B40000A6
:1000800045B600002DB6000015B60000FDB5000015
:100090002BC000008DB500002BC000002BC000005D
:1000A0002BC000002BC000002BC000002BC00000A4
:1000B0002BC000002BC000002BC000002BC0000094
:1000C0000223184A10B5116801240B431360202342
:1000D000154A164811680B431360154B1968014007
:1000E0001960196821431960124B13491A680240BC
:1000F0001A601A6822431A606C22104B1A60104B67
:1001000018680CF0AFF980220E4B120218600E4BEB
:1001100018600E4B20001A6080234022DB051A6015
:1001200010BDC0460480044080800440F8FCFFFFFE
:100130003040044034400440400D030018000040AB
:1001400018000010140000401000004000E100E022
:10015000802208201021094BD20510B511601860CB
:100160000023074814680C4201D0834204D105489B
:1001700098428041404210BD0133F3E7180000402F
:10018000FF0F0000FE0F0000802100222020134BF3
:10019000C90510B55A609A60DA600860104958685D
:1001A000012807D08A4203D1FFF7D2FF002010BDFB
:1001B0000132F4E78A42F7D000211A69013A5868FF
:1001C000FF2801D95868F2E71869904202D01A69ED
:1001D00059690A3158698142F1D1E5E718000010E8
:1001E000FF0F0000F8B5060003250C4B0C4C1F78E0
:1001F0000223A222A361013BE361E318DA77013312
:10020000DE77084BDF77FFF7BFFF0223FF3398420B
:1002100002D0013D002DEBD1F8BDC04668EC0000D6
:10022000180000101B000010064A537BD318D87327
:10023000537B0133DBB253735BB2002B01DA002333
:100240005373704728100010C143094A53699942FB
:1002500009D2591C08185169994200D27047516956
:100260008842FCD8F7E75169C91A8142FBD3F5E708
:10027000180000104023044A11680B431360012248
:10028000024B30331A707047808004401800001011
:10029000084B70B530331B7804000D00002B01D1E2
:1002A000FFF7E8FF182223689343236023681D4368
:1002B000256070BD180000100E4B70B530331B78F0
:1002C00006000D001400002B01D1FFF7D3FF701EB4
:1002D00002280AD8084B8000C25801231168AB409D
:1002E000012C04D10B43136070BD044AF5E7994318
:1002F0001160F9E71800001070EC0000FC3F00509E
:100300000F4B70B530331B7806000D001400002B26
:1003100001D1FFF7AFFF701E02280BD8094B8000F8
:100320001818C26801231168AB40012C04D10B439B
:10033000136070BD044AF5E799431160F9E7C046C0
:100340001800001070EC00000080005010B50C4C3C
:10035000606B002806D00220FFF744FF0238FF3808
:1003600043425841230038331A780A235106490F73
:100370004B430F210A4048349B186370E07110BD55
:1003800018000010F8B505000E000324A227094B41
:10039000B21C9A610022DA610133DF770133DD7725
:1003A000FFF7F2FE0223FF33984202D0013C002CFB
:1003B000EDD1F8BD1800001010B50120FFF712FFB5
:1003C0000223FF33984210D1094B01201A00383222
:1003D00014785863220706D0032203332240DA77C9
:1003E0000100FFF7CFFF200010BD01246442FAE7AF
:1003F0001800001070B50D4C636B002B13D0D5B2F4
:10040000E31CDD77130A251DDBB2EB77130CDBB29F
:10041000651D120E0634EB77E277FFF7B3FF023863
:10042000FF3843424341180070BDC0461800001019
:1004300010B5FFF7C1FF0220FFF7D4FE0223FF3300
:10044000984220D1104B1A00383212787F2A15D9E1
:100450005A6B002A12D01A000021082001242232EF
:100460009070D47051701170142226330638D970F0
:1004700018705C709A700731FFF784FF034A0421FB
:100480000920FFF7B7FF10BD1800001080808080A2
:10049000012210B510000B21FFF732FF00220B21C3
:1004A0000120FFF709FF012202210320FFF728FFA7
:1004B000002202210320FFF7FFFE10BD70B50600E9
:1004C0000024064D1835605D054B3100C01801341D
:1004D000FFF7DEFE0A2CF6D170BDC04670EC0000BE
:1004E00000400440F8B500240C4D22352B19665D00
:1004F0005F78012239003000FFF702FF023400224A
:1005000039003000FFF7D8FE142CEFD10020FFF7A0
:10051000D5FF0022024B5A65F8BDC04670EC0000C2
:1005200018000010F0B50125734B85B000900C0049
:100530009D6572B68022714B1202DA676C2200262A
:100540006F4B70481A60704B1968014019601A6847
:1005500004211A606D4B1A6802401A601A68002064
:100560001A602A00FFF7CCFE2A0004210020FFF7C2
:10057000A3FE2A0005210020FFF7C2FE2A00052164
:100580000020FFF799FE624B624D1E60FFF7AAFF45
:1005900031006148FFF77CFE31006048FFF778FECC
:1005A00031005F48FFF774FE31005E48FFF770FED0
:1005B00031005D48FFF76CFE5C4B1A685C4B1A60BB
:1005C000009B5A1E93413F225B429343594A9B181A
:1005D000594A13600423594A11680B431360584B5E
:1005E0002E601A685749584E0A401A602A680193CB
:1005F000A30700D47BE0EC235B0113432B60802333
:100600003360DB1833608023DB00336080235B01C1
:10061000336080231B013360009B002B52D00024E9
:100620004A4B4B4F1C604B4B21001C603800FFF7BE
:100630002FFE220009212000FFF762FE220009217F
:100640002000FFF739FE8021434A444813680B43DA
:10065000136007223B68763993433B603B68053A59
:1006600013433B60009B58430BF004FD03223C4BBB
:100670003C4918603C4B01981C603C4B1A603C4B59
:100680001A680A4080211A601A680A431A60802397
:1006900080229B0052023360326002687E391A4326
:1006A00002602A6813432B600123324A1360324AE6
:1006B0001160324A254913601460136010681842B3
:1006C000FCD00B6001222E4B52421A600A4BDB6DAC
:1006D000039362B630BFC046074B039ADB6D9A4264
:1006E00000D130BF0023044A936505B0F0BD8023DC
:1006F0001B0113432B608CE71800001004E100E09D
:1007000018000040F8FCFFFF304004403440044033
:100710000480044004820440084004400040044037
:10072000AC400440144004401C4004403882044063
:1007300034820440FF1800003082044010ED00E0D5
:10074000008204407FE2FFFF00E100E004C00040BF
:10075000644004400400014080800440841E000086
:1007600018C000400FF0FFFF08C0004014C0004058
:100770003CC0004078800440708004407480044095
:1007800008820440F7B50F4D6C6D002C18D1102075
:10079000FFF794FE0C4B22330193019B0022E65C91
:1007A0001B195F7830003900FFF7AAFD02340122DF
:1007B00039003000FFF780FD142CEED101236B656A
:1007C000F7BDC0461800001070EC000070B572B69E
:1007D00080248020802180250F4BC0001A1D6400DA
:1007E0004901D567D467D067D167C02252009D50B8
:1007F0009C5098509950094A094913680B4013605E
:10080000AC22084B52011A60FFF7BCFF0022064BD6
:100810001A6662B670BDC04600E100E00482044082
:100820007FEAFFFF0882044018000010F8B50700B7
:10083000FFF7A8FF002F09D0012207210220FFF7B0
:100840005FFD002207210220FFF736FD124E330024
:1008500030331B78002B01D1FFF70CFD0F4D012425
:100860002B681B0509D530363378002B01D1FFF7F3
:1008700001FD01242B68DB0A9C43002F09D00022D4
:1008800007210220FFF73CFD012207210220FFF78C
:1008900013FD2000F8BDC04618000010FC3F0050BA
:1008A000F0B5012089B0FFF7C1FF012304930028B0
:1008B0004FD104001D0004902A4E630001330393BE
:1008C000330037002233E25C1B195B780192190078
:1008D0002A0001980293FFF713FD00220299019864
:1008E000FFF7EAFC204B343630333C37069607934B
:1008F0003B787E780593079B1B78002B01D1FFF78F
:10090000B9FC059B032B0DD818000BF095FE0225B2
:100910002729164B2A00B2401B6813405A1E9341E8
:10092000002B02D16B461B7B0493039B023F0133D8
:100930000393069B9F42DBD1002202990198FFF7A7
:10094000DFFC02342A0002990198FFF7B5FC142C51
:10095000B2D1049809B0F0BD054BDBE7054BD9E7F0
:10096000054BD7E770EC000018000010FC3F00506A
:10097000FC3F0150FC3F0250FC3F0350F8B54A00D9
:10098000070004001E48520D1518132D18DC002D09
:1009900009DACB0FDB070022691C01D119490B438F
:1009A0001900100017E0184E2E4132000A4014437F
:1009B00012D0802212032A415318B3430022EFE7DA
:1009C000332D0BDD8023DB009D4205D13A000B0067
:1009D00038000CF0C7FB07003800F8BD01260B48B3
:1009E00076421218D6403E42F6D03322551B323A98
:1009F000AA40D219BA42A44164420B19B243CFE7CC
:100A000001FCFFFF0000F03FFFFF0F00EDFBFFFFC9
:100A100007B5002200280CD090231B0600920193FA
:100A200000980199802300225B050DF0C1FA03B004
:100A300000BD80235B05F1E707B5002200280CD03C
:100A4000F0231B060092019300980199E0230022F5
:100A5000DB050DF0ADFA03B000BDE023DB05F1E7E7
:100A6000F0B5D34A4B0089B007000E000C005B08BC
:100A700093423CD9CF4A934200D8F5E1CE4A934203
:100A80000DD90B031B0B034304D002000B000CF029
:100A900069FB0EE000290EDA0027C84E0BE0C84AB9
:100AA000C84B0BF0FDFD002800D1DDE10020FFF771
:100AB000C3FF07000E003800310009B0F0BDC24A84
:100AC000C24B380031000CF04DFB002200230BF02C
:100AD000D3FD0028E0D1BE4ABE4B380031000DF0F6
:100AE00067FA002C00DAA8E00024BB4DA7E0BB4A5F
:100AF000934200D8C5E0BA4A9342ECD8B94ABA4BFF
:100B0000002900DA8FE00DF0C5FC012304000D0080
:100B10000093B64AB64B02920393029A039B2000BD
:100B200029000DF0B7FC02000B0007000E002000AA
:100B300029000DF0AFFC029A039B0DF0ABFC029074
:100B400003910022A44B380031000DF031FA0490DB
:100B5000059102000B00380031000DF029FA040065
:100B60000D00A44AA44B0DF023FAA44AA44B0CF0A8
:100B7000F9FA22002B000DF01BFAA24AA24B0DF04D
:100B800089FC22002B000DF013FAA04AA04B0CF0B8
:100B9000E9FA22002B000DF00BFA9E4A9E4B0DF055
:100BA00079FC22002B000DF003FA00229B4B0CF085
:100BB000D9FA02000B0006900791049805990DF0F0
:100BC000F7F902000B00002095490DF063FC0200CC
:100BD0000B0004900591069807990DF05BFC049AB0
:100BE000059B06900791380031000DF0E1F90200F5
:100BF0000B0000208B490DF04DFC02000B00069805
:100C000007990CF0CBFD2B0022000DF0D1F9009BD1
:100C1000002B4CD102000B00380031000DF0C8F958
:100C200022002B003AE00CF09DFA01235B42009376
:100C300004000D006D4A7C4B6DE700247B4D0200E3
:100C40000B00200029000CF08DFA0DF06BFF0090D6
:100C50000DF09EFF634A644B029003910DF0A8F9DA
:100C600002000B00380031000DF014FC5F4A040054
:100C70000D00029803995E4B0DF09AF902900391D2
:100C80004BE700216A4A0091934200D959E7694A2B
:100C9000694B31000CF066FA02000B000DF0FAFB14
:100CA00002000B00380031000DF0F4FB01E7029A5E
:100CB000039B0DF0EFFB3A0033000DF079F9029A37
:100CC000039B0DF0E7FB2B0022000DF0E3FB009BE4
:100CD00004000D0001330CD102000B00380031007C
:100CE0000DF0D8FB00223C4B0DF062F900223A4B8C
:100CF000DAE7009B012B26D10022504B380031004F
:100D00000BF0BAFC002811D00022334B3800310020
:100D10000CF028FA02000B00200029000DF0BAFBAD
:100D2000C02300221B060DF043F9C2E622002B006F
:100D3000380031000DF0AEFB02000B000CF012FA8F
:100D40000022364BA3E6009B1B050293009B013358
:100D5000392B0FD93A0033000DF09CFB02000B0039
:100D600000202E490DF096FB029C0022631819000A
:100D70002A4B99E7009B132B62DC8023009A9B038C
:100D800013410020254AD11A009001913A00330006
:100D9000200029000DF07EFB02000B000098019955
:100DA0000DF078FB029C070063181E0083E6C04626
:100DB00079684340412E8640FFFFEF7F0000F0BF7F
:100DC000EF39FAFE422E864059F3F8C21F6EA50194
:100DD000FE822B654715F73F0000E03F422ED63FCD
:100DE000B1A2F03F0000E0FE422EE63F763C7935AE
:100DF000EF39EA3D2DC3096EB7FD8ABE3952E6864A
:100E0000CACFD03EB7DBAA9E19CE143F8555FE1936
:100E1000A0015A3FF41011111111A13F0000F03F41
:100E20000000084000001840EF39EABD0000E0BFB4
:100E3000FFFF8F3C9C7500883CE4377E0000D0BFEC
:100E400000980E490022091A0B05200029000CF019
:100E500089F902000B00380031000DF01BFB002265
:100E6000074B0CF07FF99DE7002C00DA27E6054AD6
:100E7000054B380031000DF09BF835E6FF0300000C
:100E80000000F03FFE822B654715F73FF0B54A00A2
:100E90005708914A89B005000C00CE0F97422DD912
:100EA0008E4A974211D90B031B0B034306D0020055
:100EB0000B00280021000CF055F910E0002E00D0A6
:100EC00006E12800210009B0F0BD854A854B0BF0F2
:100ED000E7FB0190002805D00020FFF7ADFD0500DD
:100EE0000C00EEE7804A814B280021000BF0C4FB88
:100EF000002807D00198FFF78BFDF0E77C4B9F425D
:100F000000D89BE07B497C4BF2008F426FD89F1842
:100F10003A6C7B6C280021000DF0BCFA3B6D7C6DB7
:100F2000012502900391AD1B04930594AB1B019323
:100F3000049A059B029803990DF0ACFA05000C0089
:100F40002A002300280021000DF032F806000F00CF
:100F50006A4A6B4B0DF02CF86A4A6B4B0DF09AFA0B
:100F600032003B000DF024F8684A694B0CF0FAF8A7
:100F700032003B000DF01CF8664A674B0DF08AFA10
:100F800032003B000DF014F8644A654B0CF0EAF8AF
:100F900032003B000DF00CF802000B00280021008D
:100FA0000DF078FA0B00020006000F002800210067
:100FB0000CF0FEFF019B06900791002B53D180237C
:100FC0000022DB05300039000DF064FA02000B004E
:100FD000069807990CF0E2FB2A0023000DF05AFA5C
:100FE00002000B0000204F490DF054FA77E79E18DD
:100FF00028004D4A4D4B21000CF0DAFF326E736E23
:101000000CF0B0F80DF08EFD01900DF0C1FD484AD6
:10101000484B06000F000CF0CBFF02000B0028002D
:1010200021000DF037FA444A02900391434B3000FF
:1010300039000CF0BDFF0490059179E7404B9F42C9
:101040000CD8404A404B0CF08DF80022354B0BF089
:1010500027FB002805D00022324B2AE7002301930A
:101060006EE701906CE7802132003B000020C9054B
:101070000DF010FA02000B00069807990CF08EFB99
:1010800002000B00049805990DF004FA029A039BE4
:101090000DF000FA02000B00002022490DF0FAF9D1
:1010A0002A4B019A9A4205DB019C0500260573181C
:1010B0001C0006E7FA25AD00AC46019C0022644402
:1010C000260573181900B8235B040CF071FF06E7BE
:1010D00000252C00F5E6C046412E8640FFFFEF7F3D
:1010E000EF39FAFE422E864051302DD5104987C087
:1010F000422ED63FB1A2F03F70EC0000D0A4BE72E9
:101100006937663EF16BD2C541BDBB3E2CDE25AFD3
:101110006A56113F93BDBE166CC1663F3E5555558C
:101120005555C53F0000F03FFE822B654715F73F40
:101130000000E0FE422EE63F763C7935EF39EA3D8D
:10114000FFFFEF3D9C7500883CE4377E03FCFFFF0A
:10115000F0B5BA4B8DB00E00994223DC4B005B0812
:10116000034307D1002200230020B5490CF016FBF1
:101170000DB0F0BD002906DA02000B000DF08AF96F
:1011800000220023F2E7AF4B00220CF011FF3623C0
:101190000E005B42AC4A964206DD02000B000BF0EB
:1011A000E1FFE5E70023F5E7A84C321512193603F5
:1011B000A74CD218330B02931C1980235B032340E6
:1011C000A44C029D5C401B159B18254300930022F4
:1011D000A04B29000DF05EF9029B060002331B03B1
:1011E0000F001B0B0022022B64DC00230BF03EFAE5
:1011F000002819D0009B002B00D11CE118000DF035
:10120000C7FC954A954B04000D000CF0D1FE944AA2
:1012100006000F00934B200029000CF0C9FE0200CD
:101220000B0030003900BAE78F4A904B300039008C
:101230000CF0BEFE02000B0000208D490DF02AF9D3
:10124000320004000D003B00300039000CF0B0FE0D
:101250000B000200290020000CF0AAFE009B029067
:101260000391002B06D102000B00300039000DF075
:1012700011F97DE700980DF08BFC774A774B04005D
:101280000D000CF095FE764A00900191754B200000
:1012900029000CF08DFE02000B00029803990DF05E
:1012A000F9F832003B000DF0F5F802000B00009851
:1012B0000199DCE78023DB050BF054FF02000B00F3
:1012C000300039000CF06AFA0490059100980DF096
:1012D0005FFC049A059B06900791100019000CF022
:1012E00067FE644A029B944663440B9302000B0022
:1012F000089009910CF05CFE04000D005E4A5F4B03
:101300000CF056FE5E4A5F4B0BF02CFF22002B00C8
:101310000CF04EFE5C4A5D4B0BF024FF22002B00CC
:101320000CF046FE5A4A5B4B0BF01CFF089A099BD7
:101330000CF03EFE584A08900991584B20002900B5
:101340000CF036FE564A574B0BF00CFF22002B00D8
:101350000CF02EFE544A554B0BF004FF22002B00DC
:101360000CF026FE02000B00089809990BF0FAFE1B
:10137000029A4F4B04009B1A0B9A0D001343002B4B
:1013800034DD00223A4B300039000CF011FE3200FF
:101390003B000CF00DFE0290039102000B002000B8
:1013A00029000BF0DFFE049A059B0CF001FE009B68
:1013B00004000D00002B06D102000B0002980399D7
:1013C0000DF068F84FE7244A244B069807990CF073
:1013D000EFFD234A0090019106980799214B0CF0EC
:1013E000E7FD22002B000BF0BDFE54E702000B00CE
:1013F000300039000DF04EF8049A059B0CF0D8FD32
:10140000009B04000D00002B02D102000B002CE712
:10141000114A124B069807990CF0CAFD104A009029
:101420000191069807990F4B0CF0C2FD02000B00CA
:101430002000290033E70020002199E6FFFF0F007C
:10144000000050C300005043FFFFEF7F01FCFFFF8F
:10145000645F09000000F03F0000E0FE422EE63F1E
:10146000763C7935EF39EA3D555555555555D53FBB
:101470000000E03F86EBF9FF44523EDF12F1C23F2D
:10148000DE03CB966446C73F599322942449D23F4A
:10149000935555555555E53F9FC678D0099AC33F9A
:1014A000AF788E1DC571CC3F04FA97999999D93FB1
:1014B00051B80600434218434900C00F4908014390
:1014C0000348401A414201430120C90F401A7047A6
:1014D0000000F07F03004042184349004908C00F54
:1014E00008430249081AC00F7047C0460000F07F49
:1014F000564BF0B51A0085B005000C000A409A4220
:101500000FD102000B000CF053FD02000B0028006D
:1015100021000BF027FE05000C002800210005B07B
:10152000F0BD0200002910DC4B005B080343F4D03F
:101530000020814200D180E00B0028000CF0AAFFBF
:1015400002000B000CF02AF9E5E7081575D0404BB6
:101550000903C0188023090B5B031943C30703D594
:10156000D30F4900C91852000024431049000393C7
:10157000D30FCB188021162520005200890346186E
:101580009E4202DC70189B1B6418D60F5B00013D65
:101590009B1952004908002DF1D1202680272900EF
:1015A00001963F067E19B446834202DC14D196426E
:1015B00012D865466646ED190290002E03DAEE4316
:1015C000F60F861902961B1A6245804140421B1A8B
:1015D0006046121A0298C919D60F5B00F318019ED3
:1015E0005200013E7F080196002EDBD1134303D049
:1015F0004B1C27D131000134164B6010C01849082C
:10160000E30702D580231B061943039B0D001C052D
:1016100023181C0081E7D10A153B52050029FAD096
:101620008024640321420AD020241600241AE640B4
:10163000451E82403143581B89E70023EEE74900ED
:101640000130EFE7012301319943D5E70000F07F36
:1016500001FCFFFF0000E03FF0B54F005E008DB0E1
:101660007F087608B74205DA3C0037002600040000
:1016700010002200330000920193F0223900040090
:101680003D00BB1B9204934206DD009A019B0BF0C8
:1016900069FD04000D0017E0804B9F4200DCA1E0D3
:1016A0007F4B9F4214DD3F033F0B074305D0009A59
:1016B000019B0BF057FD04000D007A4B5E40009B30
:1016C0001E4301D1009C019D200029000DB0F0BDFA
:1016D000754BF618FF18009A019B33000092019396
:1016E00096233D009B000893704B9E421BDC704B81
:1016F0009E4200DD78E0009B3343E5D000980199DD
:1017000000226C4B0CF054FC002200900191694BBC
:10171000200029000CF04CFC674A040094460D00A0
:10172000089B63440893009A019B200029000CF059
:10173000B1FE0200099102900B00049100980199FA
:101740000AF09AFF002200285ED03B00100039000A
:1017500016000CF02DFC009B049005919C46009A0D
:10176000019B8020614600068446029101996144F4
:101770000391029803990CF01BFC32000090019138
:101780003B00200029000BF0EDFC32000290039199
:101790003B00200029000CF07DFE02000B000298A7
:1017A00003990CF005FC02000B00009801990CF065
:1017B00071FE02000B00049805990CF06BFEFFF718
:1017C00097FE089B04000D00002B00D17CE7002051
:1017D0003A4A1B0599180B000200290020000CF062
:1017E000E7FB56E700237EE79623354A9B059446A0
:1017F000FF18F618089B3D0063440893009A019B6C
:101800003300009201938EE7330080210692079304
:10181000002249037B180698079916001F000CF058
:10182000C7FB0A900B918020000684460299049B16
:1018300004910999029A61440591049805990CF064
:10184000B7FB2200029003912B00200029000BF02F
:1018500089FC32003B000CF01DFE009A019B0CF04D
:10186000A7FB069A079B04000D00009801990CF055
:1018700011FE32003B000CF09BFB02000B0020002D
:1018800029000BF06FFC02000B00029803990CF08A
:1018900001FE02000B000A980B998EE70000305FF2
:1018A000FFFFEF7F0000F07F000080DAFFFFAF2036
:1018B000FFFF0F000000D07F02FCFFFF0000F03FA1
:1018C000A8FDFFFFF0B589B002920393464A4B0092
:1018D00005000C005B08934203DC0DF023F900289F
:1018E0004CD02A002300280021000CF061FB0600E8
:1018F0000F0002000B00280021000CF059FB3B4AAE
:10190000009001913A4B300039000CF051FB394AFC
:10191000394B0CF0BFFD32003B000CF049FB374A5D
:10192000374B0BF01FFC32003B000CF041FB354AFB
:10193000354B0CF0AFFD32003B000CF039FB334B64
:10194000334A0BF00FFC0E9B04900591002B19D12C
:1019500002000B00300039000CF02AFB2D4A2E4B00
:101960000CF098FD009A019B0CF022FB02000B008A
:10197000280021000BF0F6FB05000C0028002100D8
:1019800009B0F0BD002202980399244B0CF010FB23
:10199000049A059B06900791009801990CF008FBAA
:1019A00002000B00069807990CF074FD32003B0012
:1019B0000CF0FEFA029A039B0CF06CFD154A06002F
:1019C0000F0000980199144B0CF0F2FA02000B0082
:1019D000300039000BF0C6FB02000B00280021008C
:1019E0000CF058FDC8E7C046FFFF3F3E7CD5CF5AFC
:1019F0003AD9E53DEB9C2B8AE6E55A3E7DFEB15790
:101A0000E31DC73ED561C119A0012A3F1111813FD5
:101A1000A6F81011495555555555C53F0000E03FF2
:101A2000F8B50022324B0CF0C3FA00220023060066
:101A30000F000AF01BFE002854D100222D4B30006D
:101A400039000AF013FE00284FD132003B0030006D
:101A500039000CF0ADFA04000D00274A274B0CF0BA
:101A6000A7FA274A274B0CF015FD22002B000CF09B
:101A70009FFA254A254B0BF075FB22002B000CF03A
:101A800097FA234A234B0CF005FD22002B000CF0A3
:101A90008FFA214A214B0BF065FB22002B000CF042
:101AA00087FA1F4A1F4B0CF0F5FC22002B000CF0AC
:101AB0007FFA1D4A1D4B0BF055FB22002B000CF04A
:101AC00077FA1B4A1B4B0CF0E5FC22002B000CF0B4
:101AD0006FFA194A194B0BF045FB32003B000CF032
:101AE00067FAF8BD00200021FBE700201449F8E761
:101AF0000000E03F0000D03F98456D69B8D1B93F84
:101B0000722CC67097F7E63FA79ED5E9358F0E4039
:101B10000CD7D1DD74302E40CB905148830745401F
:101B2000437562CE2C2D53406EAA7567BC66544037
:101B300052BE25E6BCAB4440182D4454FB2119404D
:101B40000000F03FF8B505000C00FFF7B3FC0028DB
:101B500000D0E3E000220023280021000AF08CFDE1
:101B600000280BD0280080252D066119FFF7EAFF19
:101B70004919002200230BF0F5FAF8BD00220023DA
:101B8000280021000AF072FD061E02D0002001008C
:101B9000EFE70022644B280021000AF067FD0028CF
:101BA00000D0BEE00022614B280021000AF05EFD5B
:101BB0000028EBD15E4A60002300400890420BDD14
:101BC0002A00280021000BF0CDFA02000B000BF0D8
:101BD000E5FD05000C000FE08027E20F2900D20789
:101BE000FF05B84215DC07D1002D12D1D20FD3006A
:101BF000504AD218156F546F00224B4B2800210019
:101C00000AF044FD002857D028002100FFF708FF04
:101C1000AFE780241B031B0B64031C43464B0015DA
:101C2000C018464BE318002816D1002B00DA230019
:101C30001C0001200C43D9D0414CA3421ADD414C79
:101C4000A0421DDB3D4C0D001B191A433E4BC01832
:101C5000000502431400CFE7002B05DA6400CB0F28
:101C60001C1949000138DCE71C000C43BED05B00A6
:101C7000CC0FF5E7CD0F5B005B1949000138DCE7BD
:101C8000241A142C0ADC314DE14040191D00854016
:101C900023410D431A43110028009AE71F2C07DC4B
:101CA000E1402A4C001983400B431D001300F1E76B
:101CB0002749081A0341F8E700221C4B280021009D
:101CC0000AF0E4FC002806D02A002300002017496F
:101CD0000CF0E0FB9AE700221E4B280021000AF0DE
:101CE000D5FC002200280AD0280021000F4B0CF060
:101CF000D1FBFFF795FE80231B06C91839E7802327
:101D00002800DB0521000AF0C1FC002800D13DE7D6
:101D100080212A0023000020C905E8E700200E49A1
:101D200027E73000014924E70000E03F0000F03FD2
:101D3000FFFFEF7F70EC000000FCFFFF0000F0FFF2
:101D4000FFFF0F0002FCFFFFFF0300001E04000066
:101D5000E2FBFFFF0000F83F0000F87FF0B587B01E
:101D6000049205934B005B080093009A484B0500D2
:101D70000C009A4204DC0CF0D5FE002800D184E06F
:101D80002A002300280021000CF012F90022414B08
:101D900006000F000CF00CF93F4A029003913F4BF4
:101DA000300039000CF004F93D4A3E4B0BF0DAF9F3
:101DB00032003B000CF0FCF83B4A3C4B0CF06AFB59
:101DC00032003B000CF0F4F8394A3A4B0BF0CAF9F8
:101DD00032003B000CF0ECF8374A384B0CF05AFB61
:101DE00032003B000CF0E4F8354A364B0BF0BAF900
:101DF00032003B000CF0DCF832003B000CF0D8F86D
:101E0000049A059B06000F00280021000CF0D0F872
:101E100002000B00300039000CF03CFB2A4B009A0A
:101E200004000D009A420DDC02000B000298039999
:101E30000CF030FB020000200B0024490CF02AFBC0
:101E400007B0F0BD224B009A00269A421BDC13001B
:101E5000204A944663441F0032003B0000201B4987
:101E60000CF018FB320000900191029803993B009E
:101E70000CF010FB22002B000CF00CFB02000B00FE
:101E800000980199DAE7144FE6E700200F49D7E7F9
:101E9000FFFF3F3E0000E03FD43888BEE9FAA8BD0E
:101EA000C4B1B4BD9EEE213EAD529C804F7E923EA9
:101EB0009015CB19A001FA3E7751C1166CC1563F5F
:101EC0004C5555555555A53F3233D33F0000F03F93
:101ED0000000E93F0000E0FF0000D23F70B51400B1
:101EE0004A000B00520D0DD14B005B0803430FD08D
:101EF000224B00220CF05CF8214B9C4209DA214A6B
:101F0000214B17E0214DAA4207D102000BF02AF91C
:101F100070BD0B004A00520D363A1D4DAC420CDD2F
:101F2000C90F1C48C907084303001B4A19001000C9
:101F3000184B194A0CF03CF8EAE7A218174CA242D9
:101F4000EEDC002A05DD164C120523401343190070
:101F5000DEE71400353408DAC90F0B48C907084317
:101F60000300084A19001000C9E70D4C363223401F
:101F700012051A4311000B4B0022DBE7000050430F
:101F8000B03CFFFF59F3F8C21F6EA501FF07000028
:101F900050C300003CE4377E9C750088FE070000BB
:101FA000FFFF0F800000903CF0B54B00394A5B0DFD
:101FB00085B09E180D0004000390132E33DC002E14
:101FC00014DA354A354B0BF0CDF8002200230AF025
:101FD00067FB002807D0002D58DA6B005B081C4314
:101FE00001D000242E4D2000290026E02D4F37413E
:101FF0003B000B40034320D000900191264A274B21
:10200000009801990BF0AEF8002200230AF048FB7B
:102010000028E8D0002D03DA80235B033341ED185C
:10202000BD430024DFE7332E09DD8023DB009E4221
:1020300003D102000B000BF095F805B0F0BD0127AD
:10204000194A7F429B18DF403842F6D00090019138
:10205000114A124B009801990BF084F800220023DA
:102060000AF01EFB0028BED0002D02DA142E02D189
:102070000135BC43B7E734239E1B333BB340E41820
:10208000039B9C429B415B42ED18F2E70024250034
:10209000A9E7C04601FCFFFF9C7500883CE4377E41
:1020A0000000F0BFFFFF0F00EDFBFFFFF0B5D14CCC
:1020B000A54408900991D01E1821140002930AF03B
:1020C000D1F91823421C5B4253431B19002400938F
:1020D000029B05905D1EDF1C451BC74BAE00F6182A
:1020E000EC4200D5F1E0A300F0580CF051FDE30004
:1020F00022AAD318013418605960A742F0DA0024EC
:10210000029BDB00D3180793079B00261D190023B1
:1021100000270693069B089ADB00E91A0839D318B2
:102120001A685B68086849680BF042FF02000B0000
:10213000300039000BF016F8069B060001330693B9
:10214000069A029B0F009342E4D172AB1B1908342C
:102150001E605F60282CD7D10426059BA64A9B00F1
:102160009B180A93370072AAF300D3181C685D68A5
:102170000EA9B3005B1805930B9200229F4B200021
:1021800029000BF015FF0CF0CDFC0CF001FDBB009D
:102190005B42079300229A4B029003910BF008FFD9
:1021A00002000B00200029000CF074F90CF0BAFCBE
:1021B000059B079A013F98500B9AFB00D3181A68A9
:1021C0005B68029803990AF0CDFF04000D00002F10
:1021D000D3D1009AFFF782FEFF2300229B05040063
:1021E0000D000BF0E5FEFFF7DFFE0022854B0BF044
:1021F000DFFE02000B00200029000CF04BF90D005F
:1022000004000CF08FFC07900CF0C2FC0B000200E5
:10221000290020000CF03EF9009B04000D00002B6B
:1022200056DD721E92000EAB9B5818211F000098BD
:10223000091A0F410798C0198F40DF1B0EAB9F5042
:102240001723009A07909B1A1F410597059B002BA7
:102250004FDD079B00270133079380235B043A007F
:102260009C4691000EABCB58002F00D0A5E0002B70
:1022700004D06746FB1A0EAFCB51012701329642BC
:10228000EFD1009B002B05DD012B00D19AE0022B42
:1022900000D1A1E0059B022B2BD122002B000020B6
:1022A00059490CF0F7F804000D00002F21D0009AD6
:1022B00000205549FFF712FE02000B002000290004
:1022C0000CF0E8F804000D0013E0002000210EE7F8
:1022D000009B002B06D1731E9B000EAAD758FB153E
:1022E0000593B3E70022494B0AF0E4F9002861D1D5
:1022F000059700220023200029000AF0B7F90028E2
:1023000000D1E0E00022731E0293013B022B00D0BB
:102310006AE0002A00D19BE0009B0EAA183B0093C4
:10232000029B9B009B58002B00D1C8E0009A002024
:102330003549FFF7D3FD06000F00029C002C00DB9F
:10234000FCE00025029B324FDC0072AB1C19029BA3
:102350005B1B00D40AE100263500029C002C00DB48
:1023600029E1059B2900002B02D080231B06E918D8
:102370000B003200099901240A604B604A984B997E
:102380002B000CF087F8029BA34200DB20E1059BA9
:10239000002B02D080231B06C91802000B00072067
:1023A00009998A60CB60079B034018009B239B0020
:1023B0009D44F0BD022305934BE71648C31A0EA8AF
:1023C0000B505BE7721E92000EAB9B5802935B02B0
:1023D0005B0A0EA98B505DE7721E92000EAB9B58F4
:1023E00002939B029B0AF4E799000EA8091849681A
:1023F0000A438AE794FDFFFF98F500000000703E55
:1024000000007041000020400000F03F0000E03F6D
:10241000F0EC0000FFFFFF0001339A008A1A1269F6
:10242000002AF9D0721C0292069A00249219D20056
:102430000792079922AA8C4662440C92F318F20084
:102440000D920593029B059A934204DD160089E6DE
:1024500001230EA9E1E7079B0A9A1D1922AB5D191A
:10246000029B00269B00D0580CF092FB00272860AE
:10247000696000250C9B1B190B93089AEB00D1187F
:102480000B9A08684968D31A1A685B680BF090FDCC
:102490000B000200390030000AF064FE069B013593
:1024A00006000F00AB42E8D10D9B72AA1B19D3188E
:1024B0009E60DF60029B083401330293C2E7029BF7
:1024C000013B029328E7009B20005A422900FFF7B6
:1024D00005FD0022434B04000D000AF0EBF8002834
:1024E00023D00022404B200029000BF061FD0CF0AE
:1024F00019FB07000CF04CFB00223A4B0BF058FD87
:1025000002000B00200029000BF0C4FF0CF00AFBB6
:102510000EABB200D050731C0293009B0EAA18336E
:102520000093029B9B009F5000E7200029000CF0C5
:10253000F9FAB7000EABF8500296F7E6E50072AB79
:102540000EAA5D19A30098580CF022FB32003B0044
:102550000BF02EFD002228606960234B300039000B
:102560000BF026FD013C06000F00E7E600220023E9
:10257000002600920193B54213DBF300F918E3182B
:102580001A685B68086849680BF012FD02000B00CE
:10259000009801990AF0E6FD013600900191052EA0
:1025A000E9D1EB004AAAD31801350099019A083CF9
:1025B00019605A60CBE6E3004AAAD31830001A68C3
:1025C0005B6829000AF0CEFD013C06000D00C5E65F
:1025D000E3004AAAD3181A685B680AF0C3FD013405
:1025E000D1E6C046000070410000703E49004B0833
:1025F00019007047F7B54B005B080193019A3F4BF8
:102600009A4204DD02000B000BF0D2FC2BE03C4BA5
:10261000019A9A422DDCFFF7E9FFFEF721FA00222A
:10262000384B06000F000AF09DFD374B019A04005D
:102630000D009A4219DD32003B00300039000BF0EA
:10264000B7FC220006000F002B00200029000AF032
:1026500089FD02000B00300039000BF09FF80022CA
:10266000284B0AF07FFD04000D002000290003B074
:10267000F0BD264B019A9A4216DCFFF7B7FFFEF732
:1026800005FC0022224B04000D000BF091FC2200FF
:1026900006000F002B0000201D490BF07FF8020000
:1026A0000B0030003900DCE71A4B019A9A4206DC35
:1026B000FFF79CFFFEF7EAFB0022154BA4E7164B41
:1026C000019A9A4205DD154B9A4213D1144A904261
:1026D00010D8FFF78BFF00220D4B0BF069FCFEF7C3
:1026E000D5FB04000D000022094B0BF061FC220019
:1026F0002B0089E70020FEF79FF9B4E7FFFFEF7F8B
:10270000422ED63F0000F03FFFFF7F3CFFFF3540E9
:102710000000E03F412E8640CD338640CE338640D8
:102720007DF8B98FF0B54C4A4E0085B005000C001D
:102730000B007608964208DD02000AF013FD050042
:102740000C002800210005B0F0BD0022002944DA69
:10275000424B00920193424B9E424FDC414B9E42C2
:102760000BDC414A414B280021000AF0FBFC00220F
:102770003F4B09F095FF0028E3D128002100FFF727
:1027800035FFFEF76DF93B4B04000D009E4226DC41
:1027900002000B000AF0E6FC2200029003912B00DD
:1027A000200029000BF004FC002206000F00304B33
:1027B000200029000AF0D6FC02000B00300039008E
:1027C0000AF0ECFF02000B00029803990BF062FE86
:1027D000009A019B0BF0ECFBB1E7274BB9E7002215
:1027E000234B0AF0BFFC02000B00200029000AF076
:1027F000D5FF22002B000AF0B5FCE9E71F4B9E42F3
:1028000006DC28002100FFF7F1FEFEF73FFBDFE7C3
:102810001B4B9E4205DD1B4B9E4217D11A4A954227
:1028200014D828002100FFF7E1FE0022124B0BF024
:10283000BFFBFEF72BFB04000D0002000B0000980D
:1028400001990BF0B5FB22002B00C3E7064A074BAA
:1028500028002100BEE7C046FFFFEF7F0000E0BF79
:10286000FFFF3540FFFF2F3E3374AC3C1F7BAC7F36
:102870000000F03FFFFFEF3F0000E03F412E8640A9
:10288000CD338640CE3386407DF8B98FF7B517003B
:102890001E0004000D00FFF7A9FE00221B4B09F0EB
:1028A000F5FE00280CD020002900FFF7A3FE3860B9
:1028B000796020002900FFF735FF30607160F7BDB7
:1028C00020002900FEF7E2FA04000D0002000B00D0
:1028D00000200E490AF062FF0022009001910B4B8C
:1028E000200029000BF064FB009A019B04000D00FE
:1028F0000BF0D0FD220030607160009801992B0030
:102900000AF030FC38607960D9E7C0460000E03F4B
:1029100082B0F0B58BB00190109211930022129802
:102920001399002309F0A2FE0022002300283ED0C4
:102930001098119909F09AFE00280CD0129813995A
:10294000002200230BF034FB002200230AF00AFCD3
:10295000129C139D19E010981199FFF747FEFEF79E
:10296000C7FD0022002304000D001098119909F002
:1029700083FE00220023002812D0200029000BF043
:1029800017FB002200230AF0EDFB019B1860596041
:102990009C60DD6001980BB0F0BC08BC02B0184729
:1029A000129813990BF004FB22002B00CEE710982D
:1029B000119909F05BFE002830D012981399FFF7A7
:1029C00015FE0022764B0BF0F3FAFEF791FD002284
:1029D000002305000C000BF0EBFA002206000F00AC
:1029E00012981399002309F05BFE32003B00002887
:1029F00004D0280021000AF0B5FB06E028002100E1
:102A00000BF048FD80231B06E418019B2A00186088
:102A10005960230001998A60CB60BBE71098119937
:102A2000FFF7E4FD00225F4B09F03AFE00280AD1CF
:102A300012981399FFF7DAFD00225A4B09F030FE85
:102A4000002800D175E0109811990022564B0BF028
:102A5000AFFA0022544B04000D00129813990BF0AA
:102A6000A7FA8023002202900391DB0504920593CC
:102A700002980399002200230BF09AFA22002B00FF
:102A80000AF070FB029A039BFEF7E6FD0022444B1E
:102A90000BF08EFA002206900791414B200029008E
:102AA0000BF086FA002206000F00029803993C4BB7
:102AB0000BF07EFA002208900991002320002900E3
:102AC00009F0EEFD32003B00002846D00698079939
:102AD0000AF048FBFEF70CFD02000B0006000F0099
:102AE000089809990AF05AFEFFF780FD049A059BA1
:102AF0000BF05EFA32003B0005000C0004980599CB
:102B00000BF056FA06000F000022002328002100D7
:102B10000BF04EFA002204900591029803990023CD
:102B200009F0AAFD049A059B002835D03000390031
:102B300066E70022109811991C4B0BF039FA00221D
:102B40001A4B04000D00129813990BF031FAF92377
:102B50000290039100229B0588E7069807990BF0E5
:102B600099FCFEF7C5FC02000B0004000D0008985C
:102B700009990AF013FEFFF739FD049A059B0BF043
:102B800017FA22002B0006000F00049805990BF09D
:102B90000FFA05000C00B7E7300039002BE7C046FC
:102BA0000000E03F000010400000D03F0000504314
:102BB000F0B593B002920393039B0E0002995D005F
:102BC00004930B006D0807002B4319D180210903E2
:102BD000714002000B0092185B419B498B4206D862
:102BE00001D000F0C7FC002A01D100F0C3FC029A1A
:102BF000039B380031000AF0B5FA009001917CE0A7
:102C0000924B74000896009064089C469C4207DC36
:102C100001D1002804D1654502DC0CD100290AD07D
:102C20008B4BF3183B43E2D18021039809034840C2
:102C3000029A0300CFE700230693002E17DA854A95
:102C400095424BDC844A954211DD844B2A15D218FB
:102C5000142A23DD3420821A0298D04003009340C6
:102C60008B4204D1012210409218131A06930029B6
:102C70005ED1654521D1764BE3181F4301D100F0A9
:102C800079FC754B9C422BDD049B002B01DA00F094
:102C900075FC029B039C009301942EE0002947D110
:102CA00014239A1A2B00134119009140A94204D110
:102CB000012213409218D31A0693694B9D4220D1EA
:102CC00038003100049B00900191002B15DA3A0086
:102CD0003300002062490AF061FD8EE70223C5E758
:102CE000049B002B01DB00F049FC80221206944675
:102CF000029B0093039B634401930098019913B0D6
:102D0000F0BD8023049ADB059A4206D13A003300D5
:102D1000380031000BF04CF96FE7524B049A9A429D
:102D200006D1002E04DB38003100FEF7E1FB64E73A
:102D300038003100FFF75AFC00900191002F2ED18E
:102D4000002C04D0464AB3009B08934227D1049B31
:102D5000002B07DA009A019B002041490AF01EFD72
:102D600000900191089B002BC7DA394BE418069BB1
:102D70001C4308D1009A019B100019000BF08AFB3C
:102D800002000B00A7E7069B012BB6D1009880211B
:102D9000020001980906431800920193ADE7F20F73
:102DA000069B013A134304D13A0033003800310046
:102DB000E4E7069B013B13430022002B14D0284B71
:102DC000069207938423DB059D4200DC0AE1264B33
:102DD0009D4212DD204B9C4208DC049B002B08DA4C
:102DE0000020FDF729FE08E7204BE9E7049B002BB4
:102DF000F6DC0020FDF70CFEFFE61D4B9C420FDCCD
:102E0000069807990023002209F036FC431E9841DA
:102E100001244042049B04402000002BEADAE0E752
:102E20000F4B9C4226DD069807990023002209F0EB
:102E300023FC431E984101244042049B044020008F
:102E4000002BCEDCD6E7C0460000F0FF0000F07F8C
:102E5000000010C0FFFF3F43FFFFEF3F01FCFFFFFB
:102E60000000F03F0000E03F0000F0430000F0BF32
:102E7000FEFFEF3F0098019900224F4B0BF00AFB39
:102E8000C0224E4BD20506000F000BF091F84C4AC1
:102E9000049005914B4B300039000BF089F800226B
:102EA00000900191484B300039000BF081F802008E
:102EB0000B00464846490BF0EDFA32003B000BF0A0
:102EC00077F802000B00002042490BF0E3FA3200D1
:102ED00004000D003B00300039000BF069F80200DF
:102EE0000B00200029000BF063F83B4A334B0BF03A
:102EF0005FF802000B00009801990BF0CBFA02007A
:102F00000B0004000D00049805990AF02BF9049AAF
:102F1000059B0020009001910BF0BCFA02000B0011
:102F2000200029000BF0B6FA029C039D0024060045
:102F30000F000298039922002B000BF0ABFA009AC5
:102F4000019B0BF035F8029A039B04900591300029
:102F500039000BF02DF802000B00049805990AF0D7
:102F600001F922002B0002900391009801990BF0C7
:102F70001FF806000F000B00020002980399049648
:102F800005970AF0EFF8154B05000C0008919942DF
:102F900000DCCAE2124BCB18034300D1CCE1069807
:102FA00007990023002209F067FB431E9841012482
:102FB00040420440200014E70000F03F4715F73F6F
:102FC00044DF5DF80BAE543E0000D03F55555555DB
:102FD0005555D53F0000E03FFE822B65FFFF8F4037
:102FE000000070BFBB4B00229C420ADC0098019994
:102FF0000022B94B0AF0DCFF352200900191019CC0
:103000005242B64923155B189B182403B44DB54AA8
:103010000E93230B1D430024934209DDB24A013471
:10302000934205DD0E9B1B1900240E93AF4BED1848
:10303000009801992900AE4AE300D3180F931A6C47
:103040005B6C0C900D910A920B930BF023FA0C9A87
:103050000D9B06000F000A980B990AF083F80200F6
:103060000B0000209E490AF099FB1090119102007C
:103070000B00300039000AF09BFF08900991089A74
:10308000099B802104920593002389056D100D434F
:1030900080210493049A059B009201930022090366
:1030A0006D18A4042B190098019914001D000AF052
:1030B0007FFF02000B00300039000BF0EBF90A9A99
:1030C0000B9B06000F00200029000BF0E3F9020023
:1030D0000B000C980D990BF0DDF9009A019B0AF09A
:1030E00067FF02000B00300039000BF0D3F9109A93
:1030F000119B0AF05DFF089A099B0A900B91100042
:1031000019000AF055FF06000F007A4A7A4B0AF0C0
:103110004FFF7A4A7A4B0AF025F832003B000AF05A
:1031200047FF784A784B0AF01DF832003B000AF05E
:103130003FFF764A764B0AF015F832003B000AF062
:1031400037FF744A744B0AF00DF832003B000AF066
:103150002FFF724A724B0AF005F8320004000D008E
:103160003B00300039000AF023FF02000B00200072
:1031700029000AF01DFF009A019B04000D00089829
:10318000099909F0EFFF0A9A0B9B0AF011FF220040
:103190002B0009F0E7FF009A019B0C900D911000A5
:1031A00019000AF005FF00225E4B04000D0009F033
:1031B000D9FF0C9A0D9B09F0D5FF049E0F00320039
:1031C0000B00009801990AF0F3FE00220090019193
:1031D000544B300039000BF05DF922002B000BF04E
:1031E00059F902000B000C980D990BF053F9089A4D
:1031F000099B0AF0DDFE320004000D000A980B99CD
:103200003B000AF0D5FE02000B002000290009F067
:10321000A9FF04000D0002000B000098019909F0BD
:10322000A1FFE022049E12063F4B30000F000AF07F
:10323000BFFE08900991009A019B300039000BF005
:1032400029F902000B00200029000BF023F9374A6E
:10325000354B0AF0ADFE364A04000D00354B300008
:1032600039000AF0A5FE02000B002000290009F039
:1032700079FF0F9B1A6D5B6D09F074FF0A900B913B
:103280000E980BF085FC04000D00089809990F9B1F
:103290001E6E5F6E0A9A0B9B09F064FF32003B00C2
:1032A00009F060FF22002B0009F05CFF0498220067
:1032B0002B00009001910BF0EDF832003B000BF079
:1032C000E9F8089A099B0BF0E5F802000B000A9850
:1032D0000B9927E6FFFF0F000000404301FCFFFFB2
:1032E0000000F03F8E98030079B60B000000F0FF5D
:1032F000F0EC0000EF4E454A287ECA3F65DBC993DB
:103300004A86CD3F01411DA96074D13F4D268F51A2
:103310005555D53FFFAB6FDBB66DDB3F0333333322
:103320003333E33F0000084009C7EE3FFD033ADCBA
:10333000F5015B14E02F3EBE924A934B029803992D
:1033400009F010FF3200009001913B00280021009D
:103350000BF0A0F802000B000098019909F0A0F909
:10336000002800D01BE60021884A63005B0800911A
:10337000934225DD864A1B159B18802252039446F2
:103380001A4114196000834B400D834DC01805414C
:103390002100A9430B0061462403240B214314247C
:1033A000201A0141009108990022002902DA0099AF
:1033B00049420091300039000BF06CF804900591FF
:1033C000029A039B04980599002609F0CBFE00227F
:1033D000724B30000F000AF0EBFD049A059B089039
:1033E0000991300039000BF055F802000B000298EB
:1033F00003990BF04FF86A4A6A4B0AF0D9FD6A4A02
:1034000004000D00694B300039000AF0D1FD0200C4
:103410000B002000290009F0A5FE04000D000200A9
:103420000B000898099909F09DFE089A099B06006F
:103430000F000BF02FF802000B00200029000BF00A
:1034400029F83200029003913B00300039000AF065
:10345000AFFD04000D00564A564B0AF0A9FD564A2E
:10346000564B0BF017F822002B000AF0A1FD544A2E
:10347000544B09F077FE22002B000AF099FD524AC6
:10348000524B0BF007F822002B000AF091FD504A36
:10349000504B09F067FE22002B000AF089FD020064
:1034A0000B00300039000AF0F5FF04000D000200A7
:1034B0000B00300039000AF07BFD80230490059159
:1034C0000022DB05200029000AF0E4FF02000B00C7
:1034D000049805990AF062F9029A039B04000D0012
:1034E000300039000AF064FD029A039B09F03AFEAD
:1034F00002000B00200029000AF0CCFF32003B0044
:103500000AF0C8FF02000B00002033490AF0C2FF96
:10351000009B1B055B181A15002A29DC009AFEF790
:10352000DDFC069A079BFFF7F5FB2C4A4B005B0876
:10353000934200DC17E72A4BCB1803430CD00698C4
:1035400007990023002209F097F8431E98410124AF
:103550004042044020004DE432003B000AF09AFF54
:10356000029A039B09F0A6F8002800D1FBE6E6E7E3
:103570001900D6E70023184CFFF78DFB0023002429
:10358000FFF789FBFE822B654715973C0000E03F63
:1035900002FCFFFF01FCFFFFFFFF0F00432EE63F91
:1035A000EF39FAFE422EE63F396CA80C615C20BE72
:1035B000D0A4BE726937663EF16BD2C541BDBB3E39
:1035C0002CDE25AF6A56113F93BDBE166CC1663F17
:1035D0003E5555555555C53F0000F03FFFCB904037
:1035E00000346F3FF0B5984B85B04E0004000D00DD
:1035F000039176089E4218DD944B9E4202DC0AD16C
:10360000002808D022002B002000290009F0AAFD84
:1036100004000D0005E0039B8D4C002B00DC10E145
:103620008C4D2000290005B0F0BD8B4B9E420FDC75
:103630008A4B9E4209DC8A4A8A4B09F093FD00229C
:10364000894B09F02DF80028EBD101235B4225E0DE
:10365000FEF7CCFF854B04000D009E4200DDAAE082
:10366000834B9E4200DD90E002000B0009F07AFDE2
:1036700000227D4B0AF00EFF802306000F0000227F
:10368000DB052000290009F06DFD0B000200390068
:1036900030000AF083F8002304000D00029322009A
:1036A0002B00200029000AF083FC02000B00009090
:1036B00001910AF07DFC06000F006E4A6E4B0AF085
:1036C00077FC6E4A6E4B09F04DFD32003B000AF06C
:1036D0006FFC6C4A6C4B09F045FD32003B000AF070
:1036E00067FC6A4A6A4B09F03DFD32003B000AF074
:1036F0005FFC684A684B09F035FD32003B000AF078
:1037000057FC664A664B09F02DFD009A019B0AF0B2
:103710004FFC644A00900191634B300039000AF07D
:1037200047FC624A624B0AF0B5FE32003B000AF0E9
:103730003FFC604A604B0AF0ADFE32003B000AF0ED
:1037400037FC5E4A5E4B0AF0A5FE32003B000AF0F1
:103750002FFC5C4A5C4B0AF09DFE32003B000AF0F5
:1037600027FC02000B000098019909F0FBFC2B00DC
:1037700022000AF01DFC029B013343D102000B0022
:10378000200029000AF086FE42E70022364B0AF0AC
:1037900081FE002206000F00334B2000290009F0B3
:1037A000E1FC0B0002003900300009F0F7FF0123B3
:1037B00004000D0072E7454B9E4219DC0022444B89
:1037C0000AF068FE002206000F00414B200029008D
:1037D0000AF0EEFB0022244B09F0C4FC0B000200AF
:1037E0003900300009F0DAFF022304000D0055E72C
:1037F0000B0002003749002009F0D0FF032304002A
:103800000D004BE7029B344FDE00344BBF199E196D
:10381000326973690AF03EFE22002B000AF03AFE7C
:103820000B000200386F796F0AF034FE039B04002E
:103830000D00002B00DBF4E6802109066B181D004B
:10384000EFE6274DEDE6C046FFFF0F440000F07F96
:10385000182D4454FB21F93FFFFFDB3FFFFF1F3EC4
:103860009C7500883CE4377E0000F03FFFFFF23F8C
:10387000FFFFE53F11DA22E33AAD903FEB0D7624EE
:103880004B7BA93F513DD0A0660DB13F6E204CC58A
:10389000CD45B73FFF8300922449C23F0D55555592
:1038A0005555D53F2F6C6A2C44B4A2BF9AFDDE5209
:1038B0002DDEAD3F6D9A74AFF2B0B33F711623FEAB
:1038C000C671BC3FC4EB98999999C93FFF7F0340EB
:1038D0000000F83F0000F0BFF0EC000070ED0000C9
:1038E000FB21F9BFF7B554425E001443484F7608F8
:1038F000E40F00933443BC4209D844424D000443D2
:103900006D08E40F009101902C43BC4203D909F0EB
:1039100029FC03B0F0BD3F4C1C19144302D1FFF742
:1039200061FEF6E79C17A446022467463C40009FD0
:10393000FF0F3C43019F2F4306D1022C62D0032C82
:10394000E7D135483549E4E73700174305D1009BF7
:103950003148002B59DA3249DBE72D4FBE421BD1EB
:10396000B5420ED1022C06D0032C07D02A48012CD8
:1039700046D12C49CDE72C482C49CAE72A482C4986
:10398000C7E7022C3ED0032CDBD000200021012C05
:10399000BFD180210906BCE71D4FBD42D7D0AD1B6A
:1039A0002D153C2D16DC002B01DA3C3515DB09F01A
:1039B000F5FEFEF71BFEFFF715FE012C10D0022CC2
:1039C00013D0002CA5D01B4A1B4B0AF063FD124AF2
:1039D0001A4B12E010481A49EFE700200021ECE7EB
:1039E000802424060B19190093E7124A124B0AF09F
:1039F00051FD02000B00084810490AF04BFD88E712
:103A0000104986E704480D4983E70D4981E7C04620
:103A10000000F07F000010C0182D4454FB2109C0A5
:103A2000FB21F9BFFB21E9BFD221337F7CD90240C2
:103A30007CD902C0075C143326A6A13CFB210940B7
:103A4000FB21F93FFB21E93F82B0F0B589B00E922E
:103A50000F93019000220E980F99002308F006FEA4
:103A6000002808D0109811990022704B08F018FE19
:103A7000002800D0CCE00E9A0F9B100019000AF02D
:103A800097FA0290039102000B00002067490AF0A8
:103A900001FD109A119B04000D00100019000AF09E
:103AA00087FA02000B00200029000AF0F3FC0E9AAE
:103AB0000F9B04000D001000190009F053FB2200B9
:103AC0002B00FFF70FFF0022594B0AF071FA594AF9
:103AD000594B0490059109F061FE00220023040077
:103AE0000D0008F0E7FD0022514B002800D18AE0CC
:103AF0002000290009F036FB00224C4B04000D0089
:103B0000109811990AF0C6FC02000B000AF050FA56
:103B1000029A039B09F026FB0022002306900791DE
:103B200008F0A4FD002800D072E0290020000AF06F
:103B3000F9FF0BF02DF8002206000F0010981199E4
:103B40003A4B09F00FFB02000B000AF031FA029A1F
:103B5000039B09F007FB069A079B09F01FFEFDF780
:103B6000F7FA0022354B0AF023FA354A0290039106
:103B7000344B300039000AF01BFAA8220690079156
:103B8000D2052D4B300039000AF012FA02000B006A
:103B9000049805990AF07EFC802204000D0052056D
:103BA000294B300039000AF003FA02000B00200014
:103BB00029000AF06FFC002206000F00029803990A
:103BC00000230AF0F5F9069A079B04000D00300067
:103BD00039000AF05FFC02000B002000290009F008
:103BE000C1FA019B002218605960029803990023D2
:103BF00009F0B8FA019B9860D960019809B0F0BC4F
:103C000008BC02B01847200029000AF043FC73E703
:103C10000E4B0198196B5A6BDC6B9B6B0160426019
:103C2000029303948360C460E7E7C0460000F03F5E
:103C30000000E03F182D4454FB2109400000D03F14
:103C40006EC0453163626A3C460B213E70ED000058
:103C500082B0D3B5069207930400089A099B069890
:103C60000799FDF7F9FCFDF773FA069A079B009098
:103C7000019108980999FFF735FE002200230600FC
:103C80000F000AF095F9009A019B09F06BFAA66003
:103C9000E760206061602000D6BC08BC02B0184715
:103CA00082B0F0B593B004001A981B99189219933A
:103CB000002200230AF07CF9189A199B09F052FAA5
:103CC00000260200002700200B00454902960397BA
:103CD000049005911A981B99009001910EA808F084
:103CE000F3FC0E9A0F9B08920993109A119B0A926B
:103CF0000B93189A199B1000190009F033FA1A9ABD
:103D00001B9B0AF055F90D00079032003B00079805
:103D100029000AF04DF91A9A1B9B06000F0018980B
:103D200019990AF0B7FB1A9A1B9B0C900D911898E1
:103D3000199909F017FA02000B000C980D990AF076
:103D400037F932003B0009F00DFA02000B000020A9
:103D500023490AF09FFB32003B000AF09BFB8023C3
:103D60001B06ED180B0007990200019500910EA8A3
:103D7000FEF7CEFD0E9A0F9B0898099909F0F2F90B
:103D8000109A119B06000D000A980B9909F0EAF9A8
:103D900032002B00019100900EA8FFF759FF00227E
:103DA000104B0EA804920593802300221B0602925A
:103DB0000393109A119B009201930E9A0F9B08F0A7
:103DC00083FC0E9A0F9B200022606360109A119B67
:103DD000A260E36013B0F0BC08BC02B01847C04654
:103DE0000000F03F0000F0BF82B0F0B589B00F9343
:103DF000159B0E9207930600109A119B0E980F992F
:103E0000FDF72AFC00220023149F0290039108F082
:103E10002DFC002810D0474B196C5A6CDC6C9B6C45
:103E200031607260009301943000B360F46009B0B7
:103E3000F0BC08BC02B01847079B10981199069374
:103E40000E9A0F9BFFF74EFD129A139B049005915B
:103E500002980399FEF7ACFE374A0090019104984E
:103E60000599364B09F09AFC02000B001298139941
:103E70000AF09EF8002204000D0000233800069985
:103E800008F0F4FB00282AD1049A059B8020000644
:103E900084460799049761440591049805990AF0AE
:103EA00087F8FCF7F3FF02000B00009801990AF075
:103EB0007FF80090019102980399FDF749F93A00C3
:103EC000069B0AF075F81C4A1C4B09F067FC0200BF
:103ED0000B002000290009F045F904000D00200026
:103EE0002900FDF72FFE009A019B0AF061F82200DD
:103EF0002B0002900391002011490AF0CBFAFDF744
:103F000021FE02000B00009801990AF051F80022EE
:103F100004000D000298039900230AF049F80B00F1
:103F200002002900200009F01DF9029B039C30606B
:103F3000716079E770ED0000182D4454FB210940B1
:103F40000000E03FF0B58FB000934B005B08069394
:103F50000292D34B069A05000C000B919A425DDC4D
:103F60000AF0E0FD0490002800D07CE0149B069A43
:103F700001332B4313430FD128002100FEF736FBFA
:103F800002000B000020C74909F008FC05000C00E6
:103F9000280021000FB0F0BD149B012BF8D0029A2D
:103FA000009B2800210009F0DDF8020004980B00B6
:103FB000069007910020BC4909F0F0FB2A00089008
:103FC000099106980799089E099F23000AF062FA52
:103FD000049E02000B00029800990AF05BFA32007E
:103FE0003B0009F0E5FF320004000D000698079938
:103FF0003B0009F0DDFF0022AA4B09F0B3F80200F4
:104000000B002000290009F0ADF8089A099B09F07F
:10401000CFFF32003B0009F0A5F8B7E7A34B069AA3
:104020009A4220DD002907DA802109068C466318B0
:104030001C00009B634400932A0023009C489D4978
:104040000AF028FA06000F00029A009B9A489B4942
:104050000AF020FA3B00320009F084F80023050042
:104060000C00029300932A0023002800210009F08D
:104070009FFF02000B000490059109F099FF049A3C
:10408000059B06000F002800210009F091FF8C4AD3
:10409000089009918B4B3000390009F089FF8A4A5A
:1040A0008A4B09F05FF832003B0009F081FF884A33
:1040B000884B09F057F832003B0009F079FF864A37
:1040C000864B09F04FF832003B0009F071FF844A3B
:1040D000844B09F047F832003B0009F069FF824A3F
:1040E000824B09F03FF8049A059B09F061FF804A72
:1040F0000C900D917F4B3000390009F059FF7E4A3A
:104100007E4B09F02FF832003B0009F051FF7C4A4A
:104110007C4B09F027F832003B0009F049FF7A4A4E
:104120007A4B09F01FF832003B0009F041FF784A52
:10413000784B09F017F832003B0009F039FF764A56
:10414000764B09F00FF802000B000C980D9909F05E
:1041500009F8089A099B09F02BFF029A009B09F0C5
:1041600001F8049A059B09F023FF029A009B08F0CE
:10417000F9FF06000F0008980999694A694B09F090
:1041800017FF32003B0008F0EDFF029003910200A0
:104190000B002800210008F0E5FF444B069A0600BA
:1041A0000F009A423DDD14980AF0F2FC32000090B4
:1041B00001913B003000390009F0FAFE009A019BA2
:1041C000049005913000390008F0CCFF02000B008C
:1041D0000498059909F0E2FA029A039B0AF05AF949
:1041E00002000B00280021000AF054F902000B0025
:1041F00008F0B8FF02000B00009801990AF04AF994
:104200000B9B0400981702231840013B181A0D005D
:104210000AF0BEFC02000B002000290009F0C8FED5
:10422000B4E6149B012B37D000230096019700932E
:10423000009A019B0492059302000B0000201A498A
:1042400009F0ACFA2A000690079104980599069E99
:10425000079F23000AF01EF9009E02000B0002983F
:1042600003990AF017F932003B0009F0A1FE320071
:1042700004000D00049805993B0009F099FE002206
:10428000084B08F06FFF02000B002000290008F027
:1042900069FF069A079BBAE605000C0078E6C0465F
:1042A000FFFF2F3E0000F03F0000F0BF2794E53FE6
:1042B000182D4454FB21E93F075C143326A6813CAA
:1042C000D47ABF74702AFB3EE9A7F0320FB8123FD0
:1042D00068108D1AF726303F1583E0FEC8DB573F84
:1042E00093846EE9E326823FFE41B31BBAA1AB3F44
:1042F000735360DBCB75F3BEA69237A0887E143F64
:104300000165F2F2D844433F280356C9226D6D3F40
:1043100037D60684F464963F7AFE10111111C13F1E
:10432000635555555555D53FF0B54B008FB05B08DB
:1043300000931700DA4B009A040007919A4209DCB7
:1043400002000B003A607B6000220023BA60FB6031
:10435000002624E0D34B009A9A4200DD6DE0D24A59
:10436000002935DDD14B0AF095F8009B04001A00B6
:10437000CE4B0D009A4215D0CD4ACE4B0AF08AF8AA
:1043800002000B0020003A607B6029000AF082F8EE
:10439000C74AC84B0AF07EF80126B860F9603000C1
:1043A0000FB0F0BDD322C34B52050AF073F8C24AD6
:1043B000C24B04000D000AF06DF802000B00200053
:1043C0003A607B6029000AF065F8BB4ABB4BE1E725
:1043D000B64B08F0C7FE009B04001A00B34B0D005B
:1043E0009A4214D0B24AB34B08F0BCFE02000B0054
:1043F00020003A607B6029000AF04CF8AC4AAD4BD3
:1044000008F0B0FE0126B860F9607642C7E7D32213
:10441000A84B520508F0A6FEA74AA84B04000D00C1
:1044200008F0A0FE02000B0020003A607B6029002B
:104430000AF030F8A04AA14BE2E7A14B009A9A4259
:1044400000DDD0E0FEF7D2F89E4A9F4B04000D003D
:1044500009F0AEFD00229D4B08F084FE0AF062FBDD
:1044600006000AF095FB904A904B0490059109F0E4
:104470009FFD02000B00200029000AF00BF88C4A77
:1044800002900391049805998A4B09F091FD04006C
:104490000D0002000B000298039909F0FBFF1F2E8C
:1044A00028DC8B4A731E9B009B58009A934221D0B4
:1044B00002000B003A607B60029803997B683A68BF
:1044C0000093009B09F0E6FF22002B0009F0E2FFB9
:1044D0000B000200BA60FB60079B002B00DB5EE76D
:1044E000802212069446009B891863447B60B86062
:1044F000F9608AE7009B1B150693069A4B005B0D3B
:10450000D31A102BD4DD04980599D322694B520598
:1045100009F04EFD04000D0002000B000298039903
:1045200009F0B8FF02000B00009001910298039976
:1045300009F0B0FF22002B0009F0ACFF04000D00D1
:10454000049805995C4A5D4B09F032FD22002B006E
:1045500009F0A0FF02000B0004000D000098019973
:1045600009F098FF069A4B005B0DD31A312B08DC3B
:1045700002000B003A607B60009A019B0292039359
:104580009AE7B8220498059992054C4B09F010FD62
:1045900004000D0002000B000098019909F07AFF59
:1045A00002000B00029003910098019909F072FF3C
:1045B00022002B0009F06EFF04000D0004980599FD
:1045C000444A454B09F0F4FC22002B0009F062FF3D
:1045D00002000B0004000D000298039909F05AFF35
:1045E0003860796068E73D4B009A9A4208DD020026
:1045F0000B0009F04FFFB860F96038607960A7E6FA
:10460000009B374A1B159B18009A02931B05D51A6D
:1046100029000AF087FA0AF0BBFA02000B0020001A
:1046200029000892099309F035FF00222D4B09F06B
:10463000BFFC04000D000AF075FA0AF0A9FA0200A6
:104640000B0008AEB260F3602000290009F022FFE1
:104650000022244B09F0ACFC032430617161651E1B
:10466000EB00F318186859680022002307F0FEFFDA
:10467000002813D123003000029A3900FDF716FDFF
:10468000079B0600002B00DB89E680227B68120670
:104690009B187B60FB689B18FB60B6E62C00DEE78E
:1046A000FB21E93F7BD9024000004054FB21F93F48
:1046B0003163621A61B4D03D7370032E8A19A33B33
:1046C000FB21394183C8C96D305FE43F0000E03F02
:1046D00018F50000C14920259A837B39FFFFEF7F41
:1046E000EAFBFFFF0000704130B5204A4B0087B065
:1046F0005B08934206DC0023002200930023FDF7B1
:10470000E1F806E01A4A934205DD02000B0009F0C9
:10471000C1FE07B030BD02AAFFF706FE049C059D4E
:1047200003230340012B0AD002980399022B0DD0DA
:10473000002B15D10133009322002B00DFE722006C
:10474000029803992B00FDF709FBE2E70123220001
:1047500000932B00FDF7B6F880231B06C918D8E795
:1047600022002B00FDF7FAFAF6E7C046FB21E93FED
:10477000FFFFEF7F30B51E4A4B0087B05B089342C6
:1047800004DC00220023FDF7E9FA06E0194A93420F
:1047900005DD02000B0009F07DFE07B030BD02AA66
:1047A000FFF7C2FD049C059D03230340012B08D0A5
:1047B00002980399022B0FD0002B12D122002B005C
:1047C000E1E700932200029803992B00FDF77AF8A5
:1047D00080231B06C918E0E722002B00FDF7BEFA74
:1047E000F6E70123220000932B00FDF76BF8D4E7D6
:1047F000FB21E93FFFFFEF7F82B0D0B586B0040018
:104800000C980D990A920B9304AA02ABFEF73EF89E
:104810000A980B99FFF7AEFF029A039B09F0C8FBB9
:1048200006000F000A980B99FFF75EFF049A059B9C
:1048300009F0BEFB002200900191002330003900F6
:1048400009F0B6FB02000B000098019908F08AFC01
:10485000206061602000A660E76006B0D0BC08BCA4
:1048600002B0184782B0D3B50692079304000698A9
:104870000799FCF70BFB06000F0008980999FFF752
:1048800033FF32003B0009F093FB00900191089840
:104890000999FFF76FFF32003B0009F089FB002206
:1048A00006000F0000980199002309F081FB020027
:1048B0000B003000390008F055FC009A019B206085
:1048C0006160A260E3602000D6BC08BC02B018475B
:1048D00082B0F0B50026002797B01D931E9B1F9D48
:1048E0000E9304001C923B0032000E98290006959E
:1048F00007F0BCFE002821D01C981D9932003B0017
:1049000007F0C4FE002819D01C981D99FDF74CFB38
:104910001C9A1D9B07F0AAFE00280FD032003B0016
:1049200000208B4908F03AFFA660E76020606160D4
:10493000200017B0F0BC08BC02B0184780231C98B8
:104940001D991B06EB180F930022824B07F094FE73
:10495000002854D01C981D997F4A804B09F028FBF1
:104960007D4A06000D007D4B0E98069909F020FB4C
:1049700032002B000191009012A8FFF73DFF149A1E
:10498000159B129E139F069207931C9A1D9B002055
:104990006F4909F07FFD0B000F99020001910E99FC
:1049A00012A80091FFF794FF149A159B12A8049285
:1049B0000593129A139B02920393069A079B009207
:1049C000019332003B0007F07FFE149A159B04927E
:1049D0000593129A139B029203930022002312A8BC
:1049E000009201935C4A5D4B08F0E2F8129A139B27
:1049F00022606360149A159BA260E36098E700222E
:104A00001C981D99524B09F045FD002200230C9281
:104A10000D93012201254E4B089009910A920B93A8
:104A20004F4B50331093109AEB00D3181E685F68F9
:104A30000E9A069B2800049205930AF0A9F8089A9A
:104A4000099B08F08FFB0022002302900391009243
:104A5000019312A832003B0008F0AAF8129A139BA7
:104A60000A980B9908F07EFB149A159B0A900B91FB
:104A70000C980D9908F076FB01350C900D910B2DDB
:104A8000D1D1089809990022364B08F06BFB00221F
:104A9000304B08F067FB0500109111912E48324908
:104AA000FCF726FD002206000F0008980999294B03
:104AB00008F058FB0E9A069B02900391049205930E
:104AC000069B2A0001930E9B12A80093119BFFF7EF
:104AD0008BF91298139932003B0009F069FA320001
:104AE00006900791149815993B0009F061FA80220D
:104AF000120694460F0006000F9A109B01920E9A20
:104B00006344009212A82A00FFF7ACFE149A159B8A
:104B100012A804920593129A139B00960197029291
:104B20000393069A079B07F0CFFD0C9A0D9B12A8E2
:104B3000049205930A9A0B9B02920393149A159B75
:104B400000920193129A139B07F0BEFD4EE7C046F8
:104B50000000F03F0000E03F182D4454FB210940C5
:104B600070ED000000002240FB211940F7B506005F
:104B70000F0014001D00FCF7ADFC002805D120003B
:104B80002900FCF7A7FC00280BD0200029003200E8
:104B90003B0008F0E7FA04000D002000290003B0F4
:104BA000F0BD22002B003000390007F05FFD002827
:104BB000F3D1002200233000390007F057FD002810
:104BC0000CD0200029000022002307F055FD01240D
:104BD00000250028E1D080252D06DEE701236A4666
:104BE0003000137039000022002307F059FD00281F
:104BF00001D16B4618706A460123127830005A4082
:104C000001926A463900137022002B0007F034FD30
:104C1000002801D16B4618706B466A461B781279E2
:104C2000934204D001240025A4197D41B5E7012455
:104C30006442E517F8E7F7B5071E21DA124C134D69
:104C400047420022124B01260092019312E03742A4
:104C500007D00098019922002B0009F0A9F90090D3
:104C6000019122002B002000290009F0A1F9040085
:104C70000D007F10002FEAD10098019903B0F0BD1C
:104C80000024044DDDE7C0469A9999999999B93F56
:104C90000000F03F00002440F8B50D0017001E0092
:104CA000040009F03FFF386009F072FF02000B00BA
:104CB0002000290009F0EEFB0022104B09F078F9E2
:104CC00004000D00FBF75AFE09F02CFF306009F0DC
:104CD0005FFF02000B002000290009F0DBFB00222F
:104CE000074B09F065F9FBF749FE09F01BFF0028A7
:104CF00000D10130069B1860F8BDC04600408F40CF
:104D00000000594030B50A4B652804DD0322873383
:104D10001A70002030BD000118180930FF300268F9
:104D200043688468C5680A604B608C60CD60F0E7BA
:104D3000A808001070B505000C0000220023280010
:104D4000210007F099FC002807D0280080252D06B7
:104D50006119FDF729F9491970BD28002100FDF7F7
:104D600023F9F9E7F7B514001D0000900191002226
:104D7000184B2000290007F07FFC002801D00024F8
:104D8000144D0026134F009A019B2000290007F0C4
:104D90007DFC002803D13000390003B0F0BD3000A5
:104DA000390022002B0009F003F906000F00FCF780
:104DB00081FB0028EFD130003900FCF78BFB002885
:104DC000E9D1200029000022024B08F0CBF90400B1
:104DD0000D00D8E70000F03FF7B506000D003000E9
:104DE0002900FCF777FB071E51D130002900FCF7A2
:104DF00061FB041E4DD1002200233000290007F082
:104E000035FC002837D1002200233000290007F0AC
:104E100033FC002803D080231B06ED18DFE70022B7
:104E20001D4B3000290007F045FC002815D000225A
:104E30001A4B009201930098019932002B0007F061
:104E40002FFC002817D1009801990022134B09F07C
:104E5000AFF8013400900191EDE7114C114B009334
:104E6000019401240098019932002B0007F00EFCF8
:104E7000002802D064422000FEBD00980199002263
:104E8000064B08F08BFC013400900191EAE7002406
:104E9000F1E73C00EFE7C0460000F03F000024408F
:104EA0009999B93F9A9999990A4B10B51A007E328F
:104EB0001278002A0BD17F331B780022002B07D0F9
:104EC000054B09F075F8054A054B08F067FC10BD65
:104ED000044BF6E7A808001000007940182D445450
:104EE000FB2119400080764010B50122802806D8A9
:104EF000044980004358002B01D09847002210003D
:104F000010BDC04614F30000020008210300012078
:104F1000473A8A43D2B210B5824220D91A000424FB
:104F20006F3AA243D2B2002A19D01A00763A0A2A5E
:104F300015D9402218009043020001202B2A0ED0E0
:104F40009A1F82420BD9073AA243D2B20400002A28
:104F500005D000208B43433BDBB29C42404110BD57
:104F6000F8B501240C4D0D4E2F5D002F06D12B19E5
:104F7000013B1878FFF7C8FF00280AD03800FFF778
:104F8000C3FF431E98410019441CB442ECDDFA24CF
:104F9000E4002000F8BDC046D4000010CF07000098
:104FA00070B504000D00FFF7DBFF154B1A1AAA427B
:104FB00004DA0322134B87331A7070BD9C42FCDC69
:104FC0002919FAD4002DF8D00ADD00210E4BED1876
:104FD000A042F2DBC21816782E5411700138F7E7A0
:104FE000FA2200230848D200121B091824189A42FA
:104FF000E3DDE05CC8540020E0540133F7E7C0462D
:10500000CF070000A8080010D400001070B57C265F
:105010000C4D0D4BAC5B185DFFF776FF002807D0F9
:105020000A4B9C420AD9872303220120EA5470BD0F
:10503000074B9C42F7D80134AC53F8E70234AC5329
:105040000020F4E7A8080010D4000010CD070000ED
:10505000CE070000F7B5114C019123007C331B886B
:105060000F4D0700EA5C002A01D1002B01D1FFF7A8
:10507000CDFF7C3420880121FFF792FF268838007D
:10508000AF55FFF741FF002807D0701C0121FFF743
:1050900087FF2388ED18019B6B70F7BDA8080010EF
:1050A000D4000010F8B506000400064F351B002C94
:1050B00005DD013C385DFFF727FF0028F6D1012010
:1050C0002840F8BDD400001070B50A4E04B223B2D7
:1050D000002B01DC084809E0A5192B782B2B06D101
:1050E0002000FFF7DFFF002801D1687870BD013C88
:1050F000EDE7C046D4000010FFFFFF7FF8B57C2528
:10510000084E745B671E3800FFF7CCFF002805D1FE
:10511000002C01D07753F8BD0120FCE7023C74530A
:105120000020F8E7A808001030B5FA240023084949
:10513000E400CD5C5A1C2B2D04D18D5C854201D13D
:10514000981C30BD1300A242F3D10020F9E7C046FD
:10515000D400001010B5682802D8FFF7E5FF10BD95
:105160000A4BFE280CD1E922D2009B181868596816
:1051700009F0D8FC03004042002BF0DBD8B2ECE78A
:10518000032287331A700020E9E7C046A808001000
:1051900083280DD80F290BD88423CA085343181825
:1051A0000723194079330B41024A115C0B43135416
:1051B0007047C046B8100010F0B587B003923C4A63
:1051C0000493D3780C00834204D21378019301989E
:1051D00007B0F0BD002153689278801A1A7888428F
:1051E0001ADC991C5B78009101938B1805930C9B3A
:1051F000002B02D0019BE41A0134049BE5B2002786
:10520000002B1BD10025E4B20295019B029A934228
:10521000DDDD082600273DE002329B180131DDE785
:10522000039B2800F118C9B2FFF7B2FF0136204BEB
:105230005B789E42F4DB01350137EDB2019BBB4246
:10524000E0DD0026F3E7082E08D1059B009A934283
:10525000BDD01300002601331578009301231D42B1
:1052600015D0039BF918049BC9B2002B1CD0832CCA
:105270000DD80F290BD88422CB0853437D3A0A401E
:10528000802111410B481B19C25C8A43C2546D1026
:1052900001370136064B5B789F42D4DB029B013419
:1052A00001330293E4B2B0E72000FFF771FFEEE7AD
:1052B00000000010B810001070B50D0004000122AD
:1052C000FBF71EF8290001222000FAF7F5FF70BD58
:1052D0000122F8B5082107001000FAF7EDFF0724B6
:1052E0000826002231000120FAF7E6FF3A000125E6
:1052F000224102212A400020FAF7DEFF2A00310075
:105300002800FAF7D9FF013CEBD2F8BD002210B516
:10531000040011000220FAF7CFFF2000FFF7D8FFAA
:1053200010BDF7B5012300245026134D00930194BE
:1053300076426A46A300D05800273043C0B2FFF738
:10534000E5FF0020FFF7E2FF1020FFF7DFFFE0207E
:10535000FFF7DCFF012200210220FAF7ADFFE85D34
:105360000137FFF7B5FF842FF4D18435012C00D12C
:10537000F7BD0124DDE7C046B81000107047704744
:105380000122024B80331A707047C046A8080010F3
:10539000054B002219007C310A80190086310A7001
:1053A000A43301321A707047A808001010B5074CDA
:1053B000230085331B78002B03D00C217620FFF7C8
:1053C00049FE0123A434237010BDC046A808001074
:1053D000044B84331A787F2A02D8FF221A70704750
:1053E0000022FBE7A808001010B5064C7C34238887
:1053F000002B02D0FFF782FE10BDFFF7B1FD208029
:10540000FAE7C046A808001010B5074C2300853302
:105410001B78002B03D00B217620FFF71BFE012306
:10542000A434237010BDC046A80800108022024B8F
:1054300052007E331A807047A80800100122024BE8
:105440007E331A807047C046A80800100022024B25
:105450007E331A807047C046A808001070470022AB
:10546000014B80331A707047A80800100122024BCC
:10547000A4331A707047C046A80800100122024BDE
:10548000A4331A707047C046A80800100022054BCC
:1054900084339A56002A02DC01221A7070470022D7
:1054A000FBE7C046A8080010054B00211A00813216
:1054B000117082331A7851424A411A707047C046BF
:1054C000A8080010054B00211A00823211708133A8
:1054D0001A7851424A411A707047C046A808001015
:1054E00070B5114C114923007C331A88885C002860
:1054F00003D1002A01D0188070BD230085331B78AA
:10550000002B02D0FFF782FDF6E725000123863548
:105510002B70FFF7E9FC2B78002B01D0FFF776FD0D
:10552000002386342370E7E7A8080010D400001099
:10553000F0B585B00500019114008A4206DD002215
:10554000002302604360002005B0F0BD1000FFF7AB
:1055500072FB06000F002868696807F0EDFD0290F5
:1055600003913000390007F0C9FD07F0E5FD0B009D
:1055700002000298039908F011F9FBF7FFF907F010
:10558000BDFD019B03C59C4203D10843411E8841D8
:10559000DAE707F0D1FDFFF71FFC019BC1171C1BC9
:1055A000E30FA04259410800CEE773B51D00114B2F
:1055B00014001E001A00B836C8320090019110681D
:1055C0005168306071609068D168B060F1601E0011
:1055D000A833D836306871689C60DD601060516017
:1055E000B068F1689060D1600099019A19605A60C2
:1055F00073BDC046A808001073B514000C4A009093
:10560000019116001D000B4B983618685968103B25
:10561000186259629869D9699862D962B342F4D123
:1056200000980199A8329460D5601060516073BDF4
:10563000A808001070090010F8B51F00074B0400FF
:10564000A4331B780D001600002B05D02000290084
:1056500032003B00FFF7D0FFF8BDC046A80800109D
:10566000D0B5154C154A23000833DB6F13400CD11D
:10567000134AA534516E002902DD21705366D0BD56
:105680002378536604232370F9E7230086331B78BD
:10569000002BF4D00A4B58690A4BE358A434C01AC3
:1056A00009F0B0FA0022084B08F078F80023002235
:1056B000FFF7C2FF0123E6E7A808001000FFFF0084
:1056C000180000107C07000000408F4010B50C4C03
:1056D00000232100A83100228868C96806F0C6FFAF
:1056E00003000120002B09D0B8340023A068E16832
:1056F000002206F0BBFF43425841400010BDC046A7
:10570000A808001070B5FFF7E1FF03000020012B8F
:1057100016D00C4B0022A8331C685D680A4B200091
:10572000290006F0B3FF00280AD0084B0022200011
:10573000290006F0BFFF431E984143420120184054
:1057400070BDC046A80800100000F03F0000F0BF88
:10575000F8B55F4D2B0087331B78082B07D1FBF77B
:105760009FF80028FBD12B00072287331A70FBF724
:1057700097F8584F0400031EBE6E3FD1032E2DD163
:105780002B0085331B78002B05D12B007A331B7837
:10579000002B00D134002B0081331A78002A03D06B
:1057A000052E01D000221A702B0082331A78002AAD
:1057B00003D0092E01D000221A702B00002284335E
:1057C0009A56002A05D02F2E0FD0572E0DD000222A
:1057D0001A703A2E09D1FFF743FF06E0532E02D18B
:1057E0002B008533D3E7002ED5D12A0000237A324F
:1057F00079351370BB662B70FB663DE02A00813261
:105800001278002A21D02834FB22053B134204D110
:105810002000282106F00CFF0C00B44242D1032CDA
:105820002CD12B0085331B78002B15D00025FB6E67
:10583000022B32DD642D1FDC0120FAF705FDFBF79A
:105840002FF8002810D00135F1E72A0082321278B3
:10585000002AD9D05034D7E71F4C0120FAF7F4FCC6
:10586000FBF71EF8002801D1002405E0013C002CC4
:10587000F3D101237A352B702000F8BD532CD5D0FD
:10588000164D0120FAF7E0FCFBF70AF80028EBD0F0
:10589000013D002DF5D1A034EEE7114A9542CBD160
:1058A0000133A9E72B000833DA6F0E4BBC661A42AE
:1058B000E2D1032C01D0532CDED1C820FAF7C4FC6E
:1058C000FAF7EEFF0028CFD0012379352B70CBE714
:1058D000A808001018000010D1070000E90300001C
:1058E0005902000000FFFF00F8B51D4B1A6E002A98
:1058F00035D101321A66FFF72BFF0028FBD172B6B3
:105900008026802180208027164D174A2B6876003C
:1059100013402B60154BC9004001DF67DE67D96774
:10592000D867FAF7DFFD124A0F49136880200B4051
:105930001360AC230F4A5B0113608021C0220E4C20
:105940005200C9004001A750A650A150A0502A689B
:1059500013432B60276026602160206062B6F8BD8B
:1059600018000010048204407FEAFFFF04E100E019
:10597000008204400882044000E100E0F0B585B0F8
:1059800002900C0003921F0006F030FB451E002D14
:1059900001DB002C01DC05B0F0BD029B2100585D4D
:1059A0000123039A00933B00FFF706FC241A002F03
:1059B00002D1013C013DEAE70026B542F9D0064B91
:1059C0005B789E42F5DA039BE0B29919C9B2FFF702
:1059D000DFFB0136F3E7C04600000010F0B5264DAE
:1059E00085B02C007034200006F000FB0023C2B20A
:1059F000A275E37523766376A376E3769A4201D0A7
:105A00000133237670352B782D2B01D12C3BAB76CF
:105A10000022C3B2039316001500140011000123E5
:105A2000029201920398884212DC002D02D0124BA0
:105A30007033DC75002E03D00F4B0199703359760B
:105A4000002A03D00C4B029A7033DA7605B0F0BD11
:105A5000094870300F5C01312E2F07D0452FE1D15E
:105A6000085CCCB201942D2803D01E001D001C0040
:105A7000D8E71A000293F8E7180000107FB51C4C15
:105A80000600230070331B7E002B1DD1194D2B0007
:105A90009C331B78002B17D1174BA835196C5A6C07
:105AA000009101929A6CDB6C009801990292039329
:105AB000029A039BFFF7C0FD009A019B2A606B606E
:105AC000029A039BAA60EB600A4970347831A07D8A
:105AD000E27D0978821A8A4204DB637E002B01D1C1
:105AE000452E02D1024B70331E54FFF777FF7FBD66
:105AF00018000010A808001070ED000010B50B4C45
:105B0000230070331B7E002B06D13120FFF7B6FF38
:105B10000122074BA4331A707034637E002B04D12A
:105B20004520FFF7ABFFA37D637610BD1800001082
:105B3000A808001010B5074B7033DA7D002A08D191
:105B40001B78002B02D13020FFF798FF2E20FFF7A3
:105B500095FF10BD1800001010B53920FFF78EFF1B
:105B600010BD10B53820FFF789FF10BD10B53720E4
:105B7000FFF784FF10BD10B53620FFF77FFF10BD83
:105B800010B53520FFF77AFF10BD10B53420FFF7B0
:105B900075FF10BD10B53320FFF770FF10BD10B5B5
:105BA0003220FFF76BFF10BD10B53120FFF766FF05
:105BB00010BD10B53020FFF761FF10BDF0B5012317
:105BC000050085B02800029306F010FA2B780390A8
:105BD0002D2B09D000240194039B9C4208DB0298E2
:105BE000019B584305B0F0BD029B01355B42E9E7DC
:105BF000039B581E001BFFF71EF806000F00285DD0
:105C00000134303808F0C4FF32003B0008F0D0F90E
:105C1000060001980F0008F0BBFF02000B003000E7
:105C2000390007F09FFA08F07DFF0190D4E7F0B546
:105C300087B0019006F0DAF9019B03901B782D2BB9
:105C400026D101980130FFF7F2FF80231B06C91807
:105C500007B0F0BD019AD25C2E2A17D0452A00D198
:105C600002930133039A9342F4DB8C4206D1029BE8
:105C7000A34212D1019806F0B9F9040000250026CC
:105C80000027039B9D420ADB002011E01C00E8E78F
:105C9000214C002302942100E4E7029CEEE7029BE2
:105CA000AB420CD11800019B01301818FFF786FF9A
:105CB000FEF7C1FF32003B0008F07AF9C8E7AC42BA
:105CC00014DD0022154B3000390008F071F9060090
:105CD0000F00019B585D303808F05AFF32003B003E
:105CE00007F040FA06000F000135CAE7AC42FBDAC4
:105CF000601BFEF7A0FF019B04900591585D3038B2
:105D000008F046FF049A059B08F052F902000B00C8
:105D100030003900E4E7C046E703000000002440FB
:105D2000F0B5060085B00F0006F060F935000024DC
:105D30000390039AAB1B9A4201DD832C01DD05B071
:105D4000F0BD00232878210000933A00FFF734FAD1
:105D5000241801340135ECE7802273B500210725B2
:105D60002B4B2C4C920301912000DA67902206F015
:105D700005F9019B284EA360284B1A68AA431A60B4
:105D80000122196811431960254B1968A94319604C
:105D9000196811431960802322495B010868034395
:105DA0000B60214B1A6082323260204A12681968F7
:105DB0001F4B1868504306F05DF9E121090306F016
:105DC00059F910221B4B1C491A60030A0B6003236C
:105DD0001A4AC0B210603360194B1D60194B593517
:105DE00018680190080011001A682A40602AFBD147
:105DF0005F3A1D68154207D122708022124B920330
:105E00001A600523036073BD0D680195F1E7C04674
:105E100004E100E0281000100C800040A440044081
:105E2000A84004408080044098800440788004406A
:105E300018000010288000400480004000800040CE
:105E4000088000401480004000E100E0FA2110B515
:105E50000C4C8900206806F005FB0B4B984209D8D2
:105E600000230A4A013863611060094A136007225F
:105E7000084B1A60FFF770FFFAF722F9FAF7D8FA21
:105E800010BDC04618000010FFFFFF0014E000E046
:105E900018E000E010E000E010B5002839D08021C3
:105EA0001D4A13688B43136001231C490A681A4278
:105EB000FCD003221A4B1A6001230021194A1360F7
:105EC0001160136011681942FCD0174A174913601A
:105ED00080230C685B0223430B601100002804D16F
:105EE00080230D4A146823431360114B9A68824241
:105EF0000ED09860431E98410E4B404218400E4B06
:105F00000968C01806F0B6F80C4B1860FFF79EFF42
:105F100010BD034B1860CFE7388204400C8004406A
:105F20007080044074800440788004408080044085
:105F30000000001000512502001BB70018000010DF
:105F400010B5044816220021703006F017F8FFF74C
:105F500045FD10BD1800001070B5FFF7F1FF084BAC
:105F600008491A000C6C4D6C886CC96CA83214601E
:105F700055609060D1600022A4331A7070BDC04695
:105F8000A808001070ED000070B50E4C23009C3383
:105F90001B78002B14D10C4D7035280006F026F824
:105FA00000280DD02800FFF742FE2300A833186018
:105FB000596000220023B03422606360FFF7C0FF05
:105FC00070BDC046A808001018000010F0B589B0D8
:105FD000FFF7DAFF464B5C681B680093019400985A
:105FE0000199434BDC689B6802930394029A039BDC
:105FF000FFF722FB3F4B1C6C5D6C9E6CDF6C20003E
:10600000290032003B00FFF7F7FA3B4B2933FF33FF
:106010001C685D68384B20003933FF331A685B68B1
:1060200000920193344B29004933FF331A685B68AF
:1060300004920593304B00225933FF331E685F688A
:106040002E4B08F027FA22002B0007F0B1FF2A4B55
:10605000029003916933FF331A685B6820002900BE
:1060600007F0A6FF3200069007913B003000390090
:1060700007F09EFF02000B000698079908F00AFA45
:10608000029A039B07F08AFBFBF732FA00260027EF
:10609000194BB83318605960174B2000C0331E608D
:1060A0005F60049A059B290007F082FF009A019B1C
:1060B00004000D001000190007F07AFF02000B0029
:1060C0002000290008F0E6F9029A039B07F066FB1E
:1060D000FBF70EFA0122064B18605960064BB033ED
:1060E0001E605F60044BA4331A7009B0F0BDC04657
:1060F0005009001070ED0000A80800100000F03FEB
:10610000F7B5FFF741FF204C2500A83528686968DE
:10611000AA68EB68FFF790FA1C4B1E6C5F6C9A6CD8
:10612000DB6C00920193009A019B30003900FFF76D
:1061300063FA2300210029335931FF33FF311A68F4
:106140005B682600086849680092019307F026FB07
:10615000B8363060716021002300002600273931F5
:10616000C033FF311E605F6008684968009A019B78
:1061700007F014FB2300B0331E605F600123A434DA
:10618000286069602370F7BDA808001070ED00005A
:1061900070B5FFF7F9FE0B4C2500A835AA68EB682F
:1061A00028686968FFF748FA2300E83319685A68D5
:1061B00029606A609A68DB68AA60EB600123A434F6
:1061C000237070BDA8080010F8B5FFF7DDFE084B7E
:1061D000D8331E685F689C68DD6830002B0039008A
:1061E0002200FFF729FA0123014CA4342370F8BDE3
:1061F000A808001070B5FFF7C7FE0B4C2500A835A6
:10620000AA68EB6828686968FFF716FA074BA43498
:10621000996ADA6A29606A601A6B5B6BAA60EB6044
:106220000123237070BDC046A8080010F0ED0000E7
:10623000F0B587B0FFF7A8FE484B1C685D68484B77
:1062400020001E685F68474B29007933FF331A68C6
:106250005B6807F0ADFE444B009001911A685B68E3
:106260003000390007F0A4FE02000B0000980199ED
:1062700008F010F93B4B029003914933FF331A6841
:106280005B682000290007F093FE320004000D0037
:106290003B003000390007F08BFE02000B002000AD
:1062A000290008F0F7F82F4E00900191A8363068C9
:1062B0007168B268F368FFF7BFF92C4B1C6C5D6C1A
:1062C0009A6CDB6C04920593049A059B20002900CC
:1062D000FFF792F9009A019B0298039907F05EFA82
:1062E000204C0022B8342060616000211D4BC03377
:1062F00019605A60009801991B4B1A685B6807F097
:1063000057FE174B04001A685B680D00029803994A
:1063100007F04EFE02000B002000290008F0BAF83A
:106320000E4B04001A685B680D000098019907F095
:106330003FFE02000B002000290007F02FFA002288
:10634000306071600021074BB03319605A60012240
:10635000044BA4331A7007B0F0BDC046D00900103A
:10636000E0090010A8080010000A001070ED0000FD
:10637000F8B5FFF709FE0D4C00222500A8352E6860
:106380006F6800233000390007F012FE02000B0096
:10639000A868E96806F0E6FE2300B0331E605F607F
:1063A0000123A434286069602370F8BDA808001098
:1063B00073B5FFF7E9FD124B1E00A836B168F2680D
:1063C0000091019234687568009801991A00F832BA
:1063D000146055609060D1601A00B832106851683E
:1063E00014605560306071609068D168B060F16091
:1063F000009801999060D1600122A4331A7073BD96
:10640000A8080010F7B5FFF7BFFD144C25002300C6
:10641000F835A83319685A6829606A609A68DB6899
:10642000AA60EB602300B8331E685F689A68DB6877
:1064300000920193009A019B39003000FFF7B5F8F4
:1064400029686A682300D83319605A60A968EA6825
:106450009960DA600123A4342370F7BDA808001006
:10646000D0B52A4C8CB0220083321378002B07D091
:10647000012B03D10B3313700CB0D0BD013BFAE7F5
:10648000FFF782FD2300A83319685A680691079226
:106490009E68DF68069807990022002306F0E6F858
:1064A00000280BD0002200233000390006F0DEF86F
:1064B000002803D0873401232370DDE723000699E9
:1064C000079AE83319605A602300F0331E605F605A
:1064D00013000A00029203930022002304960597FA
:1064E0000092019308A80022094B06F061FB08996D
:1064F000099A2300A83319605A600A990B9A23005D
:10650000B03319605A60A434D5E7C046A80800101B
:106510000000F03F10B5FFF737FD064B1A00A83317
:10652000E83218685968106051609868D9689060BE
:10653000D16010BDA8080010F7B5FFF7C7F8284EC6
:10654000002803D0022387363370F7BDFFF7E2FF40
:106550003300A836B833776836681C685D68320047
:106560003B002000290007F095FF009001910200F8
:106570000B003000390006F089F80022194B002882
:106580002AD00098019906F0EDFD02000B002000D2
:106590002900FEF7E7FB009A019B04000D00300084
:1065A000390006F073F8002801D1009E019F0022F7
:1065B0000C4B30003900FEF7D5FB02000B00200029
:1065C000290007F0EBF800220023FEF7EEFF01227E
:1065D000034BA4331A70B8E730003900D3E7C04644
:1065E000A80800100000F03FF0B589B0FFF76EF882
:1065F000394C0590002804D002238734237009B059
:10660000F0BD26002936FF36FFF784FF3068716839
:106610000022324B07F03EFF069007910B0021004D
:106620002500270002003931F835A837FF312A63E9
:106630006B63086849683A687B680092019307F0C9
:1066400029FF009A019B286469641000190007F073
:10665000AFFC0B00224902000868496807F01AFFE6
:1066600028656965210023005931B833FF311A6864
:106670005B68086849680292039307F00BFF029A6F
:10668000039B286669661000190007F091FC0B0057
:10669000144902000868496807F0FCFE029A039B4F
:1066A0002867696700980199250007F081FC793512
:1066B000FF3502000B002868696807F0EBFE069AB8
:1066C000079B286069603A607B60B268F368A43415
:1066D000BA60FB60059B91E7A80800100000F03F3E
:1066E000F0090010100A0010F7B5FFF713FF134C64
:1066F0002500A835A868E968FEF71CFB2E686F68BE
:106700000090019130003900FEF714FB06000F00E5
:10671000009801990022002307F04AFC32003B0058
:1067200006F020FD2300B033286069600099019ACB
:1067300019605A600123A4342370F7BDA808001023
:1067400070B5FEF7C3FF104C012803D10223873434
:10675000237070BD2500A835FFF7DCFE2868696846
:1067600000220A4B07F024FC094B0A4A07F016F8EE
:1067700023002860696000200021B0331860596050
:10678000A4340123E4E7C046A80800100080764046
:10679000FB211940182D4454F0B587B0FEF796FF41
:1067A000334C012804D102238734237007B0F0BD95
:1067B0002500A835FFF7AEFE2E686F68300039005F
:1067C000FEF7B8FA0090019102000B00300039008A
:1067D00007F060FE0022274B07F0EAFB0022264B61
:1067E00007F0E6FBFAF7CAF80022234B06F0D6FFC3
:1067F00023000290039100200021B03318605960FB
:106800000298039908F08EF908F0C2F91B4A1C4B54
:1068100006000F0007F0CCFBFAF7B0F83200049046
:106820000591029803993B0007F034FE0022114BBA
:1068300007F0BEFB134A144B07F0BAFBFAF79EF8B9
:1068400002000B000498059906F08CFC00220F4B07
:1068500006F0A4FF00220E4B06F0A0FF009A019B59
:1068600006F080FCA4342860696001239DE7C046DF
:10687000A80800100000594084D797415555555538
:1068800043DEA341E4388EE35831454180842E41F4
:106890000088C34010B5084C230086331B78002BBA
:1068A00004D185342278002A01D0237010BDFFF76F
:1068B00031FE0123F9E7C046A8080010F0B587B003
:1068C000FFF728FE144D02A82C00A834E3680193BA
:1068D000A368009322686368FDF7B6F8029E039FE1
:1068E00026606760049A059BA260E360FEF7EEFEF7
:1068F00001280BD030003900FEF7D6FA2B002060BB
:10690000616000200021B033186059600123A43574
:106910002B7007B0F0BDC046A8080010F0B58BB0D2
:10692000FFF7F8FDFEF7EEFE204E07003500A83514
:10693000A968E8682A686B680190009106A8FDF7CD
:10694000AFF9089B099C1A4802930394069A079B87
:10695000184907F09FFD00220490059102980399C1
:10696000002307F025FB02000B000498059907F0AF
:1069700091FD340028606960B034002F0CD1029A78
:10698000039B0020002107F085FD2060616001234A
:10699000A43633700BB0F0BD002200232260636088
:1069A000FEF782FA28606960F1E7C046A808001087
:1069B000182D4454FB21F93F70B586B0FFF7AAFDAE
:1069C000FEF7A0FE124E05003400A834E36802A8CA
:1069D0000193A368009322686368FDF761F9029848
:1069E000039920606160049A059BA260E360002D1A
:1069F00009D0350000220023B0352A606B60FEF715
:106A000053FA206061600123A436337006B070BD74
:106A1000A808001070B5FFF77DFD0A4C2500A835C9
:106A2000AA68EB6828686968FAF716FE23002860F0
:106A3000696000200021B033186059600123A4343C
:106A4000237070BDA8080010F8B5FEF73FFE144C87
:106A5000002803D0022387342370F8BDFFF75AFDC6
:106A600025002300A835B8331E685F682868696868
:106A700032003B0007F00EFD00220A4B07F098FAA7
:106A80003B00320006F08AFE230028606960002087
:106A90000021B03318605960A4340123DCE7C046FC
:106AA000A80800100000594070B5FEF70FFE114C09
:106AB000002803D002238734237070BDFFF72AFD1E
:106AC00025002100A835B8312A686B680868496834
:106AD00007F06EFA084B002206F060FE23002860E3
:106AE000696000200021B03318605960A43401238C
:106AF000E2E7C046A808001000005940F0B58DB08C
:106B0000FFF708FD1D4C2500A835A968E8682A682C
:106B10006B680190009108A8FDF79AF80A9A0B9B00
:106B2000089E099F164906920793086C8A6BCB6BE7
:106B3000496C0090019108A8FDF78AF80A9A0B9B0E
:106B400008A804920593089A099B02920393069A57
:106B5000079B0092019332003B0006F029F8089A47
:106B6000099B2A606B600A990B9A2300B033196065
:106B70005A600123A43423700DB0F0BDA8080010A2
:106B8000F0ED000030B587B0FFF7C4FC0C4D02A853
:106B90002C00A834E368A4350193A368009322680D
:106BA0006368FDF755F8029A039B22606360049ABC
:106BB000059BA260E36001232B7007B030BDC04687
:106BC000A808001030B58BB0FFF7A4FC104C2500CE
:106BD000A835AA68EB680492059328686968009252
:106BE00001930290039106A82A686B6805F06CFD7A
:106BF000069A079B2A606B600899099A2300B033B4
:106C000019605A600123A43423700BB030BDC04614
:106C1000A8080010D0B5FEF759FD134C002803D08A
:106C2000022387342370D0BDFFF774FC2300B833F0
:106C30001E685F682300A8331A685B68300039005B
:106C400007F028FC0022094B06F08CFA02000B002A
:106C500030003900FEF786F800230022FEF7A5FC7D
:106C6000A4340123DEE7C046A80800100000F03F6E
:106C7000F0B591B0FFF74EFC644E33002933FF337B
:106C80005C681B68009301940098019933003933C4
:106C9000FF335C681B680293039433005933FF335E
:106CA0005C681B680493059433007933FF331A68DA
:106CB0005B6807F07DF9049A059B04000D000298BB
:106CC000039907F075F902000B002000290007F076
:106CD000E1FB33004933FF330A900B911A685B687C
:106CE0000098019907F064F9029A039B04000D00D3
:106CF0001000190007F05CF902000B0020002900C9
:106D000007F0C8FB33006933FF33069007911A6818
:106D10005B680098019907F04BF9049A059B040001
:106D20000D001000190007F043F9370002000B00B6
:106D30002000290007F0AEFBA8373B687C68089369
:106D40000994BA68FB680C900D9108980999FEF7B0
:106D500073FC2F4B1C6C5D6C9A6CDB6C0E920F936A
:106D60000E9A0F9B20002900FEF746FC0C9A0D9B03
:106D70000698079907F01CF9FAF7BAFB34000200ED
:106D80000B000A980B9906F009FDB8343300206017
:106D9000616000220021C03319605A60089A099B83
:106DA0000098019907F004F9029A039B07F072FB1F
:106DB0000A9A0B9B07F0FCF8069A079B04000D004B
:106DC0000498059907F0F4F802000B002000290050
:106DD00006F0C8F9069A079B04000D000098019977
:106DE00007F0E6F802000B002000290006F0D6FCB0
:106DF00033003860796000220021B03319605A6096
:106E000033000122A4331A7011B0F0BDA80800109D
:106E100070ED0000F0B587B0FFF77CFBFEF756FC85
:106E2000244C012819D02500A8352E686F6800224F
:106E3000214B3000390005F01FFC00280DD139002E
:106E4000300007F06FFE07F0A3FE02000B003000D9
:106E5000390005F00BFC00281DD12500A835286855
:106E600069680022144B06F07DF902000B00E86807
:106E7000A9680190009102A8FDF72AFD029A039BE0
:106E80002A606B60049A059BAA60EB600123A4341E
:106E9000237007B0F0BD084B002230003900FDF729
:106EA00061FF23002860696000200021B033186072
:106EB0005960EBE7A80800100000F03FF0B587B07C
:106EC000FFF728FB1A4C2500A835AE68EF683000A4
:106ED0002A686B68390002920393FDF72BFF00903C
:106EE000019102980399FDF725FF00220490059176
:106EF00000980199002307F05BF8049A059B06F0BF
:106F000031F902000B000298039907F0C3FA009AC6
:106F1000019B2860696025003000390007F0BAFA4B
:106F20000123B035A43428606960237007B0F0BD38
:106F3000A8080010F8B5FEF7C9FB194C012803D1C9
:106F4000022387342370F8BD2500A835FFF7E2FA45
:106F5000A868E9680022134B06F020FC02000B0031
:106F600006F000F9104A114B07F022F80022060043
:106F70000F00286869680B4B06F010FC02000B003C
:106F800006F0F0F8094B084A07F012F82300B03376
:106F90001E605F6028606960A4340123D2E7C046A8
:106FA000A808001000807640182D4454FB210940A9
:106FB000F0B585B0FEF78AFB3D4C012804D10223D1
:106FC0008734237005B0F0BDA834FFF7A3FA6568D5
:106FD000246820002900FDF7ADFE00900191020019
:106FE0000B002000290007F055FA0022314B06F073
:106FF000DFFF0F00060007F095FD040007F0C8FD55
:1070000002000B003000390007F044FA0022294B3F
:1070100006F0CEFF0022284B06F0CAFFF9F7AEFCBF
:107020000022254B06F0BAFB0022224B06000F007F
:1070300005F040FB002808D03000390000221D4B2D
:1070400007F028FA06000F0001343B2C08DD0098F9
:1070500001990022194B06F085F8009001913C3C03
:107060006420604307F094FD002202900391009891
:107070000199134B06F09CFF02000B000298039944
:1070800006F070F832003B0006F06CF80C4B002262
:1070900006F084FB064D0B4B186059602B00002056
:1070A0000021B033186059600123A4352B7089E7A3
:1070B000A808001000004E4080842E410000F03FE0
:1070C0000088C34050090010F7B5154C23009C33CD
:1070D0001B78DB0603D52B22124BE254F7BD2500AB
:1070E0002600B835A836FFF715FA326873682868A5
:1070F000696806F037F8B268F36800900191A868F3
:10710000E96806F02FF806000F00009801993B008F
:107110003200FEF74AFA0123A4342370DEE7C046AA
:10712000A808001076070000F0B589B0FEF7CEFA87
:10713000394C0590002804D002238734237009B00D
:10714000F0BD26002936FF36FFF7E4F93068716894
:107150000022324B06F006F8069007910B00210042
:107160002500270002003931F835A837FF312A639E
:107170006B63086849683A687B680092019305F080
:10718000F1FF009A019B286469641000190006F061
:107190000FFF0B00224902000868496805F0E2FF72
:1071A00028656965210023005931B833FF311A6819
:1071B0005B68086849680292039305F0D3FF029A5E
:1071C000039B286669661000190006F0F1FE0B00AB
:1071D000144902000868496805F0C4FF029A039B3D
:1071E0002867696700980199250006F0E1FE793566
:1071F000FF3502000B002868696805F0B3FF069AA6
:10720000079B286069603A607B60B268F368A434C9
:10721000BA60FB60059B91E7A80800100000F03FF2
:10722000F0090010100A0010F7B5154C23009C332C
:107230001B78DB0603D52D22124BE254F7BD250047
:107240002600B835A836FFF765F9326873682868F4
:10725000696807F01FF9B268F36800900191A868A7
:10726000E96807F017F906000F00009801993B0044
:107270003200FEF79AF90123A4342370DEE7C046FA
:10728000A808001076070000D0B5184C8AB023007B
:107290009C331B78DB0604D52A22154BE2540AB036
:1072A000D0BDFFF737F923002100B83318001E685E
:1072B0005F68A8318A68CB68049205930A684B68B6
:1072C000029203938268C36806A800920193320079
:1072D0003B0005F0F9F9089A099B06980799FEF713
:1072E00064F90123A4342370D9E7C046A80800102C
:1072F00076070000F0B5A1B0FFF70CF97B4D2B002D
:107300002C0084331B78A8345BB20693012B4CD13C
:1073100022686368A668E7681000190005F022FF7C
:1073200008900991FBF766F932003B000C900D9133
:107330003000390005F016FF0A900B91FDF71AFA9C
:1073400002000B000C980D9905F00CFF06000F00D1
:107350000A980B99FDF7C8F932003B0006F01EFAB7
:107360000A900B9108980999FBF7DCF932003B0071
:1073700006F014FA002206000F000A980B99002369
:1073800006F016FE02000B003000390005F0EAFEA0
:107390002B00B033206061600A990B9A19605A6023
:1073A000069BA4352B7021B0F0BD069B276866684C
:1073B000013338D100224E4B18A8049205930022C5
:1073C000002302920393A268E368009201933A00BB
:1073D000330005F079F91A99189A00911B99199BB5
:1073E000019118A8FCF730FB0022424B18A8049228
:1073F0000593802300221B06029203931A9A1B9B7B
:1074000000920193189A199B05F05EF9189A199B3E
:10741000226063601A991B9A2B00B03319605A607E
:10742000A4350123BEE7FEF751F901286ED02B00E9
:107430007E331B78002B34D02F4A73005B089342B5
:1074400008DC012300220093380000233100FCF700
:1074500079FD08E0294A934213DD3A0033003800F1
:10746000310007F017F82B00A83318605960B035C9
:10747000002300242B606C6001221C4BA4331A7083
:1074800091E71CAA31003800FCF74EFF1E9A1F9BA3
:107490000221400008400139081A00901C981D99EB
:1074A000D5E72B007F331B78B0350022002B1BD093
:1074B000134B3800310006F071F906000F00FAF79F
:1074C00041FB3200069007913B0000200D4906F079
:1074D000E1FFFAF737FB02000B000698079906F068
:1074E0005DF920606160C3E7074BE2E7A808001080
:1074F0000000F03F0000F0BFFB21E93FFFFFEF7FFE
:10750000000069400000E03F008066403A00E56806
:10751000A46833003800310005F024FE069007917E
:10752000FDF728F9220006000F002B00200029009B
:1075300005F018FE08900991FBF75CF802000B00BB
:107540003000390005F00EFE06000F00FBF74EF884
:1075500000229C4B05F090F8002800D1F7E0069837
:107560000799FBF743F80A900B9108980999FBF7E4
:107570003DF8954A0C900D910A980B99934B06F0A3
:107580000DF90022002304000D0005F093F80022FD
:107590008F4B002800D10BE12000290005F0E2FD0F
:1075A00007F0C0FA07F0F4FAA822884BD2050600CB
:1075B0000F0006F0FDFC02000B000A980B9906F084
:1075C00069FF802204000D005205824B3000390013
:1075D00006F0EEFC02000B002000290006F05AFF26
:1075E0007D4A04000D007D4B3000390006F0E0FCC0
:1075F00002000B002000290006F04CFF02000B00E7
:1076000006F0D6FC0C9A0D9B0026002710901191D5
:107610001000190006F0CCFC002234003D00704B35
:10762000129013910E920F930C920D930A920B935A
:1076300000226B4B2000290005F094FD0A9A0B9B59
:1076400004000D0006F0B4FC00220A900B91644B7C
:107650002000290005F086FD04000D0002000B004B
:107660000A980B9906F0A4FC0C9A0D9B0A900B91BA
:107670001098119906F09CFC0E9A0F9B0C900D919E
:107680001298139906F094FC02000B000E900F91D3
:107690000C980D9905F066FD0A9A0B9B06F07EF892
:1076A00032003B0005F05EFD0022169017914C4B16
:1076B0002000290005F056FD04000D0002000B001B
:1076C0000A980B9906F074FC002206000F00444B48
:1076D0002000290005F046FD02000B0004000D000B
:1076E0003000390006F064FC0C9A0D9B0A900B9157
:1076F0001098119906F05CFC0E9A0F9B0C900D915E
:107700001298139906F054FC0C9A0D9B0E900F9151
:1077100006F0C0FE0A9A0B9B06F040F802000B0030
:10772000149015911698179905F01CFD02000B0096
:1077300006000F001498159906F030F8FAF756FF76
:10774000284A294B04F0ACFF002800D070E7002243
:1077500000233000390004F089FF00282DD108985B
:107760000999FAF7DFFF32003B0006F017F8040032
:107770000D0006980799FCF7B7FF32003B0006F0B2
:107780000DF8002206000F0000232000290006F05B
:107790000FFC02000B003000390005F0E3FC134B36
:1077A0001A00B033A832106051601C605D6063E65F
:1077B0002000290006F06EFEF2E600240C4D0020A9
:1077C0000C49ECE70000D03F182D4454FB21094040
:1077D0000000E03F460B213E6EC0453163626A3CCB
:1077E0000000F03F4F64A14091B49F3CA8080010F6
:1077F0000000F07F0000F87FF0B5842597B0FEF719
:1078000089FE824B814C5D57A834012D42D12668F8
:107810006768A268E3683000390006920793FAF7B8
:1078200081FF0890099106980799FCF75DFF020017
:107830000B000898099906F0BBFB089009913000ED
:107840003900FAF7D7FE06000F0006980799FCF7F3
:1078500091FF02000B003000390006F0A9FB002266
:1078600006000F0008980999002306F0A1FB02000A
:107870000B003000390005F075FC644B206061603E
:107880000899099AB03319605A60604BA4331D708F
:1078900017B0F0BD22686368069207936B1C5AD13B
:1078A00006980799E36800220893594B05F05AFCA3
:1078B000A768089D02000B0001950EA80097FBF732
:1078C00027F80E9A0F9B069807990A920B93109A25
:1078D000119B0C920D9300224D4B06F0DBFD0195A0
:1078E0000B00020000970EA8FBF712F8109A119BEC
:1078F0000EA8049205930E9A0F9B029203930C9A82
:107900000D9B009201930A9A0B9B04F0DDFE069AF0
:10791000079B0E980F9905F025FC089B06000D00AB
:10792000109811993A0005F01DFC32002B000191CE
:1079300000900EA8FCF78CF90E9A0F9B22606360F2
:107940001099119A314BB03319605A6001222F4BB4
:10795000A4331A709CE7FDF7B9FE2C4DB035012811
:1079600025D02A4B00267E331B780027002B08D019
:1079700006980799FCF7FEFE206061602E606F603C
:10798000E4E7224B00227F331B78002B0DD0214BE4
:107990000698079905F002FF02000B0000201E491F
:1079A00006F078FDFAF7CEF8E6E71C4BF0E714ABEB
:1079B00012AAA068E168FAF769FF06980799FCF730
:1079C00093FE149A159B06F0F3FA07000E00089137
:1079D00006980799FCF7CEFE129A139B06F0E8FA78
:1079E00000220690079100233800089906F0E0FA7B
:1079F0000B0002000698079906F04CFD80231B0639
:107A0000F618206061602F606E609FE7A808001084
:107A10000000F03F000069400000E03F0080664049
:107A2000F0B591B0FEF776FD684D2B002C00843345
:107A30001B78A8345BB20893012B42D12668676893
:107A4000A268E3683000390006920793FAF7D2FD86
:107A50000A900B9106980799FCF746FE02000B006E
:107A60000A980B9906F0A4FA0A900B91300039009D
:107A7000FAF758FE06000F0006980799FCF77AFE01
:107A800002000B003000390006F092FA00220600D6
:107A90000F000A980B99002306F08AFA02000B00E7
:107AA0003000390005F05EFB2B00B03320606160D0
:107AB0000A990B9A19605A60089BA4352B7011B073
:107AC000F0BD636826680693089B013344D1A26821
:107AD000E36808920993049205933200069B0CA870
:107AE00002920393089A099B009201933200069B2D
:107AF00004F0EAFD0C980D990022354B05F032FB9D
:107B00000B000E99020000910F990CA80191FAF751
:107B1000FFFE0C980D993200069B05F023FB089A96
:107B2000099B06000F000E980F9905F01BFB320011
:107B30003B00019100900CA8FCF78AF80C9A0D9B71
:107B4000226063600E990F9A2B00B03319605A605F
:107B50000122A4352A70B2E72F00FDF7B7FDB03738
:107B6000012823D02B007E331B78002B0ED0300051
:107B70000699FCF7B9FD20606160002300243B609A
:107B80007C602B000122A4331A7098E72B007F330E
:107B90001B780022002B07D00E4B3000069905F011
:107BA000FDFDF9F7CFFFE6E70B4BF6E7E068A168CC
:107BB0003200069B019000910CA8FCF71DFE0C9A68
:107BC0000D9B226063600E9B0F9CD8E7A8080010F5
:107BD0000000F03F0000694000806640D0B5224CB4
:107BE0008CB023009C331B78DB0604D52F221F4B5F
:107BF000E2540CB0D0BDFEF78DFC2300A833196809
:107C00005A68069107929E68DF68069807990022D5
:107C1000002304F02BFD00280BD0002200233000AD
:107C2000390004F023FD002803D08734012323709A
:107C3000DFE72300B8331868596804960597069E55
:107C4000079F029603979A68DB68009201930200EF
:107C50000B0008A804F0ACFF089809990A9A0B9B3E
:107C6000FDF7A3FCA434E1E7A808001076070000A4
:107C700070B58AB0FEF74EFC154C2100B83188680B
:107C80000A684B680090C96801912100A8310D680D
:107C90004E68029503968868C9680490059106A805
:107CA000FCF7A2F80699079A2300F83319605A6086
:107CB0000899099A9960DA60089A099B06980799C9
:107CC000FDF773FC0123A43423700AB070BDC046D5
:107CD000A808001070B58AB0FEF71CFC134C1449BC
:107CE00025002600086C8A6BCB6B496CA835009088
:107CF00001912868696802900391F836A868E968DC
:107D00000490059106A8FCF76FF8069A079B08985F
:107D10000999326073602A606B600123A434B060FB
:107D2000F160A860E96023700AB070BDA808001077
:107D3000F0ED000030B587B0FEF7ECFB0C4D02A86B
:107D40002C00A834E368A4350193A368009322684B
:107D50006368FCF787FD029A039B22606360049AC4
:107D6000059BA260E36001232B7007B030BDC046C5
:107D7000A808001030B587B0FEF7CCFB0C4D02A868
:107D80002C00A834E368A4350193A368009322680B
:107D90006368FAF7BDFD029A039B22606360049A50
:107DA000059BA260E36001232B7007B030BDC04685
:107DB000A8080010842210B552000021014804F0E8
:107DC000DDF810BDB810001010B508210120FDF736
:107DD00073FA02210020FDF76FFA00210220FDF75F
:107DE0006BFA06210220FDF767FA03210800FDF770
:107DF00063FA032100220800F8F75EFA0022062148
:107E00000220F8F759FA012206210220F8F754FA65
:107E1000FFF7D0FFFDF785FAA220FDF777FAA02043
:107E2000FDF774FAC020FDF771FAF820FDF76EFA3D
:107E30000020FDF76BFA0A20F8F706FA4020FDF75C
:107E400065FA2C20FDF762FA3220F8F7FDF92E20B2
:107E5000FDF75CFA3220F8F7F7F92F20FDF756FA14
:107E60000A20F8F7F1F92520FDF750FA0A20F8F773
:107E7000EBF98120FDF74AFA0020FDF747FAAF2021
:107E8000FDF744FAA420FDF741FA10BD70B50A20B1
:107E9000F8F7DAF9FDF75CFC0128F8D01D4D2C004D
:107EA00048342379002B19D0002323712372E37007
:107EB0006379002B07D1C122022152000E20F8F76E
:107EC00099FA012363710C22012148352B790800AE
:107ED0001A43AB795B001A43F8F78CFAAC20FDF734
:107EE00015FAAE20FDF712FAA520FDF70FFA0020D3
:107EF0000121F8F717FB0020F8F798FC002802D1C1
:107F00000121F8F70FFBFFF75FFFFFF753FFFDF7C6
:107F100008FA70BD18000010CC2270B5D200002104
:107F20000C4804F02BF8EB230B4CDB00E518103366
:107F3000E05806F067FE094A094B05F02FFCEC23D8
:107F4000DB00E4180022002328606960226063607F
:107F500070BDC046B0090010A80800100000C0FFA6
:107F6000FFFFDF411B4B1C491A002932FF3270B55D
:107F70000C6C4D6C886CC96C146055609060D1605D
:107F80001A003932FF32146055609060D1601A00D7
:107F90004932FF32146055609060D1601A00593246
:107FA000FF32146055609060D1601A0079336932F5
:107FB000FF33FF329860D960146055609060D160E3
:107FC0001C605D60FDF7BCFF40220021034803F008
:107FD000D5FF70BDA808001070ED0000500900101A
:107FE00070B50F4C0F2223000E4E78331A703000FC
:107FF0000532002103F0C2FF230000259C330A4A0A
:108000001D700A4B0C320A493000E55403F0ABFFF7
:1080100023008334A0331D602570FDF791FF70BDF0
:10802000A8080010300900100000001076070000BA
:10803000C8F60000F7B56F4C260083363378002B66
:1080400016D0230085331B78002B10D06A4D703575
:10805000280003F0CBFF012804D12800FDF7AEFD76
:1080600001303070833421787620FCF7F3FFF7BDC0
:10807000230086331B78002B00D1A2E0FDF784FF9C
:1080800023007C331A885D4B9B185D78FDF71EFB3F
:1080900001280BD10C2D05D8594BEB409843C0B2A9
:1080A000002809D0022387342370E0E7022803D197
:1080B0002B00083B032BF5D92300A8331E685F680B
:1080C0002300681EB8331A685B68009201930B287E
:1080D00019D804F0B1FA061B262D343B4E5D6063BF
:1080E00066692100A83100228868C968002304F06D
:1080F000BDFA002812D0002200233000390004F01D
:10810000B5FA00280AD0FCF781FF07E0002200231F
:108110003000390004F0C4FA0028F4D0A43401235C
:10812000C2E7002200233000390004F0A5FAF3E78B
:10813000002200233000390004F0BCFAECE70022F2
:1081400000233000390004F0A1FAE5E72100230004
:10815000A831B8339A68DB688868C96804F086FA81
:108160000028D0D0009A019B3000390004F07EFA3C
:10817000D2E721002300A831B8339A68DB68886809
:10818000C96804F073FA0028C8D0009A019BB4E7CC
:10819000009A019BBCE7009A019BC4E7009A019BEF
:1081A000C8E7009A019BCCE72100A831002288682B
:1081B000C968002304F05AFA0028A4D00022002342
:1081C000D2E7230085331B78002B00D14FE7FFF760
:1081D00007FF220020219C3211702200012309494F
:1081E000A03211607834084908483370237003F0D6
:1081F000BAFE3CE7A808001018000010D4000010D8
:10820000C210000035800000A0F600003009001008
:10821000F7B5384C23009C331D78002D56D03648D6
:10822000364D030070331B78002B0FD12300A03391
:108230001B68AB4202D0324A93421DD1314BE35C02
:10824000002B19D17030304903F08DFE2300A0338C
:108250001A68AA4222D12B4AA25C2B2A12D12B4A9D
:108260001A602300A0331B68873498472378002BBB
:1082700029D0FDF765FE04E0230083331B78002B33
:10828000E4D1F7BD2D2A01D1214AE9E72A2A01D1FB
:10829000204AE5E72F2AE4D11F4AE1E718498A423C
:1082A000DFD1184AA25C2B2A01D11C4AD8E72D2A1B
:1082B00001D11B4AD4E72A2A01D11A4AD0E72F2A32
:1082C000CFD1194ACCE7FFF78BFEDAE7FDF75CFE6A
:1082D0002300A8331E685F689A68DB6800920193E8
:1082E000009A019B30003900A434FDF785F9257010
:1082F000C7E7C046A808001018000010A1960000AB
:108300005197000076070000A6F60000A59800002F
:10831000F99800004D990000B1990000159A0000ED
:108320005D9A0000A59A0000F99A0000F0B56D4C26
:1083300091B023009C331B785B070BD56A4B7033DD
:108340001B7E002B02D14920FDF798FBFFF760FF51
:1083500011B0F0BDFDF718FEFDF7B8F9012835D1D1
:108360002500A835AA68EB6806920793230080339E
:108370001B78B03400260027002B22D02A686B68B7
:108380000892099308980999069A079BF9F764F9E6
:10839000089A099B0A900B9106980799FBF7A2FA95
:1083A0000A9A0B9B266067602A606B60FCF77CFD75
:1083B00032003B00FDF720F901224A4BA4331A702A
:1083C000C6E72660676006980799F1E7022802D1A0
:1083D00087342070BCE72200B83210685168956875
:1083E000D6682200230008900991069507968032EE
:1083F0001278A8331868596800260027002A4CD044
:1084000023007E331B78002B0FD17F34237800228A
:10841000002B40D0354B05F0C1F902000B0004F0F1
:10842000A1FE334A334B05F0C3FD2E4B324C1A00EC
:10843000B0331E605F600023A83210605160049367
:10844000059402000B000CA8029603970096019772
:1084500004F03AF90E990C9A00910F990D9B019135
:108460000CA8FCF7FFF90E9B0F9C0CA80493059435
:108470000C9B0D9C02930394069B079C0093019414
:10848000089A099B04F020F90C980D990E9A0F9BFD
:10849000FDF78BF890E7194BBDE70024164D0296C7
:1084A0000397049405950200DC689B680CA8009370
:1084B00001940B0004F008F9089A099B0C980D9997
:1084C00004F050FE069A079B04000D000E980F99C9
:1084D00004F048FE06000F002000290032003B0097
:1084E000D6E7C046A8080010180000100000794028
:1084F000182D4454FB2109400000F03F00807640D5
:108500001FB5124C23009C331B789B070AD51048DB
:108510007030037E002B02D10E4903F024FDFFF7DB
:1085200077FE1FBDFDF7F6FF23008021A8339A6870
:1085300009060292DA68A434521803920299039A47
:108540009960DA6001232370EBE7C046A8080010A9
:1085500018000010AAF60000F0B5384B89B004935B
:108560000023374E0D00745C02A903900B739A42EE
:1085700004D01522334904A803F0F5FC2000FCF7D1
:10858000C3FC07002800FCF78DFD002F1ED000283B
:108590001ED12F007619767806AD0522002128001D
:1085A00003F0ECFCFE2E17D12749280003F0DBFC7A
:1085B000762C2DD13A00254BB6009E19B36C244978
:1085C000009304AB039803F0CEFC2CE000282CD0E1
:1085D0006F1EF45D765DDFE7FF2E01D11D49E4E7F4
:1085E0001D49FD2EE1D0632E0FD923004F3B012BF7
:1085F00004D92B2C02D0A31F012B06D8320011491D
:10860000233A280003F0AFFCD2E732001349F8E721
:10861000134BA400E358019500933A0004AB1149B1
:10862000039803F0A0FC09B0F0BD0D4BA400E35883
:108630002A0000930C4904ABC4E7C0462020000088
:10864000D400001091F7000055F70000F0ED000095
:10865000B7F60000AAF60000AEF60000B4F600007F
:1086600010F10000C0F60000CBF6000010B509289C
:108670000BD9094BFE2809D1E922D2009B181868B2
:10868000596806F04FFA03F08DFE10BD03228733C0
:108690001A700020F9E7C046A808001010B50300C2
:1086A0000E280CD90F20FE2B09D1E922044BD20051
:1086B0009B181868596806F035FA03F073FE10BD70
:1086C000A808001010B5682802D8FCF72DFD10BDD1
:1086D000094BFE280AD1E922D2009B181868596874
:1086E00006F020FA03F05EFEC0B2EEE70322873305
:1086F0001A700020EBE7C046A808001010B5030070
:1087000063280CD96420FE2B09D00130FD2B06D044
:10871000094CFF2B04D0032300208734237010BDA5
:10872000E923DB00E3181868596806F0FBF903F049
:1087300039FE6328EFDCF2E7A8080010F0B50D0061
:1087400085B0040017000268436810001900009209
:108750000193FCF741FB534A28601300A5331B78B3
:108760000600012B30D1A6321378BB4200DB7B1E02
:108770000F2F00DD0F27BE4203DA5B429E4200DB73
:1087800082E03000FCF757FA02000B0000980199D4
:1087900005F004F801262060616020686168FCF73C
:1087A0001BFBB0424FDB3F4B2F68A5331B78032BDD
:1087B00000D06CE0032E00D069E000223A4B033772
:1087C000226063602F603EE0022BDAD0032B4DD194
:1087D000009801990022354B03F06CFF002807D167
:1087E000009801990022304B03F050FF00284BD035
:1087F0003000FCF720FA02000B000098019904F009
:10880000CDFF20606160300003F0CCFD032103F058
:108810000FFF0E1E17D02B68009322686368029228
:108820000393009B002B10DD0800FCF704FA029A6A
:10883000039B05F0BDFB009B206061609F1B013620
:108840002F60002EA9D105B0F0BD03277F1A380094
:10885000FCF7F1F9029A039B05F0AAFB2060616026
:108860000420009B861BDF1B2F6096E7042BEAD1B8
:108870000E20801BFCF7DFF902000B000098019925
:1088800005F096FB2060616000232B60DBE7701E23
:10889000FCF7D1F904F032FC04F04EFC0137206003
:1088A00061608FE7A80800100000F03F00408F4093
:1088B000F0B58BB0FDF72EFE3B4C08A82300260038
:1088C000A83319685A68089109929A68DB68069279
:1088D00007930223A53635780F2205A93370FFF7D9
:1088E0002DFF0F2206A804A9FFF728FFA634357034
:1088F0002078FCF7A0F904F001FC032D03D10A2233
:10890000002303F043FC04F017FC089A099B0400C1
:108910000D0005F04DFBF8F731F822002B0004F0B4
:108920003DFF069A079B06000F002000290005F076
:108930003FFBF8F723F822002B0004F02FFF040080
:1089400005980D00FCF777F902000B0030003900A4
:1089500005F02EFB029003910498FCF76CF9124E7F
:1089600000900191002200232000290005F020FB47
:10897000009A019B05F01CFB029A039B370004F050
:10898000F1FB009A019BA83738607960370020001E
:10899000290005F00DFB0123B037A436386079605B
:1089A00033700BB0F0BDC046A8080010F0B597B00A
:1089B0000190190010000892099315001C00F8F7A7
:1089C00089FDC349049000280ED16300C14A5B08A9
:1089D000D3420ED4210000220023280003F060FEC1
:1089E000BD49002800D1BD49019803F0BCFA17B079
:1089F000F0BD002200232800210003F03DFE0028E6
:108A00000FD0B74BA5331B780895043B1A00531EB3
:108A10009A4180231B06E4181C9B0492013B099495
:108A20001C931C9A0BA908A8FFF788FE089B099CB9
:108A3000180021000693079404F060FB03000C006B
:108A4000029003910E930F9404F076FB0D00040046
:108A5000FCF7C2F9220005902B00461C06980799E6
:108A600005F018FD029B039A0690079113430F2708
:108A7000002B00D11027BF1B3800FCF7DCF80200E8
:108A80000B0004000D000698079905F091FAF7F71E
:108A900075FF04F033FB0C900D9104F04DFB2200A8
:108AA0002B0003F007FE002820D000220023012025
:108AB00000210C920D93029A039B12184B41100057
:108AC00019000B9C0E900F9104F036FBFCF784F913
:108AD000B0420BDB002C00D1B4E00598FCF7ABF8FA
:108AE00004F00CFB0E900F9101340B940B9C002CA6
:108AF00007D0200006F04CF8FCF76EF9E40F2418BC
:108B00000234774B1A00A533A63215781B782A0059
:108B1000032B02D1AA1BAE4200DC0F25002F00D18F
:108B200093E03B00974200DD13001C9A141BA11B2D
:108B30001A008B4200DD0A00D143C9170A40029295
:108B4000BA4200DB86E0BA1A39000CA8FCF7F0FC48
:108B500000281DD000220023012000210C920D933B
:108B60000E9A0F9B801859410E900F9104F0E4FA71
:108B7000FCF732F9B0420BDB0B9F002F68D0701E60
:108B8000FCF759F804F0BAFA0E900F9101370B97E1
:108B9000002C00DC0124A6425EDD341B22003100E3
:108BA0000EA8FCF7C5FC002809D00E980F990B23DE
:108BB00064220B93002303F0E9FA0E900F910B9BB4
:108BC0001C190B941422002111A803F0D7F9029A62
:108BD000444911A803F0C7F9049B012B08D101985F
:108BE00003F004FA019B2D2218183F4903F0BBF94A
:108BF000019803F0FBF9019B3C4918180E9A0F9B52
:108C000003F0B1F9029B002B4EDD019803F0EEF961
:108C1000019B11A918180C9A0D9B03F0A4F90B9B4A
:108C2000002B00D1E3E62E4B0198A5331B78042BD3
:108C300047D103F0DBF92E22019B2B49181803F0D2
:108C400092F9D4E6059E023650E701235B426CE7B9
:108C500001369DE702939BE7AE42B3DD771B3800F8
:108C6000FBF7E9FF3A0004000D000EA83100022EC8
:108C70000EDCFCF75DFC0E980F9904F05DFA220003
:108C80002B0005F095F904F039FA0E900F9199E751
:108C9000FCF74EFC0028EED0002301220E920F9329
:108CA0000B9B03330B938DE7029B002BB7D10198ED
:108CB00003F09CF9019B2E2218180B4903F053F97D
:108CC000ADE703F093F9019B0B9A18180849B6E732
:108CD000D3F6000000001080D8F60000D7F60000A0
:108CE000A8080010DCF6000091F70000E6F600008E
:108CF000EBF6000082B0F0B593B019931C9B18926C
:108D0000023BDA0FD3185B100390162200210CA847
:108D1000029303F033F91622002106A803F02EF97E
:108D20001A9C1B9D404E330080331B78002B5DD076
:108D30001898199922002B00F8F78EFC189A199BA5
:108D40000490059120002900FAF7CCFD33007E360F
:108D50007F331A78337804000D00134338D1002292
:108D6000324B05F025F9324A324B04F017FD1E262E
:108D700004000D00029B0CA80093049A059BFFF7CA
:108D800015FE0CA803F032F9029B984206D20CA8FB
:108D900003F02CF9029B5B001B1A0293029B06AFA7
:108DA000009322002B003800FFF700FE1E4B1A0034
:108DB000A5321278042A1FD133001F4900970CAA4C
:108DC000039803F0D0F813B0F0BC08BC02B0184709
:108DD0001E26002ACED00022184B05F0E9F8144ACE
:108DE000144B04F0DBFC04000D00C3E7189A199B38
:108DF000692604920593BDE780331B78002B04D0CD
:108E0000009733000CAA0E49DAE70022002329005C
:108E1000200003F045FC00963B000CAA09490028FD
:108E2000CED10949CCE7C046A808001000807640A2
:108E3000182D4454FB211940F0F600000000794041
:108E4000F7F6000000F700000AF7000070B5214CAB
:108E500023009C331B785B060AD51F487030037EC5
:108E6000002B02D11D4903F07EF8FFF7D1F970BD48
:108E70002500A835FDF788F8AA68EB6828686968B6
:108E8000FCF7DAFBEB23DB00E618154A154B3068DC
:108E9000716805F08DF804F013F9ED23DB00E05064
:108EA000114803F083FA05F073FE0D4A0D4B04F0F0
:108EB00075FCEC23DB00306071600022E6180023B3
:108EC00032607360AA60EB600123A434286069609B
:108ED0002370CCE7A808001018000010A6F60000C8
:108EE0000000C0FFFFFFDF411010001010B5284C3C
:108EF00028497034200003F08BF8002802D1FDF7D8
:108F00001FF810BD200003F071F800280FD02000DA
:108F100003F06CF80023201801380370200003F0E0
:108F200065F80028EDD11C4BA4331870E9E71A4B03
:108F30001A009C321278002A02D0FFF751F8E0E7BD
:108F40001A0085321278002A1AD07C331C88002C33
:108F5000D7D0124B185DFBF7D7FF002802D0A01C1A
:108F6000022107E02000FCF79DF801210300601CAE
:108F7000002BF5D14942FCF713F8FCF7BFF8C0E726
:108F8000200003F033F80028BBD1FCF7E5FFB8E779
:108F900018000010AAF60000A8080010D400001065
:108FA00010B50F4CFE2070342378492B13D00D4997
:108FB000200003F02DF80300FF20002B0BD00A49FE
:108FC000200003F025F80300FD20002B03D02078BB
:108FD000402801D9233010BD2000FCF7EFFDFAE74F
:108FE00018000010AAF60000A6F6000070B5FCF705
:108FF000CBFF1E4C25009C352B78002B0AD08534E6
:10900000FFF7CEFF2378002B03D0C1B27320FCF70B
:1090100021F870BD230086331B78002B15D0230068
:109020007C331A88124B9B185878FFF71FFB2300DC
:1090300087331B78002BECD10E4B2418E4182378CF
:10904000002BE6D1FBF7E2FFE3E7FEF7C9FF0523BC
:109050002B702300084AA0331A6001237834074993
:109060000748237002F07FFFD3E7C046A80800102E
:10907000D40000106C070000ED8F000013F7000013
:109080003009001070B5FCF77FFF224C25009C359D
:109090002B78002B16D0FFF783FF230085331D7834
:1090A000C0B2002D04D001006F20FBF7D3FF70BDCC
:1090B000FFF7DCFA184B2018C01805700123A43400
:1090C0002370F4E7230086331B78002B11D0230094
:1090D0007C331A88114B9B185878FFF7C7FA230086
:1090E00087331B78002BE2D10B4A201880180370BD
:1090F000E4E7FEF775FF05232B702300084AA03331
:109100001A600123783407490748237002F02BFFC7
:10911000CDE7C046A80800106C070000D40000107E
:10912000859000001FF700003009001070B5FCF7B3
:109130002BFF204C25009C352B78002B16D0FFF7F9
:109140002FFF230085331B78C0B2002B04D0010011
:109150006B20FBF77FFF70BDFFF788FA164B2018D6
:10916000C0180123A43403702370F4E7230086336E
:109170001B78002B0DD023007C331A880F4B9B18D3
:109180005878FFF773FA230087331B78002BE2D15E
:10919000E4E7FEF725FF05232B702300084AA033E0
:1091A0001A600123783407490748237002F0DBFE78
:1091B000D1E7C046A80800106C070000D4000010DA
:1091C0002D9100002BF7000030090010F8B5FCF7D6
:1091D000DBFE1D4C25009C352B78002B23D0FFF7A0
:1091E000DFFEC0B2FBF7A0FF184B984217DC02224B
:1091F000012103009446164F091AFA22CD18D20015
:10920000934206D0FA5C562A03D066460133B24335
:10921000F3D102214942491B4019FBF7C1FE00234B
:109220007C342380F8BDFEF7DBFE08232B7023007F
:10923000084AA0331A60022378340749074823708C
:1092400002F091FEEEE7C046A8080010CF0700002C
:10925000D4000010CD91000035F700003009001057
:10926000F0B5334C89B025009C352B78002B0BD002
:109270008534FFF795FE2378002B03D0C1B24B2035
:10928000FBF7E8FE09B0F0BD230086331B78002B06
:109290003CD0FCF779FE23007C331A88254B9B18C1
:1092A0005878FFF72BFA05002D0165192F00224E83
:1092B00009373100FBF726FD3068716807AB009372
:1092C00005AA06ABFBF7E8FC059A079BFF379E183B
:1092D0000798BA68FB6805960292039305F058FC5C
:1092E00002000B003868796803F03CFF029A039B88
:1092F000F835AA61EB61069B286169619E4201DD38
:10930000FBF784FE0123A4342370BBE7FCF73CFE8B
:10931000FEF766FE07232B702300084AA0331A606D
:109320000223783406490748237002F01CFEA9E79F
:10933000A8080010D4000010A009001061920000DD
:1093400042F7000030090010F0B5334C89B0250019
:109350009C352B78002B0BD08534FFF721FE23782A
:10936000002B03D0C1B24720FBF774FE09B0F0BD5B
:10937000230086331B78002B3CD0FCF705FE23002E
:109380007C331A88254B9B185878FFF7B7F90500EE
:109390002D0165192F00224E09373100FBF7B2FC71
:1093A0003068716807AB009305AA06ABFBF774FC45
:1093B000059B079AFF379E1A0798BA68FB680596BF
:1093C0000292039305F0E4FB02000B003868796811
:1093D00005F060F8029A039BF835AA61EB61069BE1
:1093E000286169619E4201DCFBF710FE0123A43471
:1093F0002370BBE7FCF7C8FDFEF7F2FD07232B70D7
:109400002300084AA0331A6002237834064907482B
:10941000237002F0A8FDA9E7A8080010D4000010EE
:10942000A00900104993000046F700003009001021
:1094300070B52D4C25009C352B78002B19D0FFF7EB
:10944000AFFD230085331B78C0B2002B1ED0010076
:109450004320FBF7FFFD70BD2D0165190935FF3570
:10946000326873682A606B60B268F368AA60EB6068
:1094700023E0230086331B78002B22D0FCF784FDE9
:1094800023007C331A88194B9B185878FFF736F95C
:1094900026002100F836A8310A684B6805003260C2
:1094A00073608A68CB68B260F360FBF72BFC652DB4
:1094B000D2DD2300032287331A700123A4342370E2
:1094C000C9E7FCF761FDFEF78BFD07232B70230036
:1094D000074AA0331A6002237834064906482370ED
:1094E00002F041FDB7E7C046A8080010D400001004
:1094F000319400004AF700003009001070B51F4C8D
:1095000025009C352B78002B12D0FFF749FD230056
:1095100085331B78C0B2002B15D001004C20FBF71F
:1095200099FD70BD01221A700323A5342370F8E75A
:10953000230086331B78002B0DD023007C331A8840
:109540000F4B9B185878FFF7A9F82300A633002883
:10955000E8DD1870E8E7FCF717FDFEF741FD230092
:1095600002227833074908481A7002F0FCFC074BC6
:10957000A034236005232B70D3E7C046A808001051
:10958000D40000104FF7000030090010FD940000D7
:1095900070B51C4C25009C352B78002B0CD0FFF7A8
:1095A000FFFC230085331B78C0B2002B0FD00100D5
:1095B0004820FBF74FFD70BD230086331B78002B3E
:1095C0000ED023007C331A880F4B9B185878FFF776
:1095D00065F82300A63318700223A5342370EAE748
:1095E000FCF7D2FCFEF7FCFC23000222783307498B
:1095F00007481A7002F0B7FC064BA034236005231D
:109600002B70D8E7A8080010D400001053F7000012
:10961000300900109195000070B51C4C25009C3558
:109620002B78002B0CD0FFF7BBFC230085331B7875
:10963000C0B2002B0FD001004420FBF70BFD70BD22
:10964000230086331B78002B0ED023007C331A882E
:109650000F4B9B185878FFF721F82300A63318709A
:109660000123A5342370EAE7FCF78EFCFEF7B8FC73
:10967000230002227833074907481A7002F073FC6E
:10968000064BA034236005232B70D8E7A8080010F0
:10969000D400001057F700003009001019960000A0
:1096A00070B5264C25009C352B78002B1BD0FFF77E
:1096B00077FC230085331B78C0B2002B20D001003B
:1096C0000D20FBF7C7FC70BD2300000120180930F6
:1096D000FF30A83319685A68016042609A68DB68F5
:1096E0008260C36014E0230086331B78002B13D004
:1096F000FCF74AFC23007C331A88114B9B185878DE
:10970000FEF7FCFF6528DFDD2300032287331A7094
:109710000123A4342370D6E7FCF736FCFEF760FC87
:1097200056232B702300074AA0331A600223783493
:1097300005490648237002F016FCC4E7A80800108B
:10974000D4000010A19600005BF700003009001063
:1097500030B5314C85B025009C352B78002B26D0B8
:10976000FFF71EFC230085331B78C5B2002B05D004
:1097700029001120FBF76EFC05B030BD274B196C9A
:109780005A6C009101929A6CDB6C009801990292DC
:109790000393029A039BFBF74FFF2800FEF7AEFFEF
:1097A0001F49FBF7AFFA0123A4342370E4E7230039
:1097B00086331B78002B1CD0FCF7E6FB23007C33A0
:1097C0001A88184B9B185878FEF798FF0500134B22
:1097D000196C5A6C009101929A6CDB6C009801999B
:1097E00002920393029A039BFBF726FF0C49280081
:1097F000D7E7FCF7C9FBFEF7F3FB56232B702300DA
:10980000094AA0331A6002237834084908482370B3
:1098100002F0A9FBB0E7C046A808001070ED0000F8
:1098200050090010D4000010519700005FF70000AD
:109830003009001070B5174C01222300A4331A70B0
:10984000230086331B780500002B0ED07C34FCF7F8
:109850009BFB2288104B9B185878FEF74FFF0400A3
:109860000E492000FBF74EFA10E023009C331B78D2
:10987000002B0DD0FFF794FB85342378C0B2002B6A
:10988000EBD001002800FBF7E5FB054C200070BD84
:10989000034CE5E7A8080010D4000010A009001050
:1098A000FFFFFF7FF7B57920FFF7C4FF05006428AD
:1098B0001FDC104C2D0127002600A837F83632682F
:1098C00073683868796803F04DFCBA68FB680090EB
:1098D0000191B068F16803F045FC009A019B64199E
:1098E000F83432607360B060F16022616361A0613E
:1098F000E161F7BDA8080010F7B57A20FFF79AFFDD
:10990000050064281FDC104C2D0126002700F836C6
:10991000A8373A687B683068716804F0BBFDBA68A4
:10992000FB6800900191B068F16804F0B3FD009A03
:10993000019B6419F83432607360B060F160226199
:109940006361A061E161F7BDA808001070B57B20DC
:109950008AB0FFF76FFF0500642824DC134C2D014B
:1099600023002600A8339968DA68049105921A68E2
:109970005B6802920393F836B268F3680092019331
:1099800064193268736806A8F83402F09DFE0698E0
:109990000799089A099B30607160B260F36020619A
:1099A0006161A261E3610AB070BDC046A808001001
:1099B00070B57C208AB0FFF73DFF0500642824DCE9
:1099C000134C2D0123002600A8339968DA6804910E
:1099D00005921A685B6802920393F836B268F368DE
:1099E0000092019364193268736806A8F83403F092
:1099F000DFF806980799089A099B30607160B26099
:109A0000F36020616161A261E3610AB070BDC0468C
:109A1000A808001073B57D20FFF70CFF642819DC3F
:109A20000D4C25002600A835F836B268F368A86802
:109A3000E96803F097FB3268736800900191286829
:109A4000696803F08FFB009A019BB034286069605D
:109A50002260636073BDC046A808001073B57E2005
:109A6000FFF7E8FE642819DC0D4C25002600A83518
:109A7000F836B268F368A868E96804F00BFD32684C
:109A80007368009001912868696804F003FD009AEA
:109A9000019BB034286069602260636073BDC0467A
:109AA000A808001030B57F208BB0FFF7C3FE6428F4
:109AB0001EDC104C06A823002500F8339968DA68EC
:109AC000049105921A685B6802920393A835AA680C
:109AD000EB68009201932A686B6802F0F5FD069A24
:109AE000079BB0342A606B60089A099B2260636010
:109AF0000BB030BDA808001030B580208BB0FFF748
:109B000099FE64281EDC104C06A823002500F833BB
:109B10009968DA68049105921A685B680292039367
:109B2000A835AA68EB68009201932A686B6803F075
:109B30003FF8069A079BB0342A606B60089A099B2D
:109B4000226063600BB030BDA808001070B5114CE6
:109B5000114E2500A0352B68B3420DD1FFF720FA36
:109B6000C0B2FBF7F7FA002803D10423873423702F
:109B700001E07C34208070BDFEF732FA230002221F
:109B80007833064906481A709C3402F0ECF92E60CE
:109B90000923ECE7A80800104D9B000063F70000C4
:109BA0003009001070B5FCF7EFF9244C25009C3506
:109BB0002B78002B0AD085342378002B05D0FFF7B3
:109BC000EFF9C1B20720FBF745FA70BD23008633D9
:109BD0001B78002B19D0230001222500A4331A7012
:109BE0007C352A88164B9B185878FBF7B3FA002867
:109BF00007D12300042287331A700123A434237071
:109C0000E3E72880FBF77AFAF7E7230085331B7830
:109C1000002B0FD0FEF7E4F90C232B702300094A28
:109C2000A0331A600223783407490848237002F0F1
:109C30009AF9CAE7FFF78AFFC7E7C046A8080010ED
:109C4000D4000010A59B00006EF700003009001042
:109C500070B5184C184E2500A0352B68B34213D1AF
:109C6000FFF79EF9061E00D10136FBF779F90500D2
:109C7000B04200DD35002800FBF714FA431E98417E
:109C80007C342D18258070BDFEF7AAF9FBF768F922
:109C900004F07EFFFBF7A0F8230001307833187042
:109CA0000649074802F05FF901239C342E602370B7
:109CB000E9E7C046A8080010519C000077F70000B3
:109CC00030090010F7B5304C220083321378002B96
:109CD00008D00C2B04D10B3B1370FBF77FFEF7BDB4
:109CE0000133F9E7294D70352B7E002B17D06E7E9E
:109CF000A97E744274410C40E97E701C2818AB198F
:109D0000AA7D0C4304D00100180002F05AF9E4E7E0
:109D1000190002F056F92D236C75AB55DDE72300D1
:109D20000122A4331A702300A8331A685E680192D6
:109D30009F68DD68002200230198310002F096FC44
:109D4000002802D180231B06F618002200233800C9
:109D5000290002F08BFC002802D180231B06ED189D
:109D6000002200233800290004F022F9019A330070
:109D700003F0F8F9064B3A00186059602B00B03434
:109D800022606360A9E7C046A80800101800001010
:109D900050090010F0B5504D89B0280002F026F9A6
:109DA0004E4E009028220021300002F0E7F84C4F80
:109DB0004C4CE35D002B0FD0280002F017F920185F
:109DC000873003782B2B39D1280002F00FF9444B50
:109DD0002018E35C87300370230083331B78424FE5
:109DE000002B4AD0414A9B00D3189A6C390002A834
:109DF00002F0B9F823009C331B78DB0603D53C49FD
:109E0000300002F007FB02A9300002F003FB230040
:109E10009C331B78002B55D02200A032354B1268A2
:109E200000259A4208D0344F7037230078331B78CE
:109E3000BA7D9B1AAB423FDC09B0F0BD280002F0AE
:109E4000D5F82018873003782D2BBDD0280002F0DC
:109E5000CDF82018873003782A2BB5D0280002F0DF
:109E6000C5F82018873003782F2BADD0280002F0DA
:109E7000BDF820188830E35DADE71222009BD31AAD
:109E80001D4A019370320092937D019A93420CDD3A
:109E90001A4A1B490F32300002F065F8009B9A7D88
:109EA000019BD21A009B9A18A0E72A0039003000C3
:109EB00002F059F8009A99E71249300002F0AAFA24
:109EC0000135B2E70C4B70339B7D0E2BB4D80D4996
:109ED000300002F09FFAAFE730090010D008001000
:109EE00076070000A8080010C8F60000F0ED00009A
:109EF00035F8000035800000180000100000001048
:109F000083F7000087F70000F0B5CD4E89B0282216
:109F10000021300002F032F8CA4D2822002128002A
:109F200002F02CF8C84C14220021200002F026F880
:109F300014220021C54802F021F8330085331B7834
:109F4000002B05D1330079331B78002B00D1E6E0DC
:109F500033007C331988002904D0013900223000F5
:109F6000FEF7FAFA37007C37012239882800FEF71D
:109F7000F3FA3888FBF7A8F80200692807DCB4492F
:109F8000632801DDB349233A200001F0ECFF9C3641
:109F90003378002B01D0FFF7FDFEA94C2300873357
:109FA0001B78002B44D0012B03D1AB49200001F0DA
:109FB000DAFF230087331B78022B03D1A749200047
:109FC00001F0D1FF230087331B78042B03D1A44970
:109FD000200001F0C8FF230087331B78052B03D135
:109FE000A049200001F0BFFF230087331B78032B1B
:109FF00003D19D49200001F0B6FF230087331B7871
:10A00000062B03D19949200001F0ADFF23008733CF
:10A010001B78072B03D19649200001F0A4FF2300F1
:10A0200087331B78092B03D19249200001F09BFF55
:10A0300023007A331B78002B03D08F49200001F0D6
:10A0400092FF230086331B78002B14D12300A53305
:10A050001B78042B0FD0230084331B7887495BB215
:10A06000012B00D1E7E0013300D0D7E01D22844965
:10A07000764801F078FF230085331B78724D002B62
:10A0800028D12300A5331B78042B23D023007E3353
:10A090001B78002B03D07B49280002F0BBF923007A
:10A0A0007F331B78002B03D07749280002F0B2F9E8
:10A0B000EF23DB00E35C002B03D07449634802F01C
:10A0C000A9F9230080331B78002B03D070492800A6
:10A0D00002F0A0F9FDF76EFE20000021FBF720FE44
:10A0E00008215848FBF71CFE002383211A00280092
:10A0F0008334FBF743FC2378002B00D1E0E00123FD
:10A10000082268216348FBF739FC01230822522109
:10A110006148FBF733FCFBF704F909B0F0BD3300ED
:10A1200086331B78002B0FD033007C331B885B4AAF
:10A13000D35C2A2B08D05A49300001F014FF59494A
:10A14000280001F010FF28E73300A53356481B789C
:10A150000C30042B50D101F049FF16245349241A26
:10A16000300001F000FF374F5149380001F0FBFE8D
:10A17000300001F03BFF3300B8331A683518059200
:10A180009E685A68DB68069207930022002330001D
:10A19000079902F06BFA002832D10799059A069BBD
:10A1A0000294019100962800FEF7A4FD380001F00A
:10A1B0001DFF234B3F18A8331A689D68DE6805927F
:10A1C0005A682800069200230022310002F04EFA5D
:10A1D00000281CD1059A069B029401960095380030
:10A1E000FEF788FD334B70331B7E002B00D0D2E688
:10A1F000134B9C331B78CCE601F0F8FE1224ADE73C
:10A200000094059A069B2800FEF7D0FBCEE7009449
:10A21000059A069B3800FEF7C9FBE3E7230082336B
:10A220001B782549002B06D1230081331B78002B96
:10A2300000D120E72149054802F0ECF81BE7C046B1
:10A24000A8080010D0080010F80800100C09001031
:10A2500094F7000089F70000B3F70000BFF7000093
:10A26000CCF70000D5F70000E2F70000EDF70000A2
:10A27000FFF700000CF8000014F800001AF80000C6
:10A280001CF8000022F8000026F8000029F8000061
:10A290002CF800002FF8000033F80000D400001064
:10A2A0009FF70000A7F7000000000010ADF70000C6
:10A2B000B0F7000018000010A5F7000020F800001B
:10A2C00008228321004824E70C090010F0B5434B15
:10A2D00083B005000191160098423DDC019B002BE4
:10A2E00059D0002840D07C21862301223C4CADB2BD
:10A2F0006552E2542800FAF7D5FE002840D1002E1E
:10A3000044D0384E384F0EE098478623E35C002B4C
:10A3100054D08723E35C002B0ED1FAF777FE002898
:10A320000AD17C23E55A735D9A00002B44D0802B20
:10A3300002D8D359002BE7D1012586230022E2540D
:10A34000FBF722FE8723E35C072B39D0019B002B10
:10A3500007D1F6F73BFA04E0872203210125204BC1
:10A360009954280003B0F0BD012386217C221C4CA7
:10A37000013528006354A352FAF794FE0028BED09A
:10A38000FAF744FE7C23E55A002EBAD1174B184A3F
:10A390005B69A350B5E7FBF7A7FA002D16D086221C
:10A3A00001217C230E4CA154E552124BE35C002B9F
:10A3B00009D07C23E55A9DE7FAF7A0FE0025BCE70B
:10A3C000FAF724FEC2E7FFF79FFDF2E7012386219B
:10A3D0007C22034C6354A352E7E7C046CF0700003A
:10A3E000A8080010D400001014F30000180000109A
:10A3F0007C07000077070000F8B5254C25009C3548
:10A400002B78002B26D0FEF7CBFDC5B22800FEF737
:10A4100059F9230085331F780600002F0AD0002841
:10A4200003D005238734237003E029002B20FAF79B
:10A4300011FEF8BD00280AD0FDF7D2FD0123A43497
:10A440003A00390030002370FFF740FFF1E787340E
:10A450000423E8E7230086331B78002BE9D1FBF7C0
:10A4600093FDFDF7BDFD08232B702300094AA0339F
:10A470001A602300022278331A7085342378064844
:10A480000649002B00D1064901F06DFDD1E7C04619
:10A49000A8080010F9A300003009001037F80000E8
:10A4A00041F8000070B5194D2B009C331B781A073A
:10A4B00009D5174B70331B7E002B03D1FBF7DEFA57
:10A4C000FDF7A6FE70BD002BFCD12B0085331E7856
:10A4D0002330C4B2002E04D021000720FAF7BAFDC1
:10A4E000F0E7FBF751FD2B000122A43320001A7086
:10A4F000FEF7E8F8002804D032003100FFF7E6FE4E
:10A50000E0E7042287352A70DCE7C046A80800107F
:10A510001800001010B54520FFF7C4FF10BD10B59E
:10A520004420FFF7BFFF10BD10B54320FFF7BAFF6F
:10A5300010BD10B54220FFF7B5FF10BD10B541208A
:10A54000FFF7B0FF10BDF8B50B4C0600250010005A
:10A55000002300220F000949E8350E604F608A6031
:10A56000CB601031A942F8D10122A8341100FFF7C5
:10A57000ADFE20686168F8BDA80800105009001001
:10A58000F0B599B016900F204042FAF754FBBA4B41
:10A59000049005911A00A83211685268B8330A92E3
:10A5A0001A685B68089100920293009A029B0898CF
:10A5B0000A9902F05BF800280BD004980599002254
:10A5C000AE4B03F0F5FC089A0A9B02F0CBFD00901D
:10A5D0000291089A0A9B0098029902F0C3FD00229A
:10A5E000A74B03F0E5FC0C900D9102000B000898BE
:10A5F0000A9902F03BF8002807D10C9A0D9B0098AD
:10A60000029902F033F800280BD004980599002233
:10A610009C4B03F0CDFC089A0A9B02F0A3FD0C9022
:10A620000D91169A08980A99FFF78DFF169A1790C0
:10A6300015910C980D99FFF786FF169A14901291B8
:10A6400000980299FFF77FFF8B4D06902B00039136
:10A6500087331C780126002C14D1159B8A4AB340FD
:10A66000F340D34209D5129BB340F340D34204D503
:10A670000B00B340F340D34207D4092201267E4B9E
:10A6800087331A70300019B0F0BD00260027320061
:10A690003B001798159901F0E9FF079000282BD08F
:10A6A0002900089A0A9BA8310A604B602B002900F8
:10A6B000B0331E605F60089A0A9BB8310A604B6035
:10A6C0002B002900C0331E605F60179A159BC831AC
:10A6D0000A604B602B00D0331E605F606B4BD83537
:10A6E000196C5A6C260029606A609A6CDB6C0092C7
:10A6F0000193AA60EB60C5E7002200231498129929
:10A7000001F0B4FF041E2BD029000C9A0D9BA83138
:10A710000A604B602B002900B0331E605F60089A0E
:10A720000A9BB8310A604B602B002900C0331E60C1
:10A730005F60149A129BC8310A604B602B00D033C3
:10A740001E605F60514BD835196C5A6C079EDC6CEB
:10A750009B6C29606A6000930194AB60EC6091E7A8
:10A76000002200230698039901F080FF002818D0EA
:10A770002900009A029BA8310A604B602B00290037
:10A78000B0331E605F600C9A0D9BB8310A604B605D
:10A790002B002900C0331E605F60C831069A039BFE
:10A7A00096E7139007901090089A0A9B0C980D99C1
:10A7B00003F070FE0C9A0D9B0E900F910098029979
:10A7C00003F068FE0A900B910E980F99F7F70EFFB1
:10A7D00004000D000A980B99F7F708FF2200089073
:10A7E0000991049805992B0001F064FF002807D116
:10A7F000089A099B0498059901F05CFF002847D04E
:10A80000109B01331093022B44DD0126079B009D12
:10A81000029C5E40184F2A0039002300A8310A60CC
:10A820004B603B00002400253900B0331C605D60A4
:10A83000009A029BB8310A604B603B003900C0337C
:10A840001C605D60069A039BC8310A604B603B0048
:10A85000D0331C605D603B001398D8331C0004F0BB
:10A8600097F90025206061600024E0373C607D603E
:10A87000002E00D001E705E7A808001000005940AD
:10A880000000E03F000014400000108070ED000068
:10A8900000231093002200232000290001F0E6FE8F
:10A8A0000028B2D1089809990022002301F0DEFEA9
:10A8B0000028AAD1149A129B0698039903F0EAFD86
:10A8C0000A9A0B9B02F06AFF0A9A0B9B04000D0088
:10A8D0000E980F9902F046FC06000F00F7F786FE6F
:10A8E000049A059B01F0D2FE00284DD020002900DB
:10A8F000F7F77CFE320008900991049805993B0017
:10A9000001F0BAFE002801D1049E059F30003900F5
:10A91000F7F76CFE02000B000898099903F048FB5A
:10A9200006000F0006980399F7F760FE984A994BC6
:10A9300003F03EFB02000B003000390001F0A6FEE0
:10A94000002800D061E722002B000698039902F04E
:10A9500025FF0B0002000299009803F09BFD169A58
:10A9600005000C00FFF7EFFD8B4B11900E91873324
:10A970001B78002B00D113E1079B002B00D1B9E11C
:10A98000009D029C002645E7179A159B1498129982
:10A9900003F080FD0E9A0F9B02F000FF02000B00F7
:10A9A0002000290003F076FD32003B0002F0F6FEA5
:10A9B00002000B000E900F910A980B9903F0F8FA21
:10A9C00022002B0002F0CEFB06000F000E980F991C
:10A9D000F7F70CFE089A099B03F0EAFA04000D0051
:10A9E00030003900F7F702FE694A6A4B0A900B9172
:10A9F00003F0DEFA02000B002000290001F046FE01
:10AA00001190002827D0089A099B0498059901F015
:10AA100033FE002803D1049B059C08930994089AEF
:10AA2000099B0A980B9903F0C3FA04000D000698DD
:10AA30000399F7F7DBFD564A564B03F0B9FA0200CB
:10AA40000B002000290001F021FE002800D0DCE6E8
:10AA500032003B0079E732003B003000390003F060
:10AA6000A7FA002204000D000E980F994B4B03F03B
:10AA70009FFA069A039B03F09BFA02000B0020004A
:10AA8000290003F007FD0022002304000D0001F05F
:10AA9000F3FD00282BD0079B002B00D070E7089A0D
:10AAA000099B0498059901F0E7FD002803D1049B58
:10AAB000059C08930994089A099B0A980B9903F03E
:10AAC00077FA04000D0006980399F7F78FFD304AD6
:10AAD000304B03F06DFA02000B002000290001F05A
:10AAE000D5FD0028B4D0009D029C012692E62000EE
:10AAF0002900F6F7FDFC0E900F9102000B003000CC
:10AB0000390002F02FFB0E9A0F9B0890099130003C
:10AB1000390003F0BFFC04000D0008980999F7F70D
:10AB200065FD06000F0020002900F7F75FFD020019
:10AB30000B003000390001F0B3FD002801D108946A
:10AB4000099508980999F7F751FD04000D000E9832
:10AB50000F99F7F74BFD02000B000A980B9902F0D2
:10AB600001FB0B4A0B4B03F023FA02000B00200001
:10AB7000290001F08BFD002800D046E6069A039BD1
:10AB80000698039902F0EEFA089A099BDFE6C046A0
:10AB90009B2BA1869B84063DA80800100000104056
:10ABA0006300594A5B08D34200D4E5E60E9B564A3F
:10ABB0005B005B08D34200D4DEE6009A029B2800CB
:10ABC000210003F067FCF7F711FD089009912800B8
:10ABD0002100F7F70BFD00224C4B06000F0001F09F
:10ABE0005FFD002801D10026484F494A494B3000FB
:10ABF000390003F0DDF9049A059B02F0B3FA089AD4
:10AC0000099B0A900B9101F055FD002877D1002295
:10AC1000002311980E9901F029FD00286FD1002220
:10AC200000230698039901F03BFD002807D000227D
:10AC3000002311980E9901F01FFD00284BD100222E
:10AC400000230698039901F017FD002807D0002281
:10AC5000002311980E9901F023FD00283BD10498A0
:10AC6000059900222C4B03F0A3F9089A099B0600D2
:10AC70000F0001F01FFD002830D0089A099B0A98A8
:10AC80000B9901F0F9FC002828D0109B0133109398
:10AC9000139B013313930C9B08930D9B0A93009B0A
:10ACA00000950C93029B02940D93149B1793129B97
:10ACB0001593069B1493039B1293119B06930E9B73
:10ACC0000393139B642B00D06EE50126079B009530
:10ACD0005E4002949EE501230793C0E7089A099B12
:10ACE0003000390001F0C8FC43425841109B4042FB
:10ACF0000340CCE7119B06930E9B0393F5E6119B53
:10AD000006930E9B03933DE6000010800000F03F89
:10AD10009B2BA1869B84063D00001040F0B53C4B68
:10AD2000A5B01590A6331B78181C0F2B00D90F2047
:10AD3000C0B24042F9F77FFF354C189019912300BB
:10AD4000A8331A685B680092019300980199230068
:10AD5000B8331E685F6832003B0001F0A1FC002898
:10AD60000CD000220023F83426606760A260E36004
:10AD7000009A019B0096019716001F00009A019B04
:10AD80003000390003F086FB32001A901B910098C6
:10AD900001993B0002F0E6F91E4B002203F008F98E
:10ADA0000023002405931493002320902191029303
:10ADB0000394059B0C2B2FD1029C039D144E1498D9
:10ADC000370003F0E5FEC8373300386079600022B1
:10ADD0000021D03319605A60029A039B2000290099
:10ADE00003F058FBF7F702FC3300B83318605960E2
:10ADF000330000210022C03319605A603300002064
:10AE0000A833B0361C605D603160726025B0F0BD63
:10AE1000A80800100000E03F059BC14C584203F019
:10AE2000B7FE0B0080210200C9050020F7F7C0FE25
:10AE3000059B1C901D915A1E9341DAB201331E935B
:10AE4000DB009B181F9301235B421693179400238A
:10AE500000240A930B94069307940492049803F039
:10AE600097FE1C9A1D9B03F0A3F804000D00F7F752
:10AE700059FC0890099120002900F7F7BBFBA94A6B
:10AE80002290239108980999A74B03F091F8C023C9
:10AE900000221B0603F08CF8F5F7F8FF00220023D0
:10AEA00004000D0001F0E2FB002800D0CEE00022FB
:10AEB0009E4B2000290002F055F9089009910200EC
:10AEC0000B002000290002F069FC02000B00129028
:10AED00013911A981B9903F06BF8009A019B0E903E
:10AEE0000F9102F03FF90E9A0F9B0C900D913000DC
:10AEF000390003F0CFFAF3230E900F9112981399B3
:10AF000000229B0501F0C2FB00281FD00C9A0D9B6C
:10AF10000098019901F0CEFB002807D00098019914
:10AF200032003B00F9F722FE0C900D910E9A0F9B18
:10AF30003000390001F0AAFB002807D0009A019BDD
:10AF400030003900F9F712FE0E900F911A981B99F4
:10AF5000744A774B03F02CF8229A239B03F028F8CD
:10AF600022002B0003F024F8089A099B04000D002E
:10AF70001000190003F01CF802000B00200029004B
:10AF800002F00CFC049B04000D00159A002B00D06D
:10AF90008EE020982199FFF7D6FA664A4B005B08AD
:10AFA000D34207D502000B002000290003F000F86F
:10AFB00010901191149B013314935F4B87331B78CE
:10AFC000002B43D1109A119B0698079902F0CAF8FA
:10AFD0000690079110981199F7F708FB02000B00F3
:10AFE00004000D000A980B9902F0BCF81F9B049A0C
:10AFF0000A900B91934200DD7EE01698179922008B
:10B000002B0001F04DFB002800D178E0069807994D
:10B01000F7F7ECFA00220890099118981999474B14
:10B0200002F0C6FF0A9A0B9B0C900D9108980999A3
:10B0300002F098F802000B000C980D9902F0B8FF8E
:10B0400022002B0001F02CFB002858D03A4B87330C
:10B050001B78002B00D0AFE61C9A1D9B0698079921
:10B0600002F0A6FF059B04000D00002B1AD00298E9
:10B0700003990022324B02F09BFF02000B002000DC
:10B08000290002F06FF8029A039B04000D0003F000
:10B0900001FAF7F7ABFA189A199B01F0EDFA0028BC
:10B0A00000D08BE6059B029403950133059380E65F
:10B0B0000C980D99FFF747FA159A0C9008910E9885
:10B0C0000F99FFF740FA089B1A4A5B005B08D342CE
:10B0D000BCD54B005B08D342B8D502000B000C98DE
:10B0E000089902F03FF82B00220002F061FF149B48
:10B0F0001090119102335FE7049B002B07D0129848
:10B10000139900220F4B01F0C1FA00289ED11E9A1C
:10B11000049B944663440493169417959EE6C04698
:10B12000FFFFEF7F182D4454FB21F93F0000F03F53
:10B13000FB21094000001080A80800100000D03F4B
:10B140000000E03F0000A03CF7B5FAF71DFF274CD8
:10B1500025009C352F78002F0AD085342378002BCA
:10B1600005D0FDF71DFFC1B20620F9F773FFF7BD4B
:10B17000260086363378002B1FD025007C352A88A0
:10B180001B4B9B185878FDF79DFA002803D1042328
:10B1900087342370EBE72B883900019323000124C7
:10B1A000A43322001C70FFF791F8002801D03770FB
:10B1B000DDE7019B34702B80D9E7230085331B78B2
:10B1C000002B0FD0FCF70CFF0C232B702300094A37
:10B1D000A0331A600223783407490848237000F02E
:10B1E000C2FEC4E7FEF734FDC1E7C046A808001060
:10B1F000D400001049B100004AF8000030090010E6
:10B2000010B5FAF7C1FE084B1A00863211780029F2
:10B2100004D000231370F9F7F9FE10BD7C331888B1
:10B220000A00FFF753F8F8E7A808001010B5064B1E
:10B2300086331B78002B05D0FEF766FEFA208000CF
:10B24000F5F702F810BDC046A8080010F8B5FAF7E7
:10B250009BFE2D4C26009C363378002B2BD0FDF71F
:10B260009FFEC5B22800FDF72DFA230085331E7816
:10B270000700002E04D029004F20F9F7EBFEF8BD9F
:10B28000FCF7AEFE002F11D02500012386352B7070
:10B29000FEF73AFEFAF728FB3800FFF73FFDF5F717
:10B2A00095FA2E700123A4342370E8E723000422CA
:10B2B00087331A70F6E7250086352B78002B13D0DC
:10B2C00026007C363788114BDB195878FDF7FAF9E0
:10B2D000002806D0FFF722FD012337802B70A4340D
:10B2E000E2E787340423DFE7FCF77AFE09233370B3
:10B2F0002300074AA0331A60022378340549064820
:10B30000237000F030FEBAE7A8080010D400001047
:10B310004DB2000053F8000030090010F7B5FAF7FD
:10B3200033FE364C26009C363578002D2BD0FDF7A9
:10B3300037FEC5B22800FDF7C5F9230085331E7816
:10B340000700002E04D029005020F9F783FEF7BD36
:10B35000FCF746FE002F11D02500012386352B7007
:10B36000FEF7D2FDFAF7C0FA3800FFF709F9F5F752
:10B370002DFA2E70A43401232370E8E72300042261
:10B3800087331A70F6E71E4B1B78002B25D026005A
:10B390007C3632881B4B27009B185878FDF792F9B2
:10B3A0008737002816D033880193FFF7E9F8019B0F
:10B3B000012233802300A4331A703B78092B04D177
:10B3C000F9F724FE3D708634D5E7002BFBD00C4BFB
:10B3D0001D70BCE704233B70B9E7FCF701FE0923AD
:10B3E00033702300084AA0331A60022378340749D7
:10B3F0000748237000F0B7FDA9E7C046A808001071
:10B400002E090010D40000101DB3000062F80000E7
:10B41000300900104F4B10B51A694F4901321A61BB
:10B420004E4A1268D2B2302A66D01AD8182A0ED0E4
:10B4300005D8082A36D0102A44D008234EE0202A06
:10B4400069D0282AF9D1D8689A69904248D2DA6836
:10B45000501CD86001339B18DB7F414ADBB213607C
:10B46000EBE7482A57D009D8382A4DD0402AE4D1F2
:10B47000DA690423012A4BD10B60DEE7502A53D04E
:10B48000582ADAD1364A12689868D2B2441C9C60B5
:10B490001C00383422540222FF325A608023F13AD1
:10B4A000DB0552E00022DA60D868421CDA605A1CE0
:10B4B0001218D27F2A48D2B2026028220A60273AA4
:10B4C0005A6010BD00229A60DA68501CD8600133BF
:10B4D0009B18DB7F224ADBB2136028230B60F0E766
:10B4E0008022D869D205002801D02023B7E70220A6
:10B4F000FF3058601023B2E780221020D205106080
:10B5000008220A60FA32DBE7822252005A6094E78E
:10B510008022D205A3E780221020D20510600822E5
:10B520000A600422FF32CBE70D4A12689868D2B253
:10B53000441C9C601C0038342254DA699868531EFD
:10B540000422834203D98023DB051A6075E70A6071
:10B5500073E7C046180000101800004004000040C7
:10B5600008000040202130B5064A074C0378002B24
:10B5700001D1180030BD013015680D42FCD02360A8
:10B58000F4E7C04614800040008000400E22174BB4
:10B5900010B51B681340062B12D1154B90321B6857
:10B5A000134205D0134ADBB25360134B1B6810BD26
:10B5B000DB07FCD5104B1868C0B2F4F735FEF6E790
:10B5C000042BF7D00C2B05D10A4AF43351680B43F6
:10B5D0005360ECE7022BEAD1054B1A68054B920643
:10B5E00002D500229A60E2E70122FBE708800040D2
:10B5F0001480004028100010008000400122034BFE
:10B600001A60034AD3680133D36070470080014059
:10B61000980000100122034B1A60034A136901339A
:10B620001361704700400140980000100122034B55
:10B630001A60034A536901335361704700000140A7
:10B64000980000100122034B1A60034A93690133EA
:10B650009361704700C0004098000010074A084BF3
:10B660005169013102D1D9690131D9615169013181
:10B6700051611A6A01321A627047C0461800001000
:10B68000980000101B4B10B59A6D002A2AD0DA6D75
:10B690000132DA65184B9868FAF7FEFB8022174BE7
:10B6A0000121DA679218DA678022D200DA678022F5
:10B6B0005201DA6780221201DA6780229200DA678B
:10B6C00000230F4A494213600E4A11600E4A13606C
:10B6D0000E4A136001220E4B1A60F4F7F1FCC046CB
:10B6E000C04610BD08220B4B87331A70F5F76EF871
:10B6F000F7E7C046180000100000001004E100E069
:10B70000048204400882044004C000403CC0004061
:10B7100000C00040A8080010F7B5F4F7ABFDC04A20
:10B72000012413681B0B1B031360BE4A13681B0B19
:10B730001B031360BC4A13681B0B1B031360BB4A3B
:10B7400013681B0B1B0313600022B94B1A60B94B23
:10B750001C601A601C601A682242FCD02322B64B7F
:10B7600001201A60FAF798FBF4F784FD40213F208E
:10B77000B24B1A688A431A60B14A1060B14A146029
:10B780001A688A431A60FCF71FFBFCF713FBFAF7F1
:10B790005DFBF4F7F7FF0021AB48F4F779FD0021DA
:10B7A000AA48F4F775FDF4F773FEF4F741FEA84CD0
:10B7B000092248340021200000F0E0FB0020E07165
:10B7C000F5F734F8A34D002822D0F4F7F5FD0C234B
:10B7D000184002D02378184320709D4C48342378B9
:10B7E0005B0711D5F4F7B2FDA378002B03D0237AC1
:10B7F000012B02D80133237201E02B6A6B62002314
:10B80000934A2B624832D3700022914B48331A700E
:10B810008F4B4833DB79002B01D1F4F797FDFA23E6
:10B8200000269B002E626B62FAF796FAF0228A4C91
:10B83000D2003100200000F0A1FB23000222A4333B
:10B84000FF321A802300FD3AA6331A7023000B3210
:10B8500078331A70814A82490C32824800F083FBA7
:10B86000FAF76EFBFAF7BAF8FEF74EFBF9F770FF3E
:10B87000061E00D143E1EF22D200A35C002B04D0CE
:10B880000023A35422007C32138000222300AA61EB
:10B8900087331F78974216D01A70FAF79FF8AA6973
:10B8A000714B9A4203D9FCF7F1FA0023AB61FEF722
:10B8B0002BFBEF23DB00E35C002BD7D103210A2015
:10B8C000F4F730FED2E7A02E66DDA021300000F0B4
:10B8D000AFFE0D2927D1FCF783FBFA27634800F060
:10B8E00037FB0126FF00624B6248995D013600F08C
:10B8F0002FFBBE42F7D1CC270026FF0033000933CF
:10B90000FF33E15C5B48013600F022FBBE42F5D11B
:10B91000594800F01DFB594E300000F019FB300073
:10B9200000F016FBB9E7112914D1FCF759FBFA22F4
:10B930003900D2004E4800F021FB2300EF227C3377
:10B940001F800123D2004E48AF62A35400F000FBD9
:10B950004A48E5E7072907D1230086331B78002BE7
:10B960009BD1FEF7F3F898E7062907D12300863329
:10B970001B78002B91D1FEF76BF98EE732298CD121
:10B98000FA223900D2003A4800F0F8FA23007C335A
:10B990001F80FCF725FB80E723009C331B78002BDE
:10B9A00074D033003D3B012B21D92821300000F019
:10B9B0003FFE12291BD004230A009A43012A16D005
:10B9C0003200153A132A03D82E4BD340DB070ED48E
:10B9D00033000422143B934304D1230083331B78A8
:10B9E000002B04D133000422373B93430FD1F0B234
:10B9F000F9F77AFA1648703000F0F8FA2300783335
:10BA00001B78984200D048E7FCF702FC45E7142970
:10BA1000F0D81D4BCB40DB07ECD52831C8B2E7E7A7
:10BA200000800050008001500080025000800350D0
:10BA30004080044044800440088004403882044030
:10BA400024800440D8800440984004409C40044036
:10BA50001800001098000010A80800100000001046
:10BA6000C8F60000300900105702000077F8000007
:10BA7000D40000106DF8000000FA00007EF800000D
:10BA800071F80000F3EE0F001091190023008533C8
:10BA90001B78F6B23000002B29D0F9F735FA0028D0
:10BAA00024D1202332009A43122A1FD033000222CD
:10BAB0009343012B1AD03300523B012B16D9612E30
:10BAC00014D02633DBB2102B03D84E4ADA40D3070A
:10BAD0000CD42821300000F053FBFB230539194218
:10BAE00004D033007F33DBB21E2B03D83000F9F7CC
:10BAF000FBF9D2E600213000F9F7ACFACDE6EF23EE
:10BB0000DB00E35C002B00D1C9E63F4A917B537B0D
:10BB1000994200D1AAE6937BD318DE7B937B013355
:10BB2000DBB293735BB2002B01DA002393730D2E0B
:10BB300003D00A2E01D0202E28D12F002C37380018
:10BB4000FAF73CF80A2201900021380000F016FABA
:10BB50002E4B5F612E4BE35C002B03D131002D484F
:10BB600000F0F6F9019BFF2B00D97FE622007C3222
:10BB7000138829498B4238D9AB6A28498B423BD874
:10BB8000274A0199D1540133AB626FE6082E01D0E8
:10BB90007F2E18D11E4BE35C002B14D12B001B4FC2
:10BBA0002C337A699A420ED908211A4800F0D0F94C
:10BBB0002021184800F0CCF90821164800F0C8F9F7
:10BBC0007B69013B7B613300303B092B9DD8104BD7
:10BBD000E35C002B03D131000E4800F0B9F90B4AA9
:10BBE0005369591C51611E708FE701339BB213805A
:10BBF00001990C4AD15439E600231380EF22D20078
:10BC0000A35433E611310100281000100000001089
:10BC10007707000091F70000CE0700005F060000E4
:10BC2000B0090010D400001070B500241E5D051985
:10BC3000002E08D1121B1300002B07DCD043C017C5
:10BC40001040001970BD06550134EFE72970013B23
:10BC50000135F1E7F8B505000C001E00571E092B51
:10BC600016D90A21180000F005FA210003003A0055
:10BC70002800FFF7EFFF04002D1830000A2100F024
:10BC80007FFA30312970601CF8BD2C70013F0135FE
:10BC9000002FFADC141E00DC0124013CEDE7F0B5B6
:10BCA00085B00B9E040003910A9F551E002E01D102
:10BCB000092F1DD90A2200233800310000F066FA4E
:10BCC0002A000090019120000399FFF7E8FF05008A
:10BCD0002418380031000A22002300F057FA681CAB
:10BCE0003032227005B0F0BD039B013D237001345A
:10BCF000002DF9DC151E00DC0125013DE9E7F7B553
:10BD00000F00D9171E005B184B4004000193551E0D
:10BD1000092B16D918000A2100F0ACF90300002EF7
:10BD200000DA43422A0020003900FFF7E8FF05004F
:10BD3000241801980A2100F023FA3031681C217080
:10BD4000FEBD002E00DA951E23006119CA1A002AD2
:10BD50000BDCE843C017054064196B1C002EE8DAC1
:10BD60002D221D0022700134E3E71F700133EDE73F
:10BD700073B5069E04001D0010003309013A002B24
:10BD800011D0009320002B00FFF7F2FF24180F239F
:10BD90001E40F3B2092E0DD830330130237076BD2A
:10BDA0002170013A0134002AFADC002800DC01206D
:10BDB0000138ECE7002D01D03733EEE75733ECE7DD
:10BDC000F0B585B0040003911D00002801D00023C8
:10BDD0000370002630001378002B00D092E0039A05
:10BDE000B24200D99AE00023013C2370013E96E064
:10BDF0005178252902D1217002328CE0302924D0DB
:10BE0000531C029320239C46029B1B782D3B5A42D5
:10BE10005341029AD31800220293029B1B781F0001
:10BE2000303F092F15D9039997198F4201D98A1BE1
:10BE3000D2B2692B46D015D8632B5ED0642B41D08B
:10BE4000582B4ED00126764269E0931C02938C4613
:10BE5000DAE70A214A439A18029B303A0133D2B2F8
:10BE60000293DAE7732B41D01FD86C2BEAD1029BE7
:10BE70005B786C2B14D1029B9B78752B10D1029BA5
:10BE800007350233072102932B008B431D001868EE
:10BE9000596800900191614620000835FFF7FFFEC8
:10BEA000029A24180132361895E7752B12D0782B98
:10BEB000C8D12B682F1D0093002361462000FFF797
:10BEC00057FF05E02B68614620002F1DFFF717FF85
:10BED0003D00E5E72B68614620002F1DFFF7BAFE05
:10BEE000F6E72B682F1D00930123E6E72B686146D8
:10BEF00020002F1DFFF798FEEAE72B680120237032
:10BF00000435CDE70399B14200D86CE7252B00D169
:10BF10006EE701322370013601345CE72370300094
:10BF200005B0F0BD10B513000A006421FFF748FF0B
:10BF300010BD00B59BB00A00010001A8FFF7F2FF99
:10BF4000632800DDFEE701A8FFF70CFB1BB000BD76
:10BF50000FB407B504A901C90191FFF7EAFF03B0C7
:10BF600008BC04B018470EB403B503AA02CA019274
:10BF7000FFF7D8FF02B008BC03B01847F0B50500C2
:10BF8000830704D003009A189A4217D1F0BD03002A
:10BF9000032AF8D9131F0F049B080C063C439E008C
:10BFA00036180C430F0204363C4310C5B542FCD191
:10BFB000032401339B00C3182240E4E719700133C6
:10BFC000E2E710B5814208D20139431E002A00D1B0
:10BFD00010BD8C5C9C54013AF8E700238142F7D9EC
:10BFE0009A42F5D0CC5CC4540133F9E70200030057
:10BFF000981A0133591E09780029F9D170470300B6
:10C000000A781A70002A00D1704701310133F7E72E
:10C01000002210B5835C8C5CA34201D0181B10BDBC
:10C020000132002BF6D11800F9E7FEE7FEE7000029
:10C03000002370B50A480B490B4C1A188A4207D3E3
:10C0400000210A4B0A4A934206D3FFF765FBFEE73D
:10C05000E55C01331570F0E719700133F3E7C04672
:10C060000000001018000010CCFA000018000010AA
:10C07000C0110010002243088B4274D303098B4285
:10C080005FD3030A8B4244D3030B8B4228D3030CA8
:10C090008B420DD3FF22090212BA030C8B4202D34A
:10C0A0001212090265D0030B8B4219D300E0090A72
:10C0B000C30B8B4201D3CB03C01A5241830B8B427B
:10C0C00001D38B03C01A5241430B8B4201D34B0364
:10C0D000C01A5241030B8B4201D30B03C01A5241C9
:10C0E000C30A8B4201D3CB02C01A5241830A8B424E
:10C0F00001D38B02C01A5241430A8B4201D34B0237
:10C10000C01A5241030A8B4201D30B02C01A52419A
:10C11000CDD2C3098B4201D3CB01C01A524183094E
:10C120008B4201D38B01C01A524143098B4201D388
:10C130004B01C01A524103098B4201D30B01C01AB3
:10C140005241C3088B4201D3CB00C01A524183082D
:10C150008B4201D38B00C01A524143088B4201D35A
:10C160004B00C01A5241411A00D2014652411046BA
:10C170007047FFE701B5002000F006F802BDC04699
:10C180000029F7D076E770477047C046002B11D1E1
:10C19000002A0FD1002900D1002802D00021C94374
:10C1A000081C07B4024802A14018029003BDC04613
:10C1B000D9FFFFFF03B4684601B5029800F006F806
:10C1C000019B9E4602B00CBC7047C046F0B54F467E
:10C1D0004646D646C0B5040082B00D00914698464A
:10C1E0008B422FD82CD04146484600F0B1F82900A8
:10C1F0000600200000F0ACF8331A9C46203B9A461B
:10C2000000D576E04B46524693401F004B466246AF
:10C2100093401E00AF4228D825D05346A41BBD41F1
:10C22000002B00DA7BE0002200230092019301231F
:10C23000524693400193012362469340009318E0D5
:10C240008242D0D900220023009201930A9B002B46
:10C2500001D01C605D600098019902B01CBC904642
:10C260009946A246F0BDA342D7D9002200230092EE
:10C2700001936346002BE9D0FB07984641467208BC
:10C280000A437B0866460EE0AB4201D1A2420CD8BD
:10C29000A41A9D41012024196D410021013E24185A
:10C2A0004D41002E06D0AB42EED9013E24196D411E
:10C2B000002EF8D100980199534600196941002BCE
:10C2C00023DB2B005246D3402A006446E2401C0088
:10C2D00053461500002B2DDB26005746BE40330089
:10C2E00026006746BE403200801A994100900191B5
:10C2F000ACE7624620239B1A4A46DA4061461300A7
:10C3000042468A4017001F4380E7624620239B1A5B
:10C310002A0066469A402300F3401343D4E762465E
:10C32000202300219B1A0022009101920122DA4071
:10C33000019280E72023624626009B1ADE402F00F0
:10C34000B0466646B74046463B003343C8E7C04662
:10C3500010B5002903D100F007F8203002E0081CD6
:10C3600000F002F810BDC0461C2101231B049842B6
:10C3700001D3000C10391B0A984201D3000A083976
:10C380001B09984201D30009043902A2105C40182D
:10C390007047C046040302020101010100000000D1
:10C3A00000000000C317C0185840704770B50568FA
:10C3B0000400002D22D01349280000F053F8C201D8
:10C3C000121A9200131ADA00D21A92001218D3002D
:10C3D000D2180D4BAA1A5A4303051B1A9B001B18AF
:10C3E0009B001B181B011B1A9B00181A8000801849
:10C3F00005D5064BC3185800400801E00448030067
:10C40000236070BD1DF30100A7410000FFFFFF7F07
:10C4100067B7E12A70B50400830717D102680F4B94
:10C42000D31893430E4A150013420FD1043002680B
:10C430000A4BD31893432B4208D104300268074BB0
:10C44000D31893432B42F1D000E001300378002B46
:10C45000FBD1FFF7D4FD200070BDC046FFFEFEFEFD
:10C460008080808003460B437FD4002243088B42A8
:10C4700074D303098B425FD3030A8B4244D3030B6B
:10C480008B4228D3030C8B420DD3FF22090212BA30
:10C49000030C8B4202D31212090265D0030B8B42AC
:10C4A00019D300E0090AC30B8B4201D3CB03C01A96
:10C4B0005241830B8B4201D38B03C01A5241430B71
:10C4C0008B4201D34B03C01A5241030B8B4201D361
:10C4D0000B03C01A5241C30A8B4201D3CB02C01ACC
:10C4E0005241830A8B4201D38B02C01A5241430A44
:10C4F0008B4201D34B02C01A5241030A8B4201D333
:10C500000B02C01A5241CDD2C3098B4201D3CB01D9
:10C51000C01A524183098B4201D38B01C01A524188
:10C5200043098B4201D34B01C01A524103098B428C
:10C5300001D30B01C01A5241C3088B4201D3CB0077
:10C54000C01A524183088B4201D38B00C01A52415A
:10C5500043088B4201D34B00C01A5241411A00D20A
:10C5600001465241104670475DE0CA0F00D0494273
:10C57000031000D34042534000229C4603098B42E3
:10C580002DD3030A8B4212D3FC22890112BA030A6B
:10C590008B420CD3890192118B4208D389019211ED
:10C5A0008B4204D389013AD0921100E08909C30972
:10C5B0008B4201D3CB01C01A524183098B4201D374
:10C5C0008B01C01A524143098B4201D34B01C01A5F
:10C5D000524103098B4201D30B01C01A5241C308D7
:10C5E0008B4201D3CB00C01A524183088B4201D346
:10C5F0008B00C01A5241D9D243088B4201D34B0061
:10C60000C01A5241411A00D20146634652415B10A2
:10C61000104601D34042002B00D549427047634683
:10C620005B1000D3404201B50020FFF7ADFD02BD15
:10C630000029F8D016E7704702B47146490849004E
:10C64000095C49008E4402BC7047C0468446101CF9
:10C6500062468C46191C634600E0C0461FB501F0D7
:10C660003FFC002801D40021C8421FBD10B501F0D5
:10C6700097FB4042013010BD10B501F031FC00289D
:10C6800001DB002010BD012010BDC04610B501F037
:10C6900027FC002801DD002010BD012010BDC04690
:10C6A00010B501F0B9FB002801DC002010BD01200D
:10C6B00010BDC04610B501F0AFFB002801DA002024
:10C6C00010BD012010BDC046F0B5DE4657464E46AF
:10C6D00045469446E0B595B09B461E9B65469946F7
:10C6E0001F9B04009846209B60460293219B029A60
:10C6F0009A46594653460A9501F05AFC239F229EBA
:10C700000490059132003B004846414603960B9742
:10C7100001F04EFC3D0006000F00039A2B000A9822
:10C7200059460C960D9701F043FC4A460690079136
:10C7300043460298514601F03BFC32003B00089012
:10C7400009910498059901F0A5FE089A099B060035
:10C750000F000698079900F005FD32000090019146
:10C760003B0030003900FFF781FF00280DD0009A10
:10C77000019B200026606760A260E36015B03CBCAE
:10C7800090469946A246AB46F0BD0098019902003A
:10C790000B00FFF76BFF0028E9D10A995B468C4636
:10C7A0000A0060465946654601F074FE4A461090FC
:10C7B000119143464846414601F06CFE0B000200D1
:10C7C000FFF754FF3822434258416B469B181870BC
:10C7D0004A46434641464846FFF748FF3822431E33
:10C7E00098416B469B181B782A0003400E93280043
:10C7F0005B465946FFF73AFF002800D123E1109825
:10C80000119902000B00FFF731FF002800D01AE158
:10C8100059460022D34B002900DAD34B9B460E9B8E
:10C820000A925A425341D14A5B421340CD4A944640
:10C830006344424600215B00D20FD2075B081343DA
:10C8400089469846029A534602985146FFF70EFFD2
:10C85000002800D168E10B99039D8C460B002A004B
:10C8600028006146FFF702FF002800D150E10123B4
:10C870000E93029A53460298514601F00BFE129015
:10C8800013910B99039D8C462A000B0028006146EA
:10C89000654601F0FFFD0B000200FFF7E7FE4022B6
:10C8A000434258416B469B181870039A2B0029008D
:10C8B0000398FFF7DBFE4022431E98416B469B180E
:10C8C0001B78029A03401093029853465146FFF793
:10C8D000CDFE002868D01298139902000B00FFF7D4
:10C8E000C5FE002860D1524600259E4B002A00DA82
:10C8F0009D4B9A46109B9D4A013B1340994A0295D5
:10C90000944663440B9A5B00D70F00220A9E5B0893
:10C91000FF073B4303920B9332005B4630005946BE
:10C92000FFF7A4FE002800D138E14A4643464846B6
:10C930004146FFF79BFE002800D125E1029A5346AD
:10C940000A98594601F034FB0B9D06000F00039A2C
:10C950002B004846414601F02BFB02000B00300043
:10C96000390001F097FD0022814B01F021FB039A71
:10C970002B0006000F000A98594601F019FB029A95
:10C980000090019153464846414601F011FB0200D8
:10C990000B000098019900F0E5FB0022744B01F0B8
:10C9A00007FB00900191E2E6109B002B00D0A4E071
:10C9B0000E9B002BC2D10498059902000B0001F0D8
:10C9C00069FD0E900F910498059902000B00FFF786
:10C9D0004DFE002846D00E980F9902000B00FFF77D
:10C9E00045FE00283ED10A9E5B4632003000594683
:10C9F000FFF73CFE002800D1A0E04A4643464846E7
:10CA00004146FFF733FE002800D1B3E0029A5346B7
:10CA100002985146FFF72AFE002800D198E0039FB4
:10CA20000B9E3A00330038003100FFF71FFE00284C
:10CA300084D100220B991300914201DA80231B0656
:10CA400003920B937AE70E9B002B00D111E7002293
:10CA500059461300914201DA80231B069B460A9235
:10CA6000404BE6E60C980D9902000B0001F012FD18
:10CA7000049005910C980D9902000B00FFF7F6FD4C
:10CA8000002807D00498059902000B00FFF7EEFD7F
:10CA90000028A8D00698079902000B0001F0FAFCC4
:10CAA000049005910698079902000B00FFF7DEFD40
:10CAB000002807D00498059902000B00FFF7D6FD67
:10CAC000002890D00898099902000B0001F0E2FCC0
:10CAD000049005910898099902000B00FFF7C6FD24
:10CAE000002800D143E60498059902000B00FFF7E7
:10CAF000BDFD002800D03AE675E7002552462B0020
:10CB0000AA4201DA80231B069A460295154BF9E6E4
:10CB100000220B991300914201DA80231B060B932C
:10CB2000012303920E93A4E652464D464B464A45D6
:10CB300001DA80231B0602959A468CE600265A46A7
:10CB40003300B24201DA80231B060A969B4654E763
:10CB5000002552462B00AA4201DA80231B060295CB
:10CB60009A465CE70000F03F0000F0BF000010C0F4
:10CB70000000F07F002241461300914201DA802339
:10CB80001B069146984641E7002241461300914218
:10CB900001DA80231B0691469846CFE600265A46C6
:10CBA0003300B24201DA80231B060A969B46BCE69C
:10CBB000F0B557464E464546DE46E0B58BB0169971
:10CBC000824689461799189888461999149E8B466B
:10CBD00041464C005946159F4900019203930500B8
:10CBE000059002004B084846610802960497FFF73B
:10CBF00043FD00284BD02A005B4648464146059538
:10CC000000F0CCFD04000D0002000B004846414638
:10CC100001F0CEF9059A5B4600F0A4FA22000690D6
:10CC200007912B000198039901F0C2F932003B00F3
:10CC30000296049700F096FA069A079B00F0AEFD64
:10CC400022002B0006000F000298049901F0B0F9B1
:10CC5000019A039B01F01EFC069A079B00F09EFDC3
:10CC6000320004000D003B0030003900FFF7FEFCED
:10CC700000283ED0534650461E605F609C60DD60D9
:10CC80000BB03CBC90469946A246AB46F0BD059E13
:10CC90004A4643463000594600F080FD04000D002E
:10CCA00002000B003000594601F082F94A46434623
:10CCB00000F058FA06000F00029A049B2000290099
:10CCC00001F076F9019A039B00F04CFA32003B0028
:10CCD0000696079700F062FD019A039B06000F007D
:10CCE0002000290001F064F902000B000298049969
:10CCF000B0E722002B0020002900FFF7B7FC002836
:10CD0000B8D10022002348464146FFF7AFFC002877
:10CD100028D00022002305985946FFF7A7FC0028D9
:10CD200020D00399019A0B000198FFF79FFC00287F
:10CD300000D176E143460024DE4D002B01DA0024C9
:10CD4000DD4D019A039B2000290001F031F9029A80
:10CD500006000F0020002900049B01F029F90400BF
:10CD60000D0087E7019803990690079102000B00D8
:10CD70000698079901F08EFB089009910399019A92
:10CD80000B000198FFF772FC00287ED008980999E3
:10CD900002000B00FFF76AFC002876D14A464346A2
:10CDA0004846414601F076FB02000B00FFF75EFCAF
:10CDB000002800D146E105995B460A000800594663
:10CDC00001F068FB02000B00FFF750FC002800D1C7
:10CDD00095E0BA4B039A029FD20F049ED2071343E9
:10CDE00001933A0033003800310001F053FB3A0060
:10CDF00004000D00330038003100FFF737FC002835
:10CE000000D153E122002B0020002900FFF72EFC67
:10CE1000002800D04AE1A94C049B0022DB0FDB076D
:10CE20001C434846019B414601F0C2F8230006001E
:10CE30000F0000220598594601F0BAF802000B00D5
:10CE40003000390000F08EF900229A4B01F0B0F862
:10CE50002300002206000F004846414601F0A8F8D2
:10CE6000002204000D00019B0598594601F0A0F82E
:10CE700002000B002000290001F00CFB00228D4B6A
:10CE800001F096F804000D00F4E60298049906906B
:10CE9000079102000B000698079901F0FBFA069033
:10CEA00007910499029A0B000298FFF7DFFB002814
:10CEB00000D1C7E00698079902000B00FFF7D6FBE8
:10CEC000002800D0BEE04A4643464846414601F0AD
:10CED000E1FA02000B00FFF7C9FB002800D1B1E026
:10CEE00005995B460A000800594601F0D3FA0B0089
:10CEF0000200FFF7BBFB0023984200D06AE70599C8
:10CF00005B4689460A000800594601F0C3FA4A46C2
:10CF1000069007915B4648465946FFF7A7FB002855
:10CF200000D1A7E60698079902000B00FFF79EFBC9
:10CF3000002800D09EE60898099902000B00FFF730
:10CF400095FB002800D195E6029989460A000499CC
:10CF500048460B0001F09EFA0B000200FFF786FB2B
:10CF60000023984200D185E64246D70F059EFF0771
:10CF70003B433200994630005B46594601F08AFA3D
:10CF8000320004000D005B4630005946FFF76EFB8F
:10CF9000002800D18CE022002B0020002900FFF7A0
:10CFA00065FB002800D083E0444E5B46DB0FDB07C7
:10CFB0001E4300224B460198039900F0F9FFB0464A
:10CFC0003300049E04000D0000223100029800F09E
:10CFD000EFFF02000B002000290000F0C3F8002240
:10CFE000002300F0E5FFB34600224B4606000F0089
:10CFF0000298594600F0DCFF002204000D00434671
:10D000000198039900F0D4FF02000B0020002900D2
:10D0100001F040FA0022002300F0CAFF04000D00D6
:10D0200028E60499029A0B000298FFF71FFB0028DC
:10D0300000D07FE60399019A0B00019801F02AFACB
:10D04000089009914A4643464846414601F022FA73
:10D050004A4606900791434648464146FFF706FB7D
:10D06000002800D14BE70698079902000B00FFF754
:10D07000FDFA002800D042E70898099902000B0049
:10D08000FFF7F4FA002800D1F4E5029989460A0076
:10D09000049948460B0001F0FDF902000B00FFF770
:10D0A000E5FA002800D1E5E5044B5DE70024B3E68E
:10D0B00000267AE70000F07F0000F0FF0000F03F5C
:10D0C00070B500220C4B04000D00FFF7F3FA0028A6
:10D0D00004D12000290001F025FD70BD064B00227F
:10D0E0002000290001F0D6F901F01CFD80231B0669
:10D0F0009C466044F1E7C0460000E04170B5002264
:10D100000B4B0D00040000F053FFFFF7D9FF0600A2
:10D1100001F078FD0022074B00F04AFF02000B00EF
:10D120002000290001F0B6F9FFF7CAFF310070BDF9
:10D130000000F03D0000F04170B50600080001F06D
:10D1400061FD0022064B00F033FF0D0004003000AB
:10D1500001F058FD2B00220000F004F870BDC0461D
:10D160000000F041F0B54F464646D6460C00090394
:10D17000C0B5490A470F5E0039431F03DB0F9C46C9
:10D1800065007B0A570F1F436D0DE40F760DA14616
:10D19000C000B846D200AB1B64457BD0002B5FDDDE
:10D1A000002E00D0A4E03E00164300D112E15E1E26
:10D1B000002E00D09EE1871A4346B84280410125E7
:10D1C000C91A4042091A0B0200D431E149024E0A41
:10D1D000002E00D16EE13000FFF7C6F80300083BD7
:10D1E0001F2B00DD61E120223900D21A9E40D14080
:10D1F0009F400E439D4200DD51E15D1B6B1C1F2BC8
:10D2000000DD7CE12021C91A3D0030008F408840BC
:10D21000DD40791E8F41310007222843D940002587
:10D2200007433A40002A09D00F233B40042B05D086
:10D230003B1DBB42BF417F42C9191F000B0200D4F6
:10D2400026E26A1CC64B55056D0D9A4200D106E1D7
:10D25000C44AFF080A40530752023B43120B8EE0B8
:10D26000002B00D0B8E06B1C5B055B0D012B00DCD4
:10D2700030E1871A4346B842B641CB1A76429E1B2C
:10D28000330200D54CE13B003343A1D100220024FE
:10D29000002570E0002B00DCE5E0002E00D183E0EB
:10D2A000AF4EB54260D0802636043743B846382B9F
:10D2B00000DC3EE1434613431F007A1E97413F18AE
:10D2C00087428041404209180B0200D4B0E0A44BD1
:10D2D00001359D4200D1C3E0A24A7B080A400121EA
:10D2E0000F401F435108D30707221F433A4099E7D5
:10D2F0009B4EB54238D0802636043743B846382B8B
:10D3000000DDDCE01F2B00DC30E11E004746203E44
:10D31000F740BC46202B04D04026F31A46469E40D8
:10D320003243170063467A1E97411F43CCE0002B1F
:10D3300000D104E24346134300D159E14B07C00832
:10D3400018438023C9081B03194208D04546ED083D
:10D350001D4204D14346D008590708432900420F13
:10D36000C9007F4D1143C0004B07CA087C49C00863
:10D3700003438D4268D012036D05120B6D0D002121
:10D3800012031800130B0A0D12051A43764B2D05D4
:10D3900013402B435B00E4075B08234319001CBCCC
:10D3A00090469946A246F0BD3E00164312D05E1E3E
:10D3B000002E00D000E1871887428041414440425E
:10D3C000091801250B0233D5022585E76446330091
:10D3D000414610001D00C7E7002D00D0DAE00C0028
:10D3E0000443F3D05C1C00D19FE15D4CA64200D108
:10D3F0002FE1DB43382B00DD66E11F2B00DD83E1ED
:10D4000020240500E41A0F00DD40D940A040434627
:10D41000A7405B1A441EA04198462F433843171A71
:10D42000BA42924143465242991A64463500CAE6CE
:10D4300007223A40002A00D0F6E64B07CA084849BE
:10D44000FF083B438D4296D11900114300D19EE164
:10D45000802109030A431203120B414D8FE7150087
:10D46000002200238BE7002B00D0C7E06B1C5F0578
:10D470007F0D012F00DCF1E0394DAB4200D1B9E066
:10D4800085180A00854289414244494251180722C1
:10D49000CF076D082F4349083A401D00C2E6072216
:10D4A0003049ED1A31403A40BCE63E00283886400B
:10D4B00000279FE63800FEF757FF20308EE64346F0
:10D4C00013431F007A1E9741C71BB8428041404258
:10D4D000091A78E60E003B0006431343002D61D184
:10D4E000002E00D0F4E0002B00D11BE1644639008F
:10D4F000100039E71A4FBB427AD03300FFE6300004
:10D500001F3DE840202B03D04021CB1A9E403743DB
:10D510007B1E9F41072207433A400021002589E7EF
:10D52000171A4346BA42B641591A76428E1B6446D0
:10D530004EE61F2B00DDADE020264746F61AB74029
:10D54000B9461700B246DF404E463E4337005646C6
:10D55000B240561EB24117434246DA408918AEE641
:10D56000FF070000FFFF7FFFFFFF0F8020264746D9
:10D57000F61AB740B9461700B246DF404E463E4362
:10D5800037005646B240561EB24117434246DA4073
:10D59000891A99E77F4CA6425BD0802424045B4221
:10D5A000214327E7002E0CD1002B00D1CBE06446AD
:10D5B00039001000774DD7E6764FBB4218D03300C4
:10D5C00075E6002B14D04B07C00818438023C90808
:10D5D0001B03194207D0FC081C4204D17907D0086C
:10D5E0000843E14621004C46420FC9001143C000E8
:10D5F000684DB9E61D0000220023C0E6002D5BD176
:10D600000D00054300D1E2E65D1C00D1B0E0614DA4
:10D61000AE421FD0DB43382B71DC1F2B00DD96E0C0
:10D6200020250F00ED1AAF40B9460700AA46DF409B
:10D630004D463D432F005546A840D940451EA841C0
:10D6400088440743BF1897429241514241443500F4
:10D650003AE6644635004146100085E60B00034378
:10D66000002D00D063E6002BF5D04346134300D1D4
:10D670007AE68718874280410722414440420918D0
:10D680003A400B0200D4D5E6434B01351940C9E5B9
:10D69000380069E61E004746203EF740BC46202B76
:10D6A00004D04026F31A46469E4032431700634694
:10D6B0007A1E97411F4302E6364DAE42CAD08025FE
:10D6C0002D045B422943A6E70843411E8841A6E694
:10D6D000002B00D148E6871A4346B842B641CB1A20
:10D6E00076429E1B33024BD5171A4346BA429241EB
:10D6F000591A5242891A072264463A4092E5014378
:10D700000F00791E8F419DE71C000F00203CE74071
:10D71000202B03D04024E31A99400843411E88413E
:10D7200038437CE60022002425E6171A4346BA4215
:10D730009241591A5242891A6446350043E54146DE
:10D740001000144D10E680220024120380E61D0014
:10D750000F00203DEF40BC46202B03D04025EB1AA4
:10D760009940084307006346781E87411F4369E7D5
:10D77000871897429B4141445B42C9183500A3E595
:10D780003B003343CED0072231003A4052E600231B
:10D790001A00F4E5FF070000FFFF7FFFF0B55746D2
:10D7A000DE464E464546E0B5834607000E03480078
:10D7B00085B092461C00360B400DCD0F002800D1DD
:10D7C0009DE0954B984239D08023F6001B041E4300
:10D7D000924A7B0F33439946944603006344009377
:10D7E00000230026FF00029323031B0B98466300CF
:10D7F000E40F52465B0D019400D1B3E086498B42A1
:10D8000000D19EE04246D100802212040A435146D4
:10D81000490F11438B46814952468C460099634417
:10D82000CB1A0021D20000932B0063409A460F2EA2
:10D8300000D905E17A4BB6009B599F465B463343BE
:10D84000994600D0B8E002230826002700900293F2
:10D85000CAE7CB463A0002990195019B9A460229F4
:10D8600027D0032900D180E2012944D06D49009BD3
:10D870008C4663441C00002C38DD530700D013E2B3
:10D88000D2085B46DB0109D55946674B19408B46E8
:10D890008021C9008C46009B63441C00634B9C4262
:10D8A00007DC5B4664055F075B0217431B0B620DD9
:10D8B00002E000230027584A00211B031C0B0B0D1C
:10D8C0001B05234314055A4A380013401C43534692
:10D8D0006400DB0764081C43210005B03CBC904693
:10D8E0009946A246AB46F0BD0122524201231B1BC2
:10D8F000382B00DCADE1002200230027DCE75B468B
:10D90000334399465ED0002E00D18AE13000FEF705
:10D910002BFD03000B3B1C2B00DD7BE11D22D31AEA
:10D920005A460100DA4008398E4013005F463343FF
:10D9300099468F403F4B00261B1A00930023029309
:10D9400052E7414653460B433B499B468C46009B5E
:10D95000634400935B46002B3BD1022300221E430D
:10D96000022161E7434613439B4637D04346002BD1
:10D9700000D162E14046FEF7F7FC03000B3B1C2B95
:10D9800000DD53E102004146083A914088461D21DE
:10D99000CB1A5146D9400B0041460B439B46534698
:10D9A00093401A00009B25499C46604403008C4626
:10D9B00063440093002137E70323B14600900C260F
:10D9C000029311E7002300930133042600270293FA
:10D9D0000AE70323C3461E43032125E701331E4301
:10D9E0000022012120E700239A46802300271B0301
:10D9F000094A61E7802349461B03194200D1E2E04E
:10DA00005946194200D0DEE00B431B0317001B0BE5
:10DA1000A246014A50E7C046FF07000001FCFFFF95
:10DA200044FA0000FF030000FFFFFFFEFE070000B6
:10DA3000FFFF0F800DFCFFFF01F8FFFFF303000065
:10DA4000D94500D9CBE000D1C6E03C0048460027CC
:10DA5000009B013B00935B46160E1B021E43130204
:10DA6000984633041B0C9946310C0191FEF788FB54
:10DA70004A4642430B04210C050019438A4207D948
:10DA80008919013D8E4203D88A4201D9851E891920
:10DA9000881A0199FEF774FB09048C464A46210452
:10DAA00064464243090C030021438A4204D9891980
:10DAB000013B8E4200D8F1E02D041D43AB464346A6
:10DAC000891A4246280C12041D0C5B46140C2200D5
:10DAD0001B041B0C5A4303946B4344430295684355
:10DAE0001B19150CEB189C4203D980246402A44630
:10DAF00060441C0C15041B042D0C20185D19814278
:10DB000077D373D00C1AA24A7D1BAF42BF41944613
:10DB1000009B7F426344E01B1C00864200D1DBE097
:10DB20000199FEF72DFB4A4642430B04290C0700DE
:10DB300019438A4207D98919013F8E4203D88A4284
:10DB400001D9871E8919881A0199FEF719FB090462
:10DB50004A46894629044D464243090C030029439D
:10DB60008A4207D98919013B8E4203D88A4201D9DA
:10DB7000831E89193F04891A3A00039F1A4338000B
:10DB800013041B0C584381460298150C6F43434302
:10DB900045434846000C8446DB1963449F4203D941
:10DBA000802040028446654448461F0C00041B0444
:10DBB000000C7D191818A94200D284E000D17FE042
:10DBC00001231A4357E680234A461B0313431B03D2
:10DBD0001B0BAA466F4A6FE6BA4200D935E74B469F
:10DBE000DC0758087B081C43FF0734E70024AF42DA
:10DBF00089D247444745A4415B466442A41964184E
:10DC0000013BA6421ED2A0426DD800D1B6E0241A34
:10DC10009B4678E703005A46283B9A4000279146E6
:10DC200088E65846FEF7A0FB203072E60300524615
:10DC3000283B9A4093460022B4E65046FEF794FBF8
:10DC400020309AE6A642E2D1B845DCD9341A9B4688
:10DC500059E71F2B65DC504C0099A4465C46614493
:10DC600008008C4011008240D940501E82410C4374
:10DC700014435A46DA401300620709D00F222240AB
:10DC8000042A05D02200141D9442894149425B18A0
:10DC90001A0262D50122002300270DE68A4200D82D
:10DCA0000AE7831E891907E70F231340042B00D1CD
:10DCB000E6E5171D9742924153429B44FA08E0E57E
:10DCC000002800D1D7E57118531EB14227D3A942CD
:10DCD00015D358D01A0073E7002B00DC04E60123AB
:10DCE00000229B44CDE502234744474589415B42DE
:10DCF0009C46494289190C19E344241A03E7434618
:10DD00005F0047459B41B8465B429E19023A89191C
:10DD1000A94200D054E7404500D051E7ABE51A00D6
:10DD2000F6E71F215F4649420C1BE740202B07D036
:10DD30001A49009B8C46634418005B4683401A4393
:10DD4000501E82413A4307270023174009D00F2174
:10DD5000002311401400042995D122005F075B02C3
:10DD60001B0BD20817430022A6E5802359461B034C
:10DD70000B431B0317001B0B064A9DE5BD42B2D89F
:10DD80009B460024BFE68045B9D31A00C3E7C046CE
:10DD9000FF030000FF0700001E0400003E04000017
:10DDA000F0B54F464646D6468446C0B58046194E25
:10DDB00018030F034D00000B5C0082463F0B6D0DF6
:10DDC000C90F9146640DDB0F0120B5420AD0B44261
:10DDD00003D0A54201D157450CD01CBC90469946B2
:10DDE000A246F0BD66463E43F7D1AC42F5D154465B
:10DDF0001443F2D10120C845EFD1994207D0002D3C
:10DE0000EBD163461F433800471EB841E5E70020C9
:10DE1000E3E7C046FF070000F0B54F464646D6464A
:10DE20004D00C0B50E03C90F8A462C491F035C0084
:10DE30008046360B6D0D91463F0B640DDB0F8D4216
:10DE40001ED08C4216D0002D1ED130438446002CAB
:10DE500001D13A4323D06246002A1AD09A4529D0EC
:10DE6000514602200139084001381CBC90469946B1
:10DE7000A246F0BD39001143E5D002204042F4E74C
:10DE80003043FAD1AC420FD0002C0FD13A43E7D047
:10DE90000CE00122013B934318000130E5E76346A3
:10DEA0000020002BE1D0DBE73A43E6D19A45D7D1F9
:10DEB000A542D5DCA54205DBBE42D1D808D0002062
:10DEC000BE42D2D250460123013898430130CCE7FC
:10DED000C845C5D80020C845F4D3C6E7FF070000F1
:10DEE000F0B54F464646D6464D00C0B50E03C90FA5
:10DEF0008A462E491F035C008046360B6D0D914605
:10DF00003F0B640DDB0F8D4218D08C4211D0002DD9
:10DF100018D130438446002C1ED13A431CD16346AD
:10DF20000020002B30D05146022001390840013832
:10DF30002AE039001143EAD0022025E03043FBD12A
:10DF4000AC4226D0002C26D13A4324D1514602209F
:10DF500001390840013817E06246002A0FD09A457F
:10DF6000E1D1A54205DBBE42DDD819D00020BE427A
:10DF70000AD25046012301389843013004E00122BF
:10DF8000013B9343180001301CBC90469946A246C1
:10DF9000F0BD3A43D0D19A45C5D1A542C3DCE0E7F4
:10DFA000C845C0D80020C845E3D3EDE7FF0700000F
:10DFB000F0B55746DE464E464546E0B58346060078
:10DFC0000F03480087B092461D003F0B400DCC0F59
:10DFD000002800D16FE0DE4B984238D08023FF004C
:10DFE0001B041F43730F3B430193DA4B00279946F1
:10DFF00000239B46F60081442B0369001B0B52460D
:10E000009846490DED0F002900D185E0D04B99428B
:10E0100000D173E04346DA0080231B0413435246C9
:10E02000CC48520F84461343524600206144D2002C
:10E0300089442100694000918C46012149448A4667
:10E040000F2F00D990E0C449BF00CF59BF465B46AF
:10E050003B43019300D06AE1022308270026814652
:10E060009B46C9E732005846019B61460091022851
:10E0700000D175E0032800D1FEE1012800D02CE199
:10E0800000230027002600253F032A0D3F0BB3483D
:10E0900012053A4302401B051343009A5B00D10767
:10E0A0005B080B433000190007B03CBC9046994612
:10E0B000A246AB46F0BD5B463B43019300D12FE146
:10E0C000002F00D1A5E13800FEF74EF903000B3B0D
:10E0D0001C2B00DD96E11D22D31A5A460100DA40BE
:10E0E0005E4608398F4013008E403B4301939C4BA2
:10E0F00000271B1A994600239B467DE7414653465D
:10E100000B4393498C46E144002B00D01AE10222D4
:10E110000220174300228CE7134300D10DE1434650
:10E12000002B00D181E14046FEF71EF902000B3AB8
:10E130001C2A00DD72E10100434608398B409846F5
:10E140001D239A1A5346D3401A004346134352469E
:10E150008A404946081A824989468144002068E776
:10E160007B4B002700268EE7140C1204120C1100C2
:10E17000370C3604350C794328008C462E0060435A
:10E180006044834656432100300C8046584679430C
:10E1900040440291844506D98846802149028C4634
:10E1A000E044414602913604010C360C00048B46D3
:10E1B00081191E0C1B041B0C0391190079438C461A
:10E1C000280075436544A8465843050C45447743E9
:10E1D000A94203D9802149028C466744290C8C4608
:10E1E00039000004000C2D042D186144AB44059146
:10E1F0005946049101990F043F0C080C3900514312
:10E200004243904602008C46090C8B4662437C4395
:10E2100044445C44A04503D98021490288464244D5
:10E22000210C884661460904090C8C463900594383
:10E23000434370437E430F0CF6182404BE19644414
:10E2400042448C46B34203D980235B029846404443
:10E25000029B61469846049B370443449B46AB456A
:10E26000AD416B420D0405992D0C8C467F19674416
:10E27000FD18A8465D462D19A542A4419346644267
:10E28000A446C344DC448F42BF4198459B4193451B
:10E290009241A445A4415B427F421F43360C524247
:10E2A0006442BF192243BF18624638184302D20D98
:10E2B000039913436A020A43501E82416146ED0DE1
:10E2C0002A434E023243D90100D4B3E0012650085C
:10E2D00032400243DE0732435B08224C5444002C98
:10E2E00062DD510709D00F201040042805D0101D11
:10E2F0009042924152429B180200D90104D58024D9
:10E300001948E400034054441848844200DD27E7DC
:10E310005E075B02D2081F0B630516435B0DB2E676
:10E32000002399460133042700269B4664E6032315
:10E33000019781460C279B465EE601220120174388
:10E34000002276E6032303201F43434671E6C046BE
:10E35000FF07000001FCFFFF84FA0000FFFF0F80B1
:10E360000DFCFFFFFF030000FFFFFFFEFE070000A4
:10E370000023802700933F030026434B83E6019B45
:10E380003200A446584670E6AC466EE680270199F6
:10E390003F0339422DD03B422BD11F433F033F0B5C
:10E3A00000951600384B6EE601252D1B382D00DD3B
:10E3B00066E61F2D40DC35481C00504416008240A4
:10E3C0008440EE40501E824134431443EB406207C8
:10E3D00009D00F222240042A05D02200141D9442A5
:10E3E000804140421B181A023ED501230027002617
:10E3F00049E68027019B3F031F433F033F0B0094E7
:10E40000214B40E603005A46283B9A4000260192E1
:10E410006DE65846FDF7A8FF203057E60300524648
:10E42000283B9A401300002293E65046FDF79CFFDC
:10E4300020307BE6CA4650E71F201E004042041BE6
:10E44000E640202D03D0124C5444A3401A43501EE2
:10E450008241324307260027164009D00F200023AF
:10E46000104014000428B9D122005E075B021F0B84
:10E47000D2081643002306E680273F031F433F03CD
:10E480003F0B1600004BFEE5FF0700001E040000D6
:10E490003E040000F8B557464E464546DE460C00A1
:10E4A0000903E0B5490A460F5F0031431E03DB0F45
:10E4B000760A9B46530F3343C84E6500C000E40FF5
:10E4C000D2006D0DA24681467F0D9C469046B74214
:10E4D00000D1B9E05B46012673409B46EE1BA34585
:10E4E00000D183E0002E63DD002F00D0B1E0634651
:10E4F000134300D123E1731E002B00D0BAE1861A2A
:10E500006346B04280410125C91A4042091A0B02F4
:10E5100000D447E149024B0A98464346002B00D1FC
:10E5200089E14046FDF720FF0300083B1F2B00DD7B
:10E530007CE120223000D21A4146D04099400200AE
:10E540009E400A439D4200DD6AE15D1B6B1C1F2B50
:10E5500000DD94E1202110003500C91A8E40DA4018
:10E560008840DD40711E8E4111000722284300259E
:10E5700006433240002A09D00F233340042B05D034
:10E58000331DB342B641764289191E000B0200D4F6
:10E590003DE26A1C914B55056D0D9A4200D119E17F
:10E5A0008F4AF6080A40570752023743120B9BE086
:10E5B000002E00D0C5E06E1C7605760D012E00DC25
:10E5C00048E16746861ACB1BB042BF417F42B8463E
:10E5D0001F004346FF1A3B00B8461B0200D55FE10F
:10E5E00037439AD100220024002579E0002E00DC78
:10E5F000FAE0002F00D18DE0784B9D4267D0802358
:10E6000067461B041F43BC46382E00DC52E16346BC
:10E6100013435A1E93411E188642804140420918F6
:10E620000B0200D4BEE06D4B01359D4200D1D2E01B
:10E630006B4A73080A4001210E401E435108D3075C
:10E6400007221E43324095E71E00164300D045E7DF
:10E6500040E7624B9D423AD0802367461B041F432C
:10E66000BC46382E00DDEBE01F2E00DC3AE1330023
:10E670006746203BDF403B00202E05D04027BF1BD4
:10E680006646BE40324390464646721E964133432C
:10E69000DAE0002B00D114E26346134300D168E1B5
:10E6A00080234E07C008C9081B030643194208D03F
:10E6B0006046C008184204D163460100D2085E07D4
:10E6C0001643F3009946C900720F444D11434B465F
:10E6D000DE08424B4F073743CA089D4200D16EE027
:10E6E00012036D05120B6D0D00211203130B0A0DA1
:10E6F00012051A433B4B2D0513402B435B00E407E7
:10E700005B082343380019003CBC90469946A2465A
:10E71000AB46F8BD6346134311D0731E002B00D0E7
:10E7200007E186188642804161444042091801256C
:10E730000B0237D502257BE73E0061469146350046
:10E74000C5E75C46002D00D0E1E00B000343F3D0A9
:10E75000731C00D1ACE1214B9F4200D13AE1F3435D
:10E76000382B00DD6FE11F2B00DD8CE120250E0032
:10E77000ED1AAE40B0460600AA46DE404546354397
:10E780002E005546D940A8406346451EA8415B1A55
:10E790009C463043161AB242924163465242991A3D
:10E7A0003D00B4E607223240002A00D0E4E60B4BDD
:10E7B000F6084F073743CA089D4200D090E73B0058
:10E7C000134300D1A6E180231B031A431203120B4B
:10E7D000024D89E715000022002785E7FF070000AA
:10E7E000FFFF7FFFFFFF0F80002E00D0C7E06B1CF4
:10E7F0005E05760D012E00DCF0E0C84DAB4200D185
:10E80000B9E085180A00854289416244494251189D
:10E810000722CE076D082E43490832401D00A9E6A5
:10E82000BF49ED1A114007223240A3E632002838D2
:10E830008240002686E63000FDF796FD203073E624
:10E84000634613435A1E9341C61AB0428041404268
:10E85000091A5CE60E00674606431743002D5ED199
:10E86000002E00D0F3E0002F00D11EE15C4661468F
:10E8700091462CE7A94FBE427BD01E00F1E6100066
:10E880001F3DE840202B03D04021CB1A9A4016436D
:10E89000731E9E410722064332400021002583E774
:10E8A000161A6346B2428041591A40420B1A9846E2
:10E8B0005C4632E61F2E00DDABE02027BB1B9A46EC
:10E8C00063465746BB40994613004F46F3401F43EB
:10E8D0003B005746BA40571EBA4113436246F240C6
:10E8E000891898E62027BB1B9A4663465746BB40CB
:10E8F000994613004F46F3401F433B005746BA402A
:10E90000571EBA4113436246F240891A9CE7834B73
:10E910009F425FD080252D047342294320E7002EBB
:10E920000CD1002F00D1D0E05C46614691467B4D72
:10E93000CDE67A4FBE421CD01E0065E6002F18D0EF
:10E94000C0084E0706438020C9080003014208D0D2
:10E950006346DC08044204D12100DA46D2085E078F
:10E960001643F300994601245346C900720F114320
:10E970001C406A4DABE61D0000220027B4E6002DC6
:10E9800059D10B00034300D1D6E6731C00D1B2E08D
:10E99000624B9F421ED0F343382B6FDC1F2B00DDF0
:10E9A00097E020250E00ED1AAE40B0460600AA46BC
:10E9B000DE40454635432E005546A840D940451E09
:10E9C000A8418C440643B618964292415142614494
:10E9D0003D0025E63D006146914678E60B00034385
:10E9E000002D00D055E6002BF5D06346134300D12F
:10E9F0006DE6861886428041614440420918002233
:10EA00000B0200D4D0E6464B01351940B2E5B146C1
:10EA10005DE633006746203BDF403B00202E05D0FB
:10EA20004027BF1B6646BE40324390464646721E94
:10EA300096413343EFE5394B9F42CBD080252D04DF
:10EA400073422943A8E70843411E8841A2E6002FEC
:10EA500000D13CE66346861ACF1AB0429B415B4226
:10EA6000FB1A98461B024ED5161A6346B2429241D3
:10EA7000591A5242891A5C4600227BE501430E0076
:10EA8000711E8E419FE71D000E00203DEE40B046F6
:10EA9000202B04D04025EB1A994008438146484674
:10EAA0004346411E8841184374E60022002417E6BD
:10EAB000161A6346B2429241591A5242891A3D00CF
:10EAC00025E561469146154D01E68022002412039A
:10EAD00079E61D000E00203DEE40B046202B04D00C
:10EAE0004025EB1A9940084381464E464346711E25
:10EAF0008E411E4367E7861896429B4161445B4204
:10EB0000C9183D008CE547463743CED00722414621
:10EB1000324049E600273A00E6E5C046FF0700001C
:10EB2000FFFF7FFF30B5144D0A034B00120B5B0D46
:10EB3000C90F0024AB4211DD104CA34210DC80242D
:10EB4000640322430E4CE41A1F2C0CDD0D48C31A3B
:10EB5000DA4013005C42002900D11C00200030BDC7
:10EB6000094BCC18FAE7094DE040AC4663449A40A3
:10EB700013000343EEE7C046FE0300001D0400003F
:10EB80003304000013040000FFFFFF7FEDFBFFFFD5
:10EB900070B500282DD0C317C5185D40C40F2800DC
:10EBA000FDF7E2FB154B1B1A5B055B0D0A2815DD13
:10EBB0000B38854000222D032D0B002110002D0362
:10EBC0000A0D2D0B12052A430D4D1B052A40134338
:10EBD0005B00E4075B082343190070BD02002900B5
:10EBE000153291400A000B21081AC5402D032D0B48
:10EBF000E3E70024002300250022DEE71E040000D6
:10EC0000FFFF0F8010B5041E25D0FDF7ADFB144BA0
:10EC10001B1A5B055B0D0A2812DD0B3884400022AD
:10EC20002403240B0021100024030A0D240B1205D9
:10EC300022430C4C1B05224013435B00590810BDB6
:10EC400002002100153291400A000B21081AC4402D
:10EC50002403240BE6E7002300240022E2E7C04659
:10EC60001E040000FFFF0F80A30000000000000052
:10EC7000FC3F0150FC3F0250FC3F0350008001501C
:10EC800000800250008003502024282C383C40444F
:10EC9000484C0207020802010003010903040204B0
:10ECA00002050305000600070008000A0100000035
:10ECB0000000E0FE422EE63F0000E0FE422EE6BFEE
:10ECC000763C7935EF39EA3D763C7935EF39EABD66
:10ECD000000000000000E03F000000000000E0BF76
:10ECE00000000000000000000000000000000080A4
:10ECF00000000040FB21F93F000000002D44743E5D
:10ED0000000000809846F83C0000006051CC783B41
:10ED100000000080831BF0390000004020257A3875
:10ED2000000000802282E336000000001DF36935F8
:10ED3000000000000000F03F000000000000F83F6D
:10ED4000000000000000000006D0CF43EBFD4C3E69
:10ED500000000000000000000000004003B8E23F97
:10ED60004FBB610567ACDD3F182D4454FB21E93FE3
:10ED70009BF681D20B73EF3F182D4454FB21F93FD2
:10ED8000E2652F227F2B7A3C075C143326A6813C58
:10ED9000BDCBF07A8807703C075C143326A6913C03
:10EDA000000000000000F87F000000000000F07F7D
:10EDB0000000000000000000000000000000000053
:10EDC000010000000000F03F8A1EBD726654B6408C
:10EDD0004E543EF2A6EFCCC078844D13BFE9CB4031
:10EDE0004FFA050429CCB8C06C5C8AE26E56944098
:10EDF000CC5CF6234F0B5BC0563BD76877D80440FA
:10EE0000AC5913DC0D687EBFA38C9F98E6E76C3E7F
:10EE10005610B1E5EB4731BE182D4454FB21094093
:10EE2000000000000000000000000000000024407E
:10EE3000000000000000000000000000FCF90000DD
:10EE400002FA000008FA00000EFA000014FA0000AE
:10EE50001AFA000020FA000026FA00002CFA00003E
:10EE600032FA000038FA00003EFA000006061038B8
:10EE70007C101010050554341C1615060611514A55
:10EE80002A2410060610242A4A5111080804423E7A
:10EE900002023E42200505007F3E1C080303403E5F
:10EEA00001070760584641465860040463554941CC
:10EEB000020225520505080C7E0C08050510307E5F
:10EEC000301006061010107C381004040404000EE4
:10EED0000505605068444005056000600060000260
:10EEE00001015F03030600060505147F147F140566
:10EEF00005042A7F2A1005052313086462050536D8
:10EF00004951225001010602023E410202413E05E2
:10EF1000054428102844050510107C1010020240FA
:10EF20003005051010101010020260600303601815
:10EF30000605053E5149453E050500427F40000556
:10EF400005625149494605052241494936050518DA
:10EF500014127F100505274545453905053C4A49EA
:10EF6000493005050171090503050536494949364A
:10EF70000505064949291E020242000202402205F7
:10EF8000050814142222050514141414140505226E
:10EF9000221414080505020151090608083C02392B
:10EFA00045453D417E05057E0909097E05057F49E8
:10EFB00049493605053E4141412205057F4141222F
:10EFC0001C05057F4949494105057F0909090105D6
:10EFD000053E4141513205057F0808087F03034182
:10EFE0007F410505304040403F05057F0814224120
:10EFF00005057F4040404005057F020C027F050566
:10F000007F0408107F05053E4141413E05057F090B
:10F0100009090605053E4151215E05057F091929AB
:10F020004605052649494932050501017F010105CB
:10F03000053F4040403F0505071860180705057F5C
:10F040002018207F05056314081463050503047860
:10F0500004030505615149454302027F410303064C
:10F0600018600202417F05050804020408050540F6
:10F070004040404002020204040420545478040436
:10F080007F44443804043844444404043844447FEE
:10F090000404385454580303087C0A040418A4A434
:10F0A0007C04047F0404780303447D400202847DD1
:10F0B00004047C10284401017F05057C0438047C8D
:10F0C00004047C0404780404384444380404FC44F4
:10F0D00044380404384444FC04047C080404050552
:10F0E00008545454200303047E4404043C40407CF0
:10F0F00005050C3040300C05053C403C403C050506
:10F100004464384C4404041CA0A07C030364544CA5
:10F1100081F800000000000087F8000000000000F7
:10F120008BF800000000000090F8000094F8000048
:10F1300098F80000000000009CF800009FF8000014
:10F14000A3F800005BF70000A8F80000AEF800008C
:10F15000B2F800005FF7000000000000B6F8000001
:10F16000BAF80000BEF80000BEF80000C4F80000C5
:10F17000C8F8000000FA0000CCF80000CEF800004B
:10F18000D0F80000ABF7000062F90000D2F80000F0
:10F19000D4F80000D6F80000D9F80000DBF8000031
:10F1A000DDF80000D7F80000BBF90000F5F9000019
:10F1B000FAF9000000000000DFF80000E3F80000AA
:10F1C000E7F8000000000000E9F80000F1F8000096
:10F1D00092F800000000000000000000F5F80000B8
:10F1E000FCF80000F9F80000FEF8000008F9000043
:10F1F00049F900000000000012F900001AF90000AF
:10F2000048F70000AEF60000AEF6000023F900005B
:10F210002AF9000031F9000034F900001FF900005C
:10F2200057F7000037F900003BF9000046F70000EF
:10F2300053F7000041F9000046F9000042F70000D2
:10F240004FF700004BF9000050F9000058F900009A
:10F250005AF900000000000000000000000000005B
:10F2600060F900000000000064F9000068F9000087
:10F270006EF900000000000071F9000074F9000050
:10F280007AF900007EF90000A6F6000082F900007D
:10F2900094F900000000000088F900008DF90000DA
:10F2A00093F9000096F9000096F900009DF900001E
:10F2B0009FF90000A3F90000A8F90000ABF90000D5
:10F2C000BEF90000AEF90000B4F90000B7F9000083
:10F2D00047F90000BAF90000BDF90000C2F90000CA
:10F2E000C5F90000CAF90000CFF9000000000000D5
:10F2F00000000000D4F90000D9F90000DEF9000098
:10F30000E3F90000E8F90000EDF90000F2F900006F
:10F31000F7F90000000000008D7E000001B200003F
:10F32000E1540000757D0000C554000049B10000A3
:10F33000A59B0000357D0000A95400000564000075
:10F34000217A0000D57C0000A1960000B163000086
:10F35000F9770000717C000051970000ED8E0000ED
:10F36000F57200006164000011820000118200004B
:10F37000FD5A0000C59C0000B35B0000A95B0000C3
:10F380008B5B00006D5B0000355B00009F5B000045
:10F39000815B0000635B000029710000955B000049
:10F3A000775B0000595B0000C97000002972000003
:10F3B00089720000DD7B00008D7E00002DB2000010
:10F3C000F9A300003DA5000000000000657F0000DB
:10F3D0008D54000033A5000000000000CD91000016
:10F3E0006D54000029A50000BD6E0000197F0000CB
:10F3F000018500001FA500005D540000615600005B
:10F400002D83000015A500004D8E00004D8E0000DC
:10F410007D5400007D530000156E00005F54000015
:10F420003194000019960000716C0000B16F00006B
:10F43000499300009195000031620000356F000093
:10F4400061920000FD940000156C000071630000E3
:10F450004DB200001DB300008D7E000095680000D5
:10F46000E9530000C56B000000000000915300004C
:10F47000D1530000856B000000000000C96100004E
:10F48000B9690000FD6A0000E9660000B18800006B
:10F490001D690000A96A00007F530000595F000049
:10F4A000BD680000496A00009161000091610000A0
:10F4B000F5610000156A0000016100008153000041
:10F4C0002D9100004D540000CD5F000099670000B1
:10F4D000859000003D540000E96500004167000090
:10F4E000ED8F00002D5400003965000035800000CC
:10F4F000AD53000009540000A5980000F9980000E1
:10F500004D990000B1990000159A00005D9A000025
:10F51000A59A0000F99A0000FB21F93FFB21094060
:10F520007CD91240FB2119407A6A1F407CD92240C5
:10F53000BBFD2540FB2129403A462C407A6A2F40EA
:10F540005C4731407CD932409C6B3440BBFD354038
:10F55000DB8F3740FB2139401BB43A403A463C40F0
:10F560005AD83D407A6A3F404C7E40405C4741401B
:10F570006C1042407CD942408CA243409C6B44407A
:10F58000AC344540BBFD4540CBC64640DB8F4740D1
:10F59000EB584840FB21494083F9A200444E6E00DD
:10F5A000FC291500D1572700DD34F50062DBC000CF
:10F5B0003C999500419043006351FE00BBDEAB00D7
:10F5C000B761C5003A6E2400D24D42004906E00002
:10F5D00009EA2E001C92D100EB1DFE0029B11C008F
:10F5E000E83EA700F535820044BB2E009CE984006C
:10F5F000B4267000417E5F00D691390053833900F4
:10F600009CF439008B5F840028F9BD00F81F3B0093
:10F61000DEFF97000F980500112FEF000A5A8B00AC
:10F620006D1F6D00CF7E360009CB2700464FB70017
:10F630009E663F002DEA5F00BA277500E5EBC70024
:10F640003D7BF100F739070092528A00FB6BEA001C
:10F650001FB15F00085D8D00300356007BFC460043
:10F66000F0AB6B0020BCCF0036F49A00E3A91D007C
:10F670005E619100081BE60085996500A0145F009B
:10F680008D40680080D8FF0027734D0006063100CA
:10F69000CA561500C9A873007BE260006B8CC000DD
:10F6A000544553543A00524E4400286929005241AF
:10F6B0004E202300257500256425732025733F0007
:10F6C0002564257320257320257300256425732068
:10F6D0002573004E414E002D494E46002E25253003
:10F6E00025646C6C7500256C6C75002045256400E4
:10F6F000257325632573002573202025632573005A
:10F700002573202B25732025630025732025732066
:10F71000256300436865636B20466C61673A00436C
:10F720006C65617220466C61673A005365742046CF
:10F730006C61673A0044656C657465205072676D52
:10F740003A004953470044534500582019200045CA
:10F750004E4700534349004649580053544F005206
:10F76000434C00476F20546F204C424C3A004754A2
:10F770004F204C424C3A00476F20546F204C696E2A
:10F78000653A00257320005F0050726F6772616DEB
:10F790002025630050726F6772616D2025640052EE
:10F7A000756E6E696E67002E202E202E00593A006D
:10F7B000583A0044697669646520627920300049CE
:10F7C0006E76616C69642074797065004E6F206C90
:10F7D0006162656C004C6162656C20657869737468
:10F7E00073004F7574206F66204D656D004D617814
:10F7F00020497465727320526561636865640055C1
:10F800007365722061626F72746564004E6F20725E
:10F810006F6F740041626F72740068006825630046
:10F8200066007261640067720020100020500020A2
:10F830001C2000201020005069636B204C424C3A81
:10F840000052756E204C424C3A00475342204C42C5
:10F850004C3A00494E54454752415445204C424C85
:10F860003A00534F4C5645204C424C3A00256420F8
:10F87000005061737465204D656D6F72793A0D0AA1
:10F8800000456D70747900522F530053515254004B
:10F890004753420047544F00655E5800521B0053C7
:10F8A000494E0031305E5800582019205900434F0E
:10F8B0005300595E580054414E00312F5800454EB8
:10F8C0005445520045455800434853003100340028
:10F8D000370035003800182B00330036003900504F
:10F8E0005345004C424C004100434C4541522018C6
:10F8F000004859500044494D004652414300434C92
:10F900004541522052454700436F6D7020636F6E32
:10F910006A0072756E54696D650059202B20695814
:10F92000201900524553554C54004D4154524958EA
:10F93000007821001C5200792C72001C482E4D5377
:10F94000004C2E522E001C5241440050792C78005D
:10F950005265201920496D001600534F4C56450042
:10F96000585E320052544E00485950201D004C4EF3
:10F9700000521A0053494E201D004C4F4700494E7B
:10F980005400434F53201D00434C20580054414E17
:10F99000201D001725004C415354205800140041ED
:10F9A0004253004D45414E001C50005346005354F5
:10F9B000444556001C4800434600182D001C444591
:10F9C0004700463F00475241440043792C78005499
:10F9D0004553540053544F2B0053544F2D00535450
:10F9E0004F2A0053544F2F0052434C2B0052434C8C
:10F9F0002D0052434C2A0052434C2F005820112016
:10FA0000300058203E20300058203C203000582044
:10FA10001220300058201320300058203D2059007B
:10FA200058201120590058203E20590058203C20D1
:10FA300059005820122059005820132059005820EE
:10FA40003D20300040DA0000B2D80000F6D80000B7
:10FA50005AD80000F6D80000E6D90000F6D8000019
:10FA60005AD80000B2D80000B2D80000E6D9000091
:10FA70005AD8000052D8000052D8000052D80000D6
:10FA8000F4D9000068E100006AE000006AE00000CC
:10FA900088E3000064E0000064E0000070E3000020
:10FAA00088E3000064E0000070E3000064E0000010
:10FAB00088E300007EE300007EE300007EE30000B8
:04FAC0008CE30000D3
:08FAC40008C7FF7F01000000EC
:10FACC000508107A6CEE00004D000000583A001F3B
:08FADC002C000000C400001022
:040000030000C03108
:00000001FF
